:020000024000BC
:100000006FD0626900000000001801180028012864
:100010000228032800290129022903290429052986
:10002000062907290829002A012A022A032A042A64
:10003000052AA62AB4E206000A4304006804002048
:10004000EA040020EA030020B80300205003002047
:10005000062A0020A2430400C44404005A470400B6
:10006000744804006242040010420400B4020020FC
:1000700054020020384D0400640800207843040036
:100080003E4A04006C7C0600527E0600B87E0600E4
:10009000025906003C59060084880500527D05007F
:1000A000427706006C4A04003660060032FC040009
:1000B000C0FC04001EFD04003C5504007A550400F9
:1000C000F053040040BE040026B90400282B002091
:1000D00064CA0400B6CD0400C8AB04006AAB0400D7
:1000E00036AF040014AC040048AB0400C0AB0400FD
:1000F000FEAA040096AC0400EEAC04009EAC040022
:10010000A2AC040030AD0400F6AC040026AD04003F
:1001100008B204000CB2040092AC04009AAC0400D3
:100120002EAD04000AB20400DCAD040068B3040084
:1001300064DB0400D6DB040010DC040086C004008D
:100140009CC00400D6C00400E2A00400E8A20400A1
:10015000B0A30400DC720400266D0400E0960400E5
:10016000A26D040096920400B8BB0600EEB3060030
:10017000F4B806006CD0060036CF06008ED3060019
:100180004AD3060086D30600DAD40600AAA20600E7
:100190006AD40600C8C60600EEC606000EC70600F2
:1001A0004AD506002ACD0600C2CC0600BAD5060004
:1001B0002EA50600C6A50600E6A5060098A5060021
:1001C0008C600500CA4A0500624E0500064C050019
:1001D000A4560500C03D0020DA760600DEA2060027
:1001E000C64E0400525A0600166006000E61060054
:1001F0001C6F0600A46F06000271060040C40400D4
:100200008E5F05004C5705009A480500FA59050015
:100210007A4A05002A0A00202A5B0600B4D30600A9
:100220004ED3060082D306007ED30600DA460400D1
:10023000BEC10400BCD306009263060058640600E9
:10024000C06406005CB90600B8D3060002D40600FC
:10025000D47C050006D406004E2000201420002087
:100260003CB90600D2BA06000AD406005ED40600E5
:1002700062D40600C0D30600FAD30600FED30600FF
:1002800066D4060044600500000000000000000085
:10029000000000000000000000000000000000005E
:1002A000000000000000000000000000000000004E
:1002B000000000000000000000000000000000003E
:1002C00097470000938707F41747000013078777C5
:1002D0006373F700828023A007009107D5BF97477B
:1002E00000009387A7E417E706E013072765974602
:1002F0000000938626F163F3F60082801043110715
:0603000090C39107CDBF80
:100308004111B7E700E022C480433707200006C642
:10031800798C23A0E7180F10000011C199E5B7E701
:1003280000E023A08710014579A80D05334505088D
:10033800130740037199B34705086366A702174579
:100348000000032525EC9746000083A626EB639161
:10035800A602174700000327A70D71D3C207DD8D3A
:10036800054502976DBF17450000032565E9E1BF04
:100378007A2131EF5A21636CF704B306F74021481C
:1003880017460000130646056375D8028328050042
:1003980003586600938687001D8FAA966117DAA214
:1003A80023A016012393060014C15EA1130788FF3A
:1003B8007AA27A226EA12105B307F7407EA2B7E799
:1003C80000E023A08710B240224441018280084106
:1003D800BDBFB7E700E08C433707200023A0E7182C
:1003E800F98D0F10000001E523A0B7108280174394
:1003F8000000032323E19748000083A828E09A8798
:10040800814663FE170903A80700636DF508636B4F
:10041800A808138787006364E508F22321670507A6
:100428006319E60017460000130636EC1822050784
:1004380018A217450000130525FAD2237A21239321
:1004480007003297334707087AA163856702174385
:1004580000000323E3DA630FF30003D36600631B92
:100468000300DE2223A0060121073E962106D2A220
:100478007AA1B6879843630417039746000083A6BA
:1004880026D8630ED700762399EAD6235223184339
:10049800A106B296D6A398C37E21A1077EA1B7E78D
:1004A80000E099B7BE86C287A9BFAA871747000090
:1004B800032747D517460000032646D4B305B540A1
:1004C8006314E6003E8529A8930687001843E3E9EC
:1004D800D7FEE3F7E7FE2E85E3E4D5FEE3F2E5FE7B
:1004E800828023AC05FE1C4199E30CC182803E87C3
:1004F80083A787FFEDFF232CB7FE8280411126C218
:10050800B7E400E04AC003A90400B707200006C604
:1005180022C43379F90023A0F4180F10000009E56C
:1005280023A0241101452DA09565938505D0C98D7B
:100538002A842105B3C5050833450508D1336DD193
:10054800FD572320050042A17CA123A024112105E9
:10055800B240224492440249410182804111B7E7E6
:1005680000E04AC003A9070026C23707200006C6D4
:1005780022C4AA843379E90023A0E7180F100000E9
:100588009747000083A747C80144014695E311C86F
:10059800A28517450000130525C7974004E0E780AA
:1005A80000F0A1652685974004E0E780C0451DA0BE
:1005B80003C7E7FF631B970215CCA2851745000008
:1005C800130585C4974004E0E78060EDA1652685A2
:1005D800EF20E06DB24022852244B7E700E023A077
:1005E8002711924402494101828011E03E8683A787
:1005F80087FF69BF3E84E5BF37E700E01C43B706C5
:1006080020002320D718F58F0F10000019C191C1C1
:1006180011E637E700E02320F71082802E960F704E
:10062800B650D5BF37E700E01C43B70620002320AB
:10063800D718F58F0F10000019C1014785E137E77A
:1006480000E02320F7108280B386E50003A80600A7
:10065800B306E5007D1623A00601110775F6C5B798
:1006680037E700E01C43B70620002320D718F58F92
:100678000F10000001C53307C50011E637E700E099
:100688002320F71082800505A30FB5FEE31DE5FEC4
:10069800F5B7B7E600E09C42370620002A87F18FBD
:1006A80023A0C6180F1000000145B306A7008386D3
:1006B800060091E637E700E02320F7108280050561
:1006C800EDB70111B7E700E026CA84434AC83707E7
:1006D800200006CE22CC2A892E86F98C23A0E71882
:1006E8000F1000009305F00432C633450608093997
:1006F8002A8401C53246CA850137F2402285624400
:10070800B7E700E023A097104249D24405618280F0
:1007180037E700E01C43B70620002320D718F58FE1
:100728000F10000001C599C1014711EA37E700E041
:100738002320F710054582800507E309E6FE330804
:10074800E500B386E500034808009422E306D8FED6
:1007580037E700E02320F7100145828037E700E003
:100768001C43B70620002320D718F58F0F10000070
:100778001307F6FFBA952A966317C50037E700E016
:100788002320F71082809821FD150505A30FE5FEAB
:10079800E5B737E700E01C43B70620002320D71849
:1007A800F58F0F10000001C53307C50019E637E7BC
:1007B80000E02320F7100145828014210505E39805
:1007C800B6FEE31CE5FE37E700E02320F7100545F9
:1007D8008280797126D297440000938464A422D43D
:1007E800804006D64AD04ECE52CC56CA5AC85EC6AB
:1007F80062C455C437C9C901814B174B0000130B9C
:10080800ABA11309F937174A0000130A6ABF974AC0
:100818000000938A6ABC97490000938969C33E2007
:1008280091EF5C4463990B009CC0032CC4002285A3
:100838004D36628489A823A6FB00C5BF83270B0019
:1008480082971C443307F5406376F50003A78900B7
:100858001D8F2A976368E9062E200820EF2020457F
:100868005C405844A9CB0C44174600000326C6BE7A
:10087800AE97BE8663E4B70063E4C700B386C7409B
:1008880014C4A28B3A8441FC174700000327C7B55C
:10089800894763E6E7009747000023A707B4B250EB
:1008A800225492540259F249624AD24A424BB24BFC
:1008B800224C4561828063940B0098C0BDB723A683
:1008C800EB00A5B703274A021DCB63EDA7023385CA
:1008D800A7401C2099EF03479A0183A68900611756
:1008E800B307A7003E8563E4E70063E4D7003385D8
:1008F800D74083A70A016374F50023A8AA00A28B36
:10090800404451B703A78900BA97D1B7011126CA45
:1009180006CE974400009384A4B322CC4AC84EC69E
:1009280052C49C288844DDC3B7E700E003A9070048
:100938003707200023A0E7183379E9000F100000DB
:10094800174700000347C78C19CB23A02711F24093
:100958006244D2444249B249224A0561828017471B
:1009680000001307A7E08357C70AB1CB9C440324B0
:10097800870A6306F404974900009389E9A503A749
:1009880009012285630DF702174A0000130ACA8875
:1009980083270A008297636EA40C83270A00098CB8
:1009A800829783A7090198443354F40AB307A40033
:1009B8003E8563E4870063E4E7003385E740B7E7F3
:1009C80000E023A027119C44639DA7021744000060
:1009D800130484A018489747000083A7E783631D82
:1009E800A70882979444374736FE130707C83697F7
:1009F800B307A7003E8563E4E70063E4D7003385C7
:100A0800D74017440000130464F95C5C99CB9746FF
:100A1800000083A666939C463707CDFF7D17F98FA4
:100A28009CC611E1884485475CD09747000083A79E
:100A3800679F829715E15C5C99CF5C5089CF97607E
:100A480006E0E780A0B1975006E0E780602C974762
:100A5800000023A707F6B53B5C5CE38A07EE17475F
:100A680000000327678E1C47B7063300D58F1CC7C5
:100A7800F9BD9C443E9415B7829714489844B387AF
:100A8800A6003E8563E4D700E3EDE7F63385E7404B
:100A98008DBF9737000023ABA77611C58547173759
:100AA80000002307F7768280AA8799E51747000098
:100AB8000347079B09C7F1BF11476369B700174789
:100AC80000001307A797B3C5E5209CC1828097371C
:100AD800000083A7A77385C3411106C6829797377D
:100AE800000083C7E77289E79737000023A00772E1
:100AF800B240410182809737000083C7677191E750
:100B08009737000023A4077082808280411122C495
:100B180026C206C64AC097440000938424E883C7C7
:100B280034021744000013046491B9C71744000045
:100B38001304848A173900001309C96E03270900B2
:100B48001C2014300146B3A5E7208E21A5CD11C283
:100B58001CA00820636FD50697470000238E0786E0
:100B68009737000083A7476BC5EFB24022449244F1
:100B780002494101828082971C40F5FF9747000097
:100B880083C7078E85E3DC48858B89CFD84C994786
:100B9800631EF7009747000023AC07E0EF10B01979
:100BA8005C4482971C44D9D3829749B7D84C9D4757
:100BB800E31AF7FE9747000023AC07DEEF10B017E3
:100BC8001C48C5B7850793F7F70F0546E3EDD7F639
:100BD80041B73327E5200E2323100700973700007D
:100BE800239907629737000083A74763B347F52027
:100BF8009C4382971C20832609001737000003575F
:100C080047613377E540B3A6D7209222518F9AA245
:100C180099C385071CA018201C30E368F7F42DBF82
:100C28009747000083A747831CC8653683C73402EB
:100C38008DFF83C7140299CBDC4C89EB97470000E2
:100C4800A38E07D6975006E0E780C02B97370000A1
:100C580083A7477D99DB1C4889DB18308326090068
:100C6800814763C9E702D84C9147E3E0E7F097472B
:100C7800000083C7E7AD918BE39907EE9737000033
:100C880083C70759E39307EE2244B24092440249CE
:100C98004101ADB933A6D7201222E31806EC850727
:100CA800C9B7B7C700401387C7201443139626490E
:100CB80010C301000100938787261735000003251C
:100CC80065739C436A0514C393C7F7FF99835D8DC9
:100CD80082809737000083A7675591C382871305E1
:100CE800F00F82809737000023A2A754828017460E
:100CF8000000130626A3974600009386A6A4DC36B8
:100D0800383E4C4ABA97FD8B33D7F5001CB2DCB697
:100D1800058B0DE7943A13050002B3F7D702814615
:100D280033D8E548630908006394D70018B2828075
:100D3800850693F6F60F0507E314A7FE828097470A
:100D4800000083A7E7C6C1E741114AC097370000F2
:100D580083A7874C06C622C426C28297174900007B
:100D68001309499E83278900638DA7046363F504EB
:100D78001D8D974400009384E49ABC2C13545500AD
:100D88006361F404AD37BC2C0327890093965700A0
:100D980036971D8C2324E900E376F4FE224488303C
:100DA800B2409244024981454101173305E067008A
:100DB800C36B173700000327276AB307F7403E9530
:100DC8004DBFB24022449244024941018280828050
:100DD800011126CA9737000083A7074406CE22CC04
:100DE8004AC84EC652C4829797440000938484959B
:100DF8009844AA870145630DF70463E3E706998FD2
:100E0800174900001309099293F9F70113D4570001
:100E18008347A901636AF402173A0000130A4A6378
:100E2800F9350347A9018C4403268A009317570014
:100E3800AE97198CBE8663E4B70063E4C700B38637
:100E4800C74094C4E37EE4FC1315540033653501B0
:100E5800F2406244D2444249B249224A0561828042
:100E68009736000083A6465F3387E640BA9749BFA6
:100E7800411122C417440000130444B21C4426C282
:100E880006C6858B9744000083A4849491EBEF30C9
:100E980040072244B2402685924441016F10507F9A
:100EA80098289747000023AF07AE8947E301F7FE6C
:100EB8000146930550020145EF10F01A8145177558
:100EC80005E0130565F0CD36014681450545EF106F
:100ED800207F5C44858BC5DFB240224492444101A7
:100EE80082809747000083A76792639307180111D0
:100EF80022CC2A84094506CE26CA4AC84EC6EF30F7
:100F0800E008973900009389294303A6090093074D
:100F1800800717390000130929417CD29737000050
:100F28002388072E83270900973400009384C4413F
:100F3800B7053300D8572285719B13671700D8D798
:100F480098431377F7CF98C398431377F7CF13676E
:100F5800072098C398401447CD8E14C7B7060300DE
:100F68009386862534CA5457F59A54D7984334241F
:100F7800137707F893F6F607558F98C3EF20A00864
:100F880083A60900370500827D15DC4293E7170028
:100F9800DCC203260900030784065C569375F70331
:100FA800E605E98FCD8F5CD69305A0039C4063D5F9
:100FB800E508F84FB70500074D8FF8CFB7C7898EFA
:100FC800938767ED1CC6B7575500938757555CC282
:100FD8008347A40683444406DD8C894717470000ED
:100FE800232CF79C9747000023A0079C7C44BCDE79
:100FF8009737000083C7C74699C7FC52FDFF97473C
:10100800000023A1079A18289D478145172500004D
:101018001305A53F6306F70017050000130585E5CE
:10102800613410386244F2404249B249A685D2443C
:10103800014505616F10C0689305200263DAE50079
:10104800F84FB70500F9FD156D8FB7050005ADB769
:10105800B70500F96945FD156357E500F84F6D8F31
:10106800B705000391BFF84F6D8F13178729B1B7E4
:101078008280973700009387676FE85305475425A8
:101088006390E60203C747079147631AF700011107
:1010980006CE2AC6EF10905B3245F240056191B545
:1010A800828083278511E5CB411122C406C65825C5
:1010B8008345E5049437D2272A841377C70F1395FD
:1010C800466063F7C50663510506882793F6F60759
:1010D80094B70546936627006314C5009366170006
:1010E80054A4D8430907D8C3032504114CB82E8645
:1010F800CC430905EFF04FD0832784115438D843E7
:101108003697D8C3DA27158FDAA789473CBC034737
:1011180064039737000083C7C72F6369F706B24097
:1011280022440145410182801367170058A46DBF0E
:101138009376F60F635505028827854513662700C1
:101148006314B5001366170050A454B8A3840700AD
:1011580085473CBC832784119C43D5FBC9B71367DB
:10116800170058A454B8A384070003250411CC43DE
:101178000905EFF06FC8832784115438D843369790
:10118800D8C3DA27158FDAA78D47E1B75C2493E730
:1011980007015CA469B705458280411197370000B3
:1011A80083A7C71622C406C6858B2A84CDEB782967
:1011B8008357051D63E5E70A4165130525F59790F3
:1011C80005E0E780608E41CD3C253EA583270412CB
:1011D800ADE32320A4122322A41285472311F4048B
:1011E800232005007C2854415EA5583418A50547DE
:1011F80018B513851702173700000327E77D1581F7
:101208001C437D151375F50F9CC25C43DCC21C475B
:101218009CC65C47DCC61C4B9CCA5C4BDCCA1C4F9A
:101228009CCE5C4FDCCE0DC19386060213070702E5
:10123800C1BF8327441288C3835724042322A412DE
:101248008507B3C7070859BF1737000013070752A8
:101258001E2785071EA7B2402244410182805C24D4
:1012680023090400054593C747005CA4EDB7142D76
:10127800854763EED70A1C3D2A870145DDEB5C27CD
:1012880013F507013C2B99CB83466703973700007A
:1012980083C7371863ECF60001E5828059E5828040
:1012A8008357271E0357671EBA9721A08357271E07
:1012B80075F90145BDCF9387C7121735000003554F
:1012C800E519B3B5A70237460F00411113060624E6
:1012D800814622C426C206C67D543385A70297C01C
:1012E80006E0E780806E9734000083C4F412AA9465
:1012F8009737000083A7C75003A707099C433354B7
:10130800E40AFDFB9737000083A707F1829781471E
:101318006364A400B307A440B240224433B59700E5
:10132800134515009244410182808147A5BF0145BC
:101338008280828017370000032707003C5BFDFF8F
:1013480001000100828039C901116C0022CC06CE4F
:101358002A84EF20F00715C9FD57630DF502B2473F
:101368009735000083C5550B63EBB700034594021E
:101378006244F240B385B74005616F10F017173724
:1013880000000327670DBA97D5B76244F24005619C
:101398006F204047F2406244056182808280797103
:1013A80052CC173A0000130A6A3C26D283244A0911
:1013B80006D622D44AD04ECED5C897370000938798
:1013C800E75DD44F15476386E604DC532A8989CF45
:1013D800975006E0E7808018975006E0E780409332
:1013E8009737000023AE075CFD596C002685EF2077
:1013F800207E0DE91725000013050541EFF06FE980
:101408009737000083A747F33707100098C70547A9
:10141800B8DB0D45B250225492540259F249624A3F
:1014280045618280637435013244AA898440D5FCC1
:10143800FD571305F00FE38FF9FC914763F187021D
:101448009307B4FF2320F9002324FA0A99E7973772
:10145800000083A767002320F900014565BF97377F
:10146800000083A767FFED17A297E9BF09455DB79D
:10147800797126D206D622D44AD04ECE52CC56CA3C
:101488005AC85EC68347550303447513AA843E941D
:101498001374F40F9307400263F687001304B4FD36
:1014A8001374F40F03A9841383A9C413A38B8412A0
:1014B80022864A85CE8597C006E0E780404C05899C
:1014C80015E503CBD412014A814A337B6403930B9D
:1014D800500252864A85CE8597C006E0E780204AAA
:1014E80005890DC563916A031374FA0F238B84125F
:1014F800B250225492540259F249624AD24A424B9B
:10150800B24B45618280850A939A4A60050AE312C4
:101518007AFDE9BF8327850903560504797193D6B7
:101528000701BD8EB3C60608358E93575640898B82
:10153800135776485D8F93573640918B5D8F93573D
:101548001640A18B5D8F93171600C18B5D8F931783
:10155800360093F707025D8F9317560093F7070439
:101568005D8F9317760093F7F70F22D45D8F2A8447
:101578009357D6001355B6001189898B9355860069
:10158800C98F1355F6002582C98F218AD18F1396EA
:101598001500418AD18F1396350013760602D18F34
:1015A8001396550013760604D18F1396750013769B
:1015B800F60FD18FA207C5455D8F3307B70226D234
:1015C8004AD04ECE032984138329C4135AC806D699
:1015D80052CC56CA36973347070813565740098ADC
:1015E80093577748D18F13563740118AD18F1356A6
:1015F8001740218AD18F13161700418AD18F1316ED
:10160800370013760602D18F131657001376060497
:10161800D18F131677001376F60FD18F1358B700B2
:101628001356D70013784800098A13558700336684
:1016380006011358F700258333660601218B518F65
:1016480013161500418A518F1316350013760602BA
:10165800518F1316550013760604518F1316750013
:101668001376F60F518F2207D98FB387B7025EC65C
:10167800B697B3C7070813D55740098913D77748D2
:10168800498F13D537401189498F13D517402189C0
:10169800498F139517004189498F139537001375A2
:1016A8000502498F1395570013750504498F139543
:1016B80077001375F50F598D13D8B70013D7D700D6
:1016C80013784800098B13D687003367070113D8AE
:1016D800F700A58333670701A18BD98F131716006D
:1016E800418BD98F1317360013770702D98F131739
:1016F8005600137707041E06D98F1376F60FD18F7D
:10170800A2073367F5003307B702130650024A856C
:10171800CE853697B98EB3C4060833F6C402137B58
:10172800F60F97C006E0E7808025058905E9834A1A
:10173800D412014A930B5002B38A9A02814493DA75
:101748000A0126864A85CE8597C006E0E7802023D1
:1017580005890DC563914A0313FBF40F230B64132A
:10176800B250225492540259F249624AD24A424B28
:10177800B24B45618280050A137AFA0F8504E39219
:1017880074FDE9BF8327C50803568508797193D688
:101798000701BD8EB3C60608358E93575640898B10
:1017A800135776485D8F93573640918B5D8F9357CB
:1017B8001640A18B5D8F93171600C18B5D8F931711
:1017C800360093F707025D8F9317560093F70704C7
:1017D8005D8F9317760093F7F70F22D45D8F2A84D5
:1017E8009357D6001355B6001189898B93558600F7
:1017F800C98F1355F6002582C98F218AD18F139678
:101808001500418AD18F1396350013760602D18FC1
:101818001396550013760604D18F13967500137628
:10182800F60FD18FA207C5455D8F3307B70226D2C1
:101838004AD04ECE0329040A8329440A5AC806D638
:1018480052CC56CA36973347070813565740098A69
:1018580093577748D18F13563740118AD18F135633
:101868001740218AD18F13161700418AD18F13167A
:10187800370013760602D18F131657001376060425
:10188800D18F131677001376F60FD18F1358B70040
:101898001356D70013784800098A13558700336612
:1018A80006011358F700258333660601218B518FF3
:1018B80013161500418A518F131635001376060248
:1018C800518F1316550013760604518F13167500A1
:1018D8001376F60F518F2207D98FB387B7025EC6EA
:1018E800B697B3C7070813D55740098913D7774860
:1018F800498F13D537401189498F13D5174021894E
:10190800498F139517004189498F1395370013752F
:101918000502498F1395570013750504498F1395D0
:1019280077001375F50F598D13D8B70013D7D70063
:1019380013784800098B13D687003367070113D83B
:10194800F700A58333670701A18BD98F13171600FA
:10195800418BD98F1317360013770702D98F1317C6
:101968005600137707041E06D98F1376F60FD18F0A
:10197800A2073367F5003307B702130650024A85FA
:10198800CE853697B98EB3C4060833F6C402137BE6
:10199800F60F97C006E0E78080FE058905E9834ACF
:1019A8001408014A930B5002B38A9A02814493DACD
:1019B8000A0126864A85CE8597C006E0E78020FC86
:1019C80005890DC563914A0313FBF40F230F6407C0
:1019D800B250225492540259F249624AD24A424BB6
:1019E800B24B45618280050A137AFA0F8504E392A7
:1019F80074FDE9BF8327450903568508797193D695
:101A08000701BD8EB3C60608358E93575640898B9D
:101A1800135776485D8F93573640918B5D8F935758
:101A28001640A18B5D8F93171600C18B5D8F93179E
:101A3800360093F707025D8F9317560093F7070454
:101A48005D8F9317760093F7F70F22D45D8F2A8462
:101A58009357D6001355B6001189898B9355860084
:101A6800C98F1355F6002582C98F218AD18F139605
:101A78001500418AD18F1396350013760602D18F4F
:101A88001396550013760604D18F139675001376B6
:101A9800F60FD18FA207C5455D8F3307B70226D24F
:101AA8004AD04ECE0329040B8329440B5AC806D6C4
:101AB80052CC56CA36973347070813565740098AF7
:101AC80093577748D18F13563740118AD18F1356C1
:101AD8001740218AD18F13161700418AD18F131608
:101AE800370013760602D18F1316570013760604B3
:101AF800D18F131677001376F60FD18F1358B700CE
:101B08001356D70013784800098A1355870033669F
:101B180006011358F700258333660601218B518F80
:101B280013161500418A518F1316350013760602D5
:101B3800518F1316550013760604518F131675002E
:101B48001376F60F518F2207D98FB387B7025EC677
:101B5800B697B3C7070813D55740098913D77748ED
:101B6800498F13D537401189498F13D517402189DB
:101B7800498F139517004189498F139537001375BD
:101B88000502498F1395570013750504498F13955E
:101B980077001375F50F598D13D8B70013D7D700F1
:101BA80013784800098B13D687003367070113D8C9
:101BB800F700A58333670701A18BD98F1317160088
:101BC800418BD98F1317360013770702D98F131754
:101BD8005600137707041E06D98F1376F60FD18F98
:101BE800A2073367F5003307B702130650024A8588
:101BF800CE853697B98EB3C4060833F6C402137B74
:101C0800F60F97C006E0E78080D7058905E9834A83
:101C1800F408014A930B5002B38A9A02814493DA7A
:101C28000A0126864A85CE8597C006E0E78020D53A
:101C380005890DC563914A0313FBF40F230F64074D
:101C4800B250225492540259F249624AD24A424B43
:101C5800B24B45618280050A137AFA0F8504E39234
:101C680074FDE9BF411126C206C622C44AC0973492
:101C7800000083A424B56389041003A4C40AAA86B7
:101C8800054525C43C241307700A6392E7085830B9
:101C98001C34172900001309A97B03268900B38780
:101CA800E7020357C900B387E70213070032938797
:101CB8000719B3D7E70203A744093E97BA846364B8
:101CC800F7006364C700B304C7409727000083A7E1
:101CD800A75484C28297B387A44063F5A40003275E
:101CE8008900BA9789EB1305F00FB2402244924459
:101CF80002494101828058309306204E3307D702AB
:101D0800E3F3E7FE930780FA3CA40145F9BF130704
:101D1800800AE39AE7FC9727000083A7E74F82979A
:101D28002A893545EF208026AD471737000023253F
:101D3800F7C858301C341726000013066671B3879D
:101D4800E7025A261046B387E70213070032938743
:101D58000719B3D7E70203A744093E97BA86636415
:101D6800F7006364C700B306C740E31ED9F617D56A
:101D780005E01305A5E0EFE0DFD19727000083A772
:101D8800A75B0947F8D785B7054585B7397156D296
:101D9800973A0000938A8AC083A70A033707080086
:101DA80026DA06DE22DC4AD84ED652D45AD05ECE87
:101DB80062CC66CA6AC86EC6F98F9734000083A4DD
:101DC80064A0638A071C83A9C40A83C7990003A473
:101DD800C90092073E942820B14705053305F5024E
:101DE8005E203E9533450508EFE04FF1AA8C630F5E
:101DF800051A130DC5002324A50134203146370BDD
:101E08000300B386C602231304000149172A000001
:101E1800130A8A52972B0000938B0B51972D0000C1
:101E2800938D8D52130B8B15054CEA9654C483C6BB
:101E380079009307D00783250A00B386F602C167A5
:101E48009CC5370833008606B4D183A60B009042A0
:101E58001376F6CF90C290421376F6CF136606201B
:101E680090C203A50D0010453366060110C503A6F0
:101E7800090023A865059305500290C672205444B2
:101E8800B2962324DD0014300146CA96A301DD0072
:101E980003C504089736000023A406B0EF00B01C61
:101EA80083260A00CC4613961549D0C60F100000A9
:101EB80083260A003706020090C61306000823A8E6
:101EC800CA0003A60B00104213567648631E860B01
:101ED8001306E018F0D2CCC617360000232A06AC49
:101EE80017360000232E06AA23A08601A925EF2075
:101EF800400183A64A00858AD9CAEA85268597E0E3
:101F080005E0E780C0D10DE903465D0049C27620AF
:101F18004E20B29663DDB606B428AC4803258D0082
:101F2800918E8906B695EFE02FED23020D0003464A
:101F38005D007620B29676A003260A00310D345251
:101F4800FDFE342005091379F90FE362D9EE9C24CC
:101F58006685A381FC001C20A3820C002383DC007F
:101F68002382FC006254F250D2544259B259225A88
:101F7800925A025BF24B624CD24C424DB24D2161F7
:101F8800172305E0670063DA1306E01AA1B7FD56C8
:101F98002302DD0055B79727000083A7E739FC57D0
:101FA80091C78547172700002304F726F25062548B
:101FB800D2544259B259225A925A025BF24B624C9D
:101FC800D24C424DB24D21618280797122D426D201
:101FD8002E84AA84414697C506E09385A5DA0A852A
:101FE80006D6972004E0E780E03E414697C506E024
:101FF800938545D90808972004E0E780A03D3C3048
:1020080010088A85DC875C2026855C875C30DC8646
:10201800974006E0E780E0890347F1011C2001456D
:10202800631EF7000347E1011C3001456318F70000
:102038000345D1013C201D8D13351500B2502254A3
:10204800925445618280011122CC26CA4AC84EC6E4
:1020580006CEAA84172400000324847D13092500D2
:10206800854905C09C303830858B6304F700405C97
:10207800CDBF1946930544004A85EFE06FE9E318A0
:1020880035FFF24022856244D2444249B249056193
:102098008280411122C426C24AC006C61724000005
:1020A8000324047993042500054901E8B2402285F8
:1020B80022449244024941018280A6851305A40264
:1020C8002937E30525FF405CCDB7411122C426C25C
:1020D8004AC006C61724000003248475930425000B
:1020E800054901E8B240228522449244024941014F
:1020F8008280A6851305A401C93DE30525FF405C40
:10210800CDB7011126CA644122CC4AC84EC652C472
:1021180006CE2A841D4993096505054A3C4463E4B3
:10212800F4000545A1A05834DC20631927050347AE
:1021380084026304F7008440D5B7D8308347540538
:10214800E31BF7FE19469305640513856400EFE069
:102158002FDC8547E311F5FED82483479402E31C5E
:10216800F7FCFA243E34E318F7FC0145F2406244D8
:10217800D2444249B249224A05618280E31DF7FAF6
:10218800D83083475405E318F7FA1946CE851385E6
:102198006400EFE0EFD7E31045FBC1BF411122C453
:1021A80006C626C24AC0172400000324A4635DC8DB
:1021B8008347840B1307700A6393E7080347140ED9
:1021C8008347A40B1729000013098928832689004F
:1021D800B387E7020357C900B387E7021307003242
:1021E80093870719B3D7E7020327440A3E97BA84AF
:1021F8006364F7006364D700B304D74097270000EF
:1022080083A7870104C18297B387A44063F5A4001C
:1022180003278900BA9785CB0347140E9306204EEF
:102228003307D70263F1E702930780FA230CF40A15
:102238000145B24022449244024941018280130779
:10224800800A639EE700173506E013050581EFE075
:102258005F849727000083A7270E0947F8D713053F
:10226800F00FC1BF0545F1B7011122CC26CA06CE31
:102278002AC42EC6172400000324045B854419E0F1
:1022880001450DA09C841830858B6304F700004439
:10229800FDB719469305A10013052400EFE04FC7C9
:1022A800E31795FEF2406244D24405618280000043
:1022B800EFE0FF817300000000000000972200009B
:1022C800938202F50383020023800200630F030058
:1022D800F32510342EC0970500009385A5FD739053
:1022E8001534EF0080617300203086DCEF00E06079
:1022F800E6508280000041114AC0172900001309E6
:10230800A9020327090026C206C61C5F22C4972417
:1023180000009384240193D76748C1C79307000638
:102328001CDF1724000013046467184C9307000887
:102338006317F7009C409C4393F707041CCC1C4090
:1023480093F7070499CB9727000083A7E7EC8297B8
:1023580048D81C4093F7F7FB1CC01C4093F70702B2
:1023680099CF1C4017270000032707FDB706080070
:1023780093F7F7FD1CC05C5414C786077CD71C482C
:1023880093F7070499EF85475CC83707020097273A
:10239800000083A767FA98C71307000C18C81854D9
:1023A800F8D383270900985F1357474805C3985FF8
:1023B8001367070198DF9727000083A7E7F723A291
:1023C80007068547172700002322F75E9C40D8435D
:1023D8001357174819C7D843759BD8C3D843799B57
:1023E800D8C3B24022449244024941018280213735
:1023F80073002030972700009387475A3707040057
:1024080088DB698F11CF172700000327E7F2FD56F5
:1024180034D797260000938626FCD84E0507D8CED9
:10242800137785000DC398479726000083A6C6EF4B
:102438001367170098C71307000898CBD856719BE5
:1024480013671700D8D61377150011CFD8439726EE
:10245800000083A666ED13671700D8C3D856719B92
:1024680013671700D8D6137765000DC31377450097
:1024780059C798431367170098C39726000083A687
:10248800A6EAD856719B13671700D8D64167698F9B
:102498000DC39726000083C6A634C18A17270000FB
:1024A8001307C72CB5C28346470793E60602230ADB
:1024B800D70637070200698F11CF984B13770708A3
:1024C80019C3054798CB9727000083A7E7E6370786
:1024D800020098C7B70708007D8D0DC117270000B7
:1024E80003471730058B97270000938727281DCBB4
:1024F80003C7570713672700A38AE7068280D847D0
:1025080013671700D8C795BF834647070946BD8A92
:102518006388C600834647070D46BD8AE39BC6F815
:10252800914671B703C75707118B69DB03C7570774
:1025380013678700D1B79726000083A6E6DF172721
:1025480000001307A7451C43858B91E75C43858BE7
:1025580099E3FC52EDFB9727000023AB07448280E8
:1025680097260000938646DC2A8788421C5D93D70D
:102578005748C1EB81C51C59BD839CA115C69C4217
:10258800945BC60693D7660163D6060093E707C037
:10259800B3C707088316060093975760A9CABE9663
:1025A8008947B3C6F60216A29727000083A7C7D8A3
:1025B800BC4B083393D757488DCF29C597260000C1
:1025C80083A6463F93F606049307950009459DCADE
:1025D800BA979C230547194593F6F7066394E602D4
:1025E80001459397476063DF0700394582801EA243
:1025F80065BF2A9748331375F5077D153335A00055
:102608008280054582809727000083A767D299CBEF
:10261800944BD04B9842518F98C294439C47984210
:10262800D98F9CC217260000130606D10548184208
:102638009726000083A646CF972700009387073682
:102648006314050503A806001368080823A00601FB
:1026580083C62702B3C5D52054479385A50C139884
:102668001649232607010F100000184237060200FA
:10267800860510C71306000890CB6CD354C797275C
:1026880000002385A7CA828088421375F5F788C29F
:1026980083C62702B3E5D52054479385E50E1395E5
:1026A800164948C70F100000184237060200860571
:1026B80010C71306000890CB6CD354C70945C1B79F
:1026C800411122C4AA8706C626C22E8517240000F7
:1026D800130484C6B285CDEB1C40F8537DFF370741
:1026E800020098C79727000023AE072A9724000006
:1026F800938404D1DC5085C7B7E700E03707200092
:1027080023A0E728B7F700E0938707D0984B6D9B85
:1027180098CB984B1367870398CB73005010E53517
:102728009727000083A747C098431317772998C3B2
:10273800D857719BD8D79727000023AB0726972730
:10274800000023AF07241C40094798C3DC5099CBED
:1027580037F700E0832707D193E787002328F7D0CE
:1027680073005010144017270000130727231C4735
:10277800858B91E75C47858B99E3FC52EDFBB24072
:1027880022449244410182800D476390E7069727CF
:10279800000023A907209727000023A707209724D4
:1027A80000009384E4C5DC5085C7B7E700E037072D
:1027B800200023A0E728B7F700E0938707D0984BBD
:1027C8006D9B98CB984B1367870398CB7300501079
:1027D8001D3D9727000083A727B59843131777292E
:1027E80098C3D857719BD8D795B70547E39CE7F6A8
:1027F800972600009386C6C0DC5285C7B7E700E07D
:102808003707200023A0E728B7F700E0938707D011
:10281800984B6D9B98CB984B1367870398CB7300A5
:1028280050101C40D04713171649D8C70F10000086
:102838001C403707020098C71307000897250000B7
:1028480023A6E51617270000032707AE18431357DA
:10285800774819C71307E018F8D3D0C7DC52C5BDAD
:102868001307E01AD5BF9727000083A767AC89CF65
:10287800D44303A8870098423367070198C2D44716
:10288800DC4B9842D98F9CC205479727000083A745
:10289800A7A995056310E50498431367070898C32B
:1028A800984F137707C01367A71398CF13078007AC
:1028B800B8BB939735009387C70317270000130702
:1028C800E70D1CD7972700002382A7A619C2060682
:1028D80010D78280984309451377F7F798C3984F24
:1028E800137707C01367271398CF1307F007B8BBF0
:1028F800939745009387C703C9B79727000083A715
:10290800A7A38847D847798D01C988C797270000AA
:1029180083A747A291C3828782808967172700000F
:10292800032787A1938707F47CD39726000083A603
:10293800A6A183A7060993D7A74991C783A7060924
:1029480093D7974999E37C53EDF78280411106C6E6
:1029580022C426C24AC063030510AD472A8463EA2D
:10296800A70C1304F5FF1374F40F1385F5FF014644
:102978009305F00F1375F50FFD3597240000938428
:10298800A49C9840172900001309099A13640404A9
:102998005C571374F407170500001305250DF59B04
:1029A8005CD7032709001C4393F707F8C18F1CC3A2
:1029B800B7477671938797121CC7B7575500938707
:1029C800575517240000130424975CC31840972711
:1029D800000023A507FC5C43F99B5CC3A5471727A8
:1029E8000000232BF7FCEFE0CF8A14409727000064
:1029F80023A007FC9727000023A407FA0327090050
:102A080085479CC21C4337063300014593F7F7CF2F
:102A18001CC31C4393F7F7CF93E707201CC39840C8
:102A28001C47D18F1CC7B707030093878715BCCAFB
:102A380005A0B1476307F5029307600263E5A700A5
:102A48001304E5FF0DB7930770024945E30FF4F04F
:102A5800B240224492440249410182801304500248
:102A680029B71304600211B717270000032747F39B
:102A7800058B97270000938767CF01CF17270000A2
:102A88000327878A185F1357574801E79A270507CE
:102A98009AA703C68703EC33C8234DBD411122C44E
:102AA80006C626C24AC02E849DCD13F9150081475B
:102AB800414763040904131745003E97B14633079D
:102AC800D7029714000083A42476B317F02833C9DB
:102AD8000708BA949C40C840829723A0040023A208
:102AE800040033448900B2402285224492440249BA
:102AF80041018280B356F448DDFE8507E39CE7FE7A
:102B0800CDB7011126CA06CE22CC4AC84EC6AE841D
:102B1800B1C593F7150001444147A1CF931745006C
:102B2800A2973147B387E702971900009389C96FC5
:102B380003A909003E998327090081C70325490095
:102B4800829731473307E40283A70900BA979C4765
:102B58008DC733148028B3470408BD8CF240624403
:102B68004249B2492685D24405618280B3D6844859
:102B7800D5F60504E31CE4FECDB723200900232283
:102B88000900C1BFAA87171500000325656911E16F
:102B980082803A216315B7001821E30BF7FE4845F8
:102BA800FDB77971B7E700E022D4804352CC06D64E
:102BB80026D24AD04ECE56CA5AC85EC662C43A8A8F
:102BC80037072000798C23A0E7180F10000005E1D3
:102BD80023A087100945B250225492540259F24951
:102BE800624AD24A424BB24B224C456182809717C7
:102BF800000083A76762B6892A89AE8A328B971B41
:102C08000000938B6B62829703A70B008144B14647
:102C1800C147338CD40233068701104241E2C165B3
:102C2800938505F04145EFD0AFED19ED97270000EA
:102C380083A7078081C7814511458297B7E700E0E0
:102C480023A087102D4541BF171700001307475DC4
:102C58001C43A1E308C323000500B31790283EA135
:102C680083A70B00232605002324650123224501A1
:102C7800E29723A0270123A2570123A447016384D5
:102C8800090023809900B7E700E023A087100145D9
:102C980099B73E87DC47F5FF48C775BF8504E39AB7
:102CA800F4F6B7E700E023A0871021452DB7B7E772
:102CB80000E09843B706200023A0D718758F0F109F
:102CC80000009716000083C636716373D502971605
:102CD800000083A626553325D5201621D58D0EA1B3
:102CE8009716000023A2067023A0E71001458280F2
:102CF80023A0E7100D4582800111B7E700E022CC40
:102D080080433707200006CE26CA4AC8798C23A0FC
:102D1800E7180F100000BD4763E9A70431473307E0
:102D2800E5029717000083A72750BA979C4395CFD1
:102D38003315A0282E89B345050801452EC69935B7
:102D4800AA8409C9B2450145972004E0E78020908C
:102D580023A42401B7E700E023A087100145F2402F
:102D68006244D244424905618280B7E700E023A06B
:102D780087100945EDB79726000083C6669A97170E
:102D8800000083A7E75201476394E600014582806B
:102D98008E23138687026394A5003E8582800507EB
:102DA8001377F70FB287CDB79727000083C75797D8
:102DB800AA868507171500000325455001471221EB
:102DC8006307D60005071905E36BF7FE0145828006
:102DD8002A87171500000325E54E11E182801C455E
:102DE800B227636BC70003584500B306C800635594
:102DF800D7008146639406010841C5B703D3A700ED
:102E0800938807016316E30091C192A13E858280F1
:102E18008506C687B3C60608F1BF9726000083C695
:102E280026909717000083A7A74C01476394E600F4
:102E380001458280AE231386C7036394A5003E85AF
:102E4800828005071377F70FB287CDB7411122C4E7
:102E580006C6972700002385079817140000032447
:102E6800244A05C06C390145B315B028B3C5050817
:102E7800972004E0E780C0CA930710273305F502BE
:102E880002942244B2408145014541016FD0DFC11F
:102E9800411106C6383D19C734256310D704B2401E
:102EA80041016DB73C2DE5DF3825E30AF7FE3CA567
:102EB800814517E5FFFF1305051CEFD0FFBE9717E7
:102EC800000083C7E75999C79717000083A7C7462B
:102ED8005147F8D3B240410182803C2D89C7E3981D
:102EE800F6FC38A5F1B7C5FEEDBF41114AC0172958
:102EF80000001309A9AA8327890022C426C206C68E
:102F08009724000093848486858BE0509DCB972777
:102F1800000023A907A883C74407C18B85CFEF000A
:102F2800507E83C7440793F70702E5DF83C744074A
:102F3800228593F7F70C238AF406974005E0E7808B
:102F48004006EF00107C22852244B2409244024998
:102F58004101EDBD83C75407858B91CBEF00707A93
:102F68008D47230EF406BC5822858297D9BF83C7A4
:102F780044071547BD8B6395E7048347B4060345AB
:102F880034060146930550025D8DEFF0DF8D014652
:102F980081450545EFF0CFF28327C900858BD5D34E
:102FA80022859727000023A107A0974005E0E78026
:102FB80000E741F9B240224492440249410182802B
:102FC80083C744071947BD8BE39DE7F68347B406DB
:102FD800034534060146930550025D8DEFF0BF8826
:102FE800014681450545EFF0AFED8327C900858B84
:102FF800A9DB22859727000023A8079A974005E0B8
:10300800E78020BB7DB7411122C426C206C67C25B5
:1030180078452A84BD8B1CA91CA31D476445639B66
:10302800E7340547B8A08347F5058D466395D7185B
:103038005E2DCDE37C491147B18B638DE70831479D
:103048006398E700034715068347F5076304F70805
:103058008547BCB019469305640313854400EFD037
:10306800AFD9BC20990793F7F70FBCA00347040614
:103078001377070401CFB83013670704B8B0784452
:10308800BA975838B8B3BC208507BCA0971700007A
:1030980023880774BC2013F7F703050718B80347FC
:1030A800E4051A07D98FBCA083475403858B91E7A1
:1030B8000347440389476317F70078441C2393E7C1
:1030C80007041CA37C44183898B3B24022449244A5
:1030D80041018280A147BCB08357C4069715000000
:1030E8009385C5681716000013060625DCA08357CC
:1030F800C406034714067444A1831207BD8BD98FF5
:10310800DCB2B4208547890693F6F60FB4A01717EA
:1031180000000347E76C631EF706183C9387E60038
:103128008E07231AF4069387C708B387E702794501
:1031380010420948238A0507C1650CC6938707FB17
:10314800B3C7070893877716B3C7A70233C707081B
:10315800B387A70286073CD2BC3093E70701BCB00F
:103168007C44B6978346240693E60604B4B3B42099
:103178007C44B697D8A3B4207C4421837D8BB69732
:10318800834634069606558FD8B3BC208D07BCA05D
:1031980011B71042F947385205833357F7023C52AA
:1031A80068528583FD8BAA977CD28D47238AF506C2
:1031B8003347070855B71946639DC7125E2DC1E30B
:1031C80093056503B8B013854400EFD0EFC2BC2067
:1031D8001385A4009907BCA0BC3093E72700BCB0B6
:1031E80083475403898B95CF0C58BC299DCB19462E
:1031F800D105EFD06FC078441C2393E707F81CA3D0
:10320800BC20990793F7F70FBCA003470406137770
:103218000704E30D07E6B430784493E60604B4B037
:1032280085B58347D40391C778441C2393E707F8EF
:103238001CA319469305E403EFD00FBCD1B7A147EF
:10324800BCB08357C506DCA08357C50603461506E0
:103258006C45A1831206BD8BD18FDCB1B020171548
:1032680000001305A550971500009385E50C090685
:103278001376F60FB0A09717000083C767566398B8
:10328800E704183C9307E6008E07231AF406938791
:10329800C708B387E70279488946230AD5069441C7
:1032A800C1658CC6938707FBB3C707089387771652
:1032B800B3C7070333C70708B38707038607BCD21A
:1032C800BC3093E70701BCB07C44B29761BD8C4128
:1032D800B851F94705833357F702BC5103A845068F
:1032E8008583FD8BC297FCD1230AD506334707088F
:1032F800C1BFA147BCB08357C506DCA08357C5062C
:10330800034615066C45A1831206BD8BD18FDCB12F
:10331800B020171500001305654509061376F60F4A
:10332800B0A09717000083C7A74B9715000083A587
:10333800A500E39FE7F8183C9307E6008E07231AD9
:10334800F4069387C708B387E702F9460948230AB2
:103358000507416588C5938707FBB3C707089387A7
:103368007716B3C7D70233C70708B387D7028607CC
:10337800BCD1B9B70547639EE706B1471CB9834777
:103388005503898BA1CB0C59BC29A9C71946D1056E
:1033980013858400EFD04FA678441C2393E707F8E1
:1033A8001CA368441946930564030905EFD0CFA40C
:1033B80011679717000083A76748F98FE38607CE40
:1033C8007C24B98BE39207CE78441C2393E7070249
:1033D8001CA3D9B98347D40389C79C2093E707F86E
:1033E8009CA0684419469305E4032105EFD0CFA0BB
:1033F8004DBF522D0C559307660093F7F7031CB980
:1034080013858400E5B7011126CA97140000938438
:10341800E4589C4422CC06CE17140000130404354B
:10342800858B6850D9C32AC69717000023AC075666
:10343800EF00302D03474407894732456307F700FB
:10344800034744078D47631EF7029716000083A6BB
:10345800A6EEBC520357450785831307C71263F2CC
:10346800E702BC528583B1C3914703474407E31E73
:10347800F7FE6244F240D2440561174305E0670055
:10348800A3DB382D3C3D09CF34256309D702638877
:10349800F60238A56244F240D24405616FD07FA499
:1034A80099CF382509EF3CA5F5B72AC6EF00702556
:1034B80062443245F240D244056149BAEDF7DC4C2A
:1034C800EDF70347440789476307F70003474407B5
:1034D8008D47E31CF7FC914703474407E31EF7FEBB
:1034E80049BF63000532011122CC06CE26CA4AC85C
:1034F8004EC652C456C2582585472A846318F72CED
:103508009717000093878749D44F1547638AE600C9
:10351800D44F0D476386E600D84FAD476312F702D4
:103528006C386244F240D2444249B249224A924A33
:1035380001450561B315B028B3C505086FF02FF72D
:10354800163113070064971400009384242233472C
:10355800D7029C20E8D0850793F7F70F9CA063CA91
:10356800E700972004E0E78020A297170000238F48
:10357800071E78249D47631FF70483479406B1C349
:103588008356040763ECF6020C24930730041CAC42
:103598001305300493F6F60F0146977006E0E780AE
:1035A80080C722856244F240D2444249B249224A45
:1035B800924A0561174305E06700037885062318DA
:1035C800D406930530020545972004E0E780A094CF
:1035D8002301A4060549238A2407183C8D47631C48
:1035E800F70E971004E0E78000FD0D89630F0514BE
:1035F80063162517930760023CA4930750023CAC5E
:103608009307700278243CBC85476302F7088965F4
:103618009385F57013051027171A0000130A4AE35B
:1036280083497401972004E0E78060910E30835A43
:10363800CA002A8913060064B38555038146138599
:103648000532B335B50097A006E0E7800038AA84B4
:10365800B335590337460F00130606248146330550
:10366800590397A006E0E780403683270A00AA940A
:103678008297B307950003278A00BE8563E4A700F5
:1036880063E4E700B385E7404E85EFF0EFE6834754
:103698005403898BE9CB8347C403F1C70C58E1C5B0
:1036A800BC25F1C38947230AF4021946B10513055D
:1036B8006403EFC07FF40347C407894763E9E70A57
:1036C80022856244F240D2444249B249224A924A8F
:1036D80005616FD01F8189467C346315D70213F7C3
:1036E800170019CB898B1307500291EB93077002CF
:1036F80038A43CAC814739B713076002C5BF9307AC
:103708006002FDB799CF93F617001307500291E6B0
:10371800898B13B717001307670238A4230D040019
:10372800D1BF3C2C130740026368F700930750028F
:103738003CAC3C2C3CA47DBF850793F7F70F3CAC11
:1037480013077002E364F7FEEDB7130770029307DF
:1037580050023CAC38A4930760026DB513075002C1
:1037680093077002FDB78547230AF402A9B7032718
:10377800C40A9716000083A626AA3C27ADC31C37A7
:103788005833971400009384A4CC9044B387E7027D
:10379800DA24B387E7021307003293870719B3D7F0
:1037A800E702032744093E973A896364F700636494
:1037B800C7003309C7408296B307A9406374A900BC
:1037C8009844BA9703576407E3FCE7EEF240624473
:1037D800D2444249B249224A924A056182808324EE
:1037E8008409829663E9A400835764073385A4405B
:1037F800E378F5ECE1BF9717000083A7E7C5BE940F
:10380800E5B7828001114EC697190000938909F621
:1038180022CC03A4C9094AC817190000130949C3CF
:103828000357C90026CA835464088327040906CEAF
:10383800B384E40237470F009306F72313070724DE
:1038480052C456C25AC0B694B3D4E40263E0970493
:10385800171A0000130A4A9CB384974083270A006A
:10386800829763E9A4023385A4406349050283571C
:103878000404A30F040085072310F40483470414E9
:10388800639E07102285EFD0BFBE21AA03278900B7
:10389800BA977DBF83278900BE94F1B783270A00B2
:1038A8008297032784086366E50A198D7E3C0357CF
:1038B800C9008E07B387E7021307003293870719F9
:1038C800B3D7E70263ECA708B74A0F00138BFA23B4
:1038D800938A0A248357040485072310F404834732
:1038E800041481E72285EFD0BFB82285975005E000
:1038F800E780002E63170524032604090327C4085C
:10390800832689003297BA876364C7006364D70047
:10391800B307D740783C0356C9002328F4080507A5
:1039280078BC035764083307C7025A9733575703BD
:10393800B384E74063F5E700998EB384F6008327E4
:103948000A00829763E6A4043385A440E34405F89B
:1039580039BF83278900998F3E9589BFA145228564
:10396800975005E0E780E01EA305A4029717000022
:1039780083A707AC6387071C6244F240D2444249DC
:10398800B249224A924A024B894515450561828708
:1039980083278900A6973385A7404DBF2285EFD09E
:1039A8007FB72285975005E0E7808022631B0518C2
:1039B8000355C90083576408B7460F001386F623DA
:1039C800B387A7029386062403270409230B04025E
:1039D800832A8900B297B3D7D702636EF716B30765
:1039E800F7408326C4082324F408014BB387E60074
:1039F800BE8463E4D70063E45701B38457411E30A3
:103A080023289408A1CB835604045A3037460F0064
:103A180056B03387E640B387E7023A3013060624E8
:103A280081468145BA97B3C707083385A7023EB0D8
:103A380097A006E0E78060F911CD2695B33495008C
:103A4800A695AA876314BB0063645501B307554163
:103A58002328F40883270A008297AA8483270A0068
:103A68008297E30D95FE83270A00832484088297B2
:103A780063E8A40E3385A44063010510035AC90006
:103A880083576408B7440F001387F423B3874703A9
:103A980093840424BA97B3D79702171700000347F3
:103AA800B797BA9763EBA70CB3359502835A2402EC
:103AB800528681463305950297A006E0E780E0F03C
:103AC8003389AA0033854A0337460F0013060624B4
:103AD8008146814597A006E0E78020EF15C1B337FE
:103AE800950252868146B385B4023385A402BE95F9
:103AF80097A006E0E78060EDB38AAA40231154033B
:103B08003545692123AE890838348547631EF70493
:103B1800930700FD7CA48145171500000325058047
:103B2800EFC09FF89547171700002327F7E83707D6
:103B380010009717000083A7278098C7060923A8B5
:103B48002707F2406244D2444249B249224A924A83
:103B5800024B05618280B3065701B387F64051B521
:103B680083278900BE9439B7930710FC7CA481454C
:103B7800170500000325057A65B79717000023A5E8
:103B880007C8834709019DC31705000003258577EA
:103B9800EFD04F95624483274900F240D24442490E
:103BA800B249224A924A024B0561828783459402B0
:103BB8006244F240D2444249B249224A924A024BF4
:103BC80001450561B315B028B3C505086FF02F8E00
:103BD800011122CC26CA4EC606CE4AC852C456C2C5
:103BE8005AC038358547832405092A84AE89631469
:103BF800F70C83570508835AC503171A0000130AE0
:103C08002A85035BCA0063FE57191429639BE618CB
:103C180003278511631707180327450A6313071835
:103C280074351D47639FE6162A3DB38AFA40930709
:103C3800204E330555030329440937460F00130660
:103C4800062481463305F5029707000083C7C77C21
:103C580033592503B335AB023E9933490908231379
:103C680024093305AB0297A006E0E78000D6B30726
:103C7800950033B5A7002E9503278A00BE8419E165
:103C880063E4E700B384E740B307690337470F00ED
:103C98009306F7231307072423A09900B697B3D7F1
:103CA800E702D69763E4F4009D8C31A003278A00CD
:103CB800B307F740BE94170900001309E955832795
:103CC800090023A09900829763E2A4103385A440D9
:103CD800635D050A83270900170B0000130B4B7758
:103CE800829703A709006369E50E198D7E3C035787
:103CF800CB008E07B387E7021307003293870719B3
:103D0800B3D7E70263EFA70C374A0F00930AFA23E9
:103D1800130A0A248357040485072310F4048347ED
:103D2800041481E72285EFD0AFF42285975005E08F
:103D3800E78000EA61E5832604098327C40803278E
:103D48008B00B697BE8463E4D70063E4E700B384CE
:103D5800E7407C3C8356CB002328940885077CBC2D
:103D680083576408B387D702D697B3D7470363E668
:103D7800F40A9D8C8327090023A09900829763E1A8
:103D8800A40A3385A440E34705F89707000083C7D2
:103D9800B76863E6A7069717000023A787A601451B
:103DA800B9A88357640837470F009306F723B387EA
:103DB800670313070724B697B3D7E702E3F6F4EED1
:103DC80003278A002697B304F740F5B59707000044
:103DD80083A78768BE94DDBD83278B00998F3E95A6
:103DE80031B7A1452285975005E0E78080D6A30525
:103DF800A4029707000083A7A76381EF7D55F240CF
:103E08006244D2444249B249224A924A024B05616D
:103E18008280894515458297D5B71D8FBA9499BF79
:103E280083278B00BE94B1BF9707000083A7C74FB5
:103E380098433706CEFF7D161377F7CF1367071021
:103E480098C31707000003272750144737080300B3
:103E58001375F51FF18E14C79706000083A6C64D8B
:103E680023A8060523A40700904B93F5F50713082C
:103E780088151366F60390CB90431366060890C323
:103E8800F04F137606E0498EF0CF23AC070423A049
:103E980007065057759A50D79043137606F84D8EFB
:103EA80090C31306401FF0D217160000232206B055
:103EB80017160000232606AE054690C29043B705A4
:103EC80033001376F6CF90C390431376F6CF13667C
:103ED800062090C310474D8E10C723A80605D85357
:103EE8001317F728D8D32547F05201C6B04FE37D02
:103EF800C7FED8531317F748D8D3A853133545002E
:103F0800828017070000130727431443BC4ABD9B50
:103F1800BCCA01000100010001001C43B44B93F628
:103F2800F68FB4CB944393E6860094C30100010056
:103F3800010001009706000083A6063F9C4293F704
:103F4800F7CF93E707109CC2170600000326C63F69
:103F58001C46B706CEFFFD16F58F1CC61C43370757
:103F68000300B8CB9707000083A7873C99CBD443BD
:103F780090479842518F98C2944BDC4B9842D98F06
:103F88009CC29717000023A907A282809707000008
:103F980083A7873A9C438D8BF9C74111B7E700E0A7
:103FA8004AC003A9070026C23707200006C622C454
:103FB800AA843379E90023A0E7180F10000017142A
:103FC80000001304A49D584C8D47631AF700970707
:103FD800000083A727760146814545458297194702
:103FE8006393E4048347140289CB834704026396EE
:103FF800970097170000A383079C584CA1476315A7
:10400800F700930780101EB097070000238207204F
:10401800CD3DB2402244B7E700E023A027119244E7
:104028000249410182809D47639BF4008347140243
:10403800E9D7034704028D47E311F7FC5DBF544CF1
:104048006389E600584C6306F700584CA147E31D06
:10405800F7FA83471402CDFB5C4C2300F402854732
:10406800A300F40255B78280411122C42A84354541
:1040780006C6293F59CCAD4763EB87067D141374F8
:10408800F40F9707000083A7272C984BB70600C1A9
:10409800FD161374F403758F6204418F98CB1707CC
:1040A8000000032767285857944B71766583137768
:1040B800F7031306F60FF18E2207558F98CBF84FAA
:1040C800B706F9FFFD1613674700F8CF984B01456F
:1040D800758F1317172998CB370702001307874FD7
:1040E80098C7B147171700002328F78C39A8B1479C
:1040F8006304F4029307600263E48700791441B70C
:10410800930770024945E30EF4F6B2402244410198
:10411800828013045002B5B7130460029DB70000F3
:104128002A8309CA83830500230073007D160503CB
:1041380085056DFA82809707FC1F83A7A7E11707FB
:10414800FC1F0327A7E001456313F7008280F623CD
:1041580099E2D62336959C43C5BF1707FC1F130762
:1041680027FF1C435A23411193860711E117BA9779
:1041780085651706FC1F232FD6DC1706FC1F23278F
:10418800F6DC06C69D051356370063F4E5001306F2
:1041980000203387C6009705FC1F23ABE5DA6116BC
:1041A80098C2D2A2239306001CC3998FE1175EA37D
:1041B800231307004937B2409707FC1F2399A7F636
:1041C800410182809707FC1F83A7C7D81707FC1FE8
:1041D8000327C7D701456313F7008280F62381E6DA
:1041E800D6233375D50A9C43FDB7184183A785FFAD
:1041F8006319B7001CC1FD5723AC05FE238FF5FEDC
:104208008280232CF6FEC5BF411122C437E400E0AA
:1042180026C204403707200006C6F98C2320E4187C
:104228000F10000009E9232094101545B2402244DC
:104238009244410182800347E5FF9307F00F63062C
:10424800F700232094101145D5B797C0FB1FE780CE
:1042580080ED014523209410D1BF41114AC037E9B0
:1042680000E022C403240900B707200006C626C2BE
:104278007D8C2320F9180F10000089E52320891070
:10428800154515A0AA849707FC1F83C7F7E92E8553
:1042980063F5F400894763EE9700BD37B7E700E0A0
:1042A80023A087100D45B24022449244024941019F
:1042B800828083A785FF99E703C7E5FF9307F00F7F
:1042C8006308F7009137B7E700E023A087104DBFD8
:1042D800238F95FE1705FC1F130505C897C0FB1F04
:1042E800E78060F5A165268597E0FB1FE780607190
:1042F80001452320891045BF9707FC1F23AE07C43B
:1043080082804111B7E700E026C2844337072000C6
:1043180006C622C4F98C23A0E7180F1000009707DF
:10432800FC1F83A7E7E41704FC1F130424BA91C7F2
:1043380082971C40AA971CC031A09707FC1F83A72F
:10434800A7C2FDF70840B74703009387D73F330557
:10435800F502B7A72600938737ECB2403E9508C010
:104368002244B7E700E023A09710924441018280DD
:10437800411122C406C69707FC1F83A7A7BE1704CE
:10438800FC1F130464DA89C782975C48AA975CC843
:104398004848B240224441018280B7E700E0984390
:1043A800B706200023A0D718758F0F1000009706B6
:1043B800FC1F83C676D76370D5029706FC1F83A6B9
:1043C80066BB3325D5201621B3F5B6400EA123A030
:1043D800E7100145828023A0E7100D45828079719E
:1043E800B7E700E026D284433707200006D622D458
:1043F8004AD04ECE52CCF98C23A0E7180F100000FB
:10440800930705FF93F7F70F7D476363F70A314773
:104418003307E5029707FC1F83A707B6BA979C43A3
:10442800C1CB135445003D893315A028AE89B34547
:10443800050822852EC697E0FB1FE780E0492A89F8
:1044480039C9B2452285170AFC1F130A6AD5B13744
:104458009707FC1F83A747B182978357CA002A840E
:1044680081463387370313060064B3B73703130550
:104478000732B335E500BE95EF90E229B307850012
:1044880083268A003E8763E4A70063E4D700338766
:10449800D7402324E900B7E700E023A0971001459F
:1044A800B250225492540259F249624A45618280BC
:1044B800B7E700E023A097100945DDB7797122D44A
:1044C80037E400E04AD003290400B707200006D6E5
:1044D80026D24ECE52CC56CA5AC85EC63379F90097
:1044E8002320F4180F1000009707FC1F83C7D7C3B9
:1044F8006378F500970BFC1F83AB0BA763970B0042
:10450800B7E700E023A0271199A0970AFC1F938A18
:104518002AC903AB8A00B74736FE938707C83E9B74
:1045280083D7CA002E8AAA84B385C702B289814676
:10453800B3B7C70213850532B335B5001306006457
:10454800BE95EF90421D6370AB02232024110145F4
:10455800B250225492540259F249624AD24A424B0A
:10456800B24B45618280829B83D7CA002A84130696
:104578000064B38537038146B3B737031385053223
:10458800B335B500BE95EF900219B307850003A7B0
:104598008A003E8463E4A70063E4E7003384E740CD
:1045A800D285268597E0FB1FE780003301C900C547
:1045B800B7E700E023A02711054559BF93E504F0AC
:1045C8004145B3C5050897C0FB1FE780A0A811E9BE
:1045D8009707FC1F83A7C7BA85D7A6851145829779
:1045E80005B71707FC1F1307A7981C4389EF08C3D3
:1045F80085472326050000C52311450104A11CB1E8
:104608002322050075B73E87DC47F5FF48C7CDB7BD
:104618007971B7E700E026D284433707200006D631
:1046280022D44AD04ECE52CC56CA5AC85EC662C4AC
:1046380066C2F98C23A0E7180F10000035C12A893B
:104648002E8AB28AB6894144B14C170BFC1F130B52
:10465800AB92130C0003B30B940383270B00DE9774
:104668009C43B9EF135544409375F400568613756F
:10467800F50FB315B028B3C50508893531C18327AF
:104688000B00DE9723A0270123A2470163840900BA
:1046980023808900B7E700E023A09710014521A0F7
:1046A80023A097100945B250225492540259F24956
:1046B800624AD24A424BB24B224C924C45618280AC
:1046C8000504E31A84F9B7E700E023A09710214511
:1046D800D9BF011122CC37E400E026CA04404AC8F9
:1046E8004EC652C406CEB70720002A892E8AB28940
:1046F800FD8C2320F4180F100000C933D2854A8599
:1047080097E0FB1FE780401D01ED23209410214511
:10471800F2406244D2444249B249224A0561828049
:104728009707FC1F83D787A8B38537032A89130601
:1047380000648146B3B7370313850532B335B50036
:10474800BE95EF80527D2322A900232094100145B5
:10475800C1B7011126CAB7E400E04AC803A904009A
:1047680022CC4EC6B707200006CE52C4AA892E8492
:104778003379F90023A0F4180F10000097E0FB1F0D
:10478800E7808015170AFC1F130A0A9A1DE1A28503
:104798004E85213183470A006382370523A02411FF
:1047A8001945F2406244D2444249B249224A05615D
:1047B800828023110500A2854E85C53683470A00ED
:1047C8006386370123A024110145E1BF17F7FB1FBA
:1047D800130727791E23C18F1EA3EDB797F7FB1F79
:1047E800938727789A23598C82A34DBF01114AC811
:1047F80037E900E022CC03240900B707200006CEE1
:1048080026CA4EC67D8C2320F9180F100000930786
:10481800F00263E7A704B144B304950297F9FB1FBC
:104828009389897583A70900A6979C4395CB9375AF
:10483800F5001181B315B028B3C50508193F83A742
:1048480009000145A69723A0070023A207002320FB
:104858008910F2406244D2444249B24905618280DB
:10486800B7E700E023A087100945E5B74111B7E78E
:1048780000E026C2844306C622C437072000F98C0C
:1048880023A0E7180F10000097E0FB1FE780C00483
:1048980019E90145B2402244B7E700E023A0971088
:1048A800924441018280004597F7FB1F83A7C76B9D
:1048B80082979707FC1F9387A78E6367A402984780
:1048C800B74636FE938606C83305A4403697E3728A
:1048D800E5FC13070064B335E502D22781463305AA
:1048E800E502EF8052637DB798473A94C9BF4111FA
:1048F80006C697F7FB1F23A7A7660295B24097073E
:10490800FC1F23AFA7820145410182804111514616
:1049180081451705FC1F1305658706C622C426C2F4
:1049280097F7FB1F23A6076497F7FB1F23AC0762C3
:1049380097F7FB1F23AA076297F7FB1F23820762DB
:1049480097F7FB1F23AC076097C0FB1FE78080A683
:1049580013068002814517F5FB1F1305E57C97C0F8
:10496800FB1FE78020A5EFF04FFF97F7FB1F93870A
:10497800277EE82BFC3B17F4FB1F1304E47A8545DC
:104988003E958D473305F5029307000497F4FB1F06
:104998009384845E39051375F50F3375F50A9947C5
:1049A80028A03305F502130505243345050897B0FB
:1049B800FB1FE780206A88C035C9302099478145A8
:1049C8003306F6021306062497C0FB1FE780809E75
:1049D8009C40382097F4FB1F9384445993870724FD
:1049E8009CC0B347F72017F7FB1F2325F758293238
:1049F80025211C30944017E6FB1F1306C6E533C774
:104A0800D72010C3138717001377F70F17E6FB1F7C
:104A1800130606DE3347D72010C3138737008907EC
:104A280018B093F7F70FB3C7D72090C3B24022440A
:104A380092444101828097F6FB1F9386E66E2A878F
:104A4800BC228832637DF5001306150097F7FB1F1B
:104A580083A7C75190B2B347F52098C38280130546
:104A6800F00F82801C41E5CB370700F07D8FB70639
:104A7800002089476312D70E5A21411122C406C665
:104A88002A8469C719469305F00F690597C0FB1F6B
:104A9800E78060A505478D47630AE50A1C4491C76E
:104AA8005858994745C7185C55C31306C003814534
:104AB80017F5FB1F1305C56997C0FB1FE780808F9B
:104AC8001306C003A28517F5FB1F1305656897C079
:104AD800FB1FE780A08797F7FB1F93876767DA2795
:104AE80001E713070010DAA7F82719E30547F8A725
:104AF8009A2B19E36D479AABF83719E31547F8B7BE
:104B0800B82B19E30547B8ABB83B19E3F837B8BB7E
:104B1800D83B11C7937637000983F4ABF8BBD82B81
:104B280019E35547D8AB182C01E71307C00398AF12
:104B38009C5791C7829797F7FB1F239BA75EFD574A
:104B480017F7FB1F2300F75ED1338147B240224499
:104B58003E854101828089473E85828079714ECEAB
:104B680097F9FB1F9389C96383A7090006D622D446
:104B780026D24AD052CC829713090064B335250354
:104B880003D6C900814617FAFB1F130AEA5932C631
:104B980033052503EF80323883248A012A840145AE
:104BA8006386840232463305944063EF840003A58C
:104BB80089008146B335A9023305A902EF80B235D1
:104BC800B307954033858700232C8A00B2502254BE
:104BD80092540259F249624A45618280011122CCFD
:104BE8000A852E844146979502009385A5EC06CE4A
:104BF800EFF00FD318083324E420035704FFF240E2
:104C0800624497F7FB1F83D7875A37450F00BA9737
:104C1800130505243355F5020561828097F7FB1FBC
:104C280083D7E75851471D45637CF70279471945F3
:104C38006378F7021307200315456373F702130718
:104C4800B0041145637EF700130740060D456379EC
:104C5800F7001307600909456374F70013B5B70F28
:104C68008280411122C426C22E84AA8406C6058CDD
:104C7800EFF02FE9B327A402B2402244338597000E
:104C88001375F50F924441018280411122C426C256
:104C98002E84AA8406C6058CEFF0AFE6B327A402DB
:104CA800B2402244338597003345050892444101B8
:104CB8008280411122C426C22E84AA8406C6058C8D
:104CC800EFF02FE43335A402B240224426959244F3
:104CD8004101828041114AC017F9FB1F1309494756
:104CE8008327890206C622C426C28DCF829797F4ED
:104CF800FB1F938464439E242A848DC733F7A70A35
:104D080033470708B3D7A70AB3C70708B307F7405D
:104D180051476359F7008327C90291C38297EF105F
:104D2800823E82A4B24022449244024941018280D8
:104D3800011122CC97F7FB1F23A2072417F4FB1FAE
:104D4800130404415C5406CEAA8581C72AC68297FB
:104D5800B245D1C59C410545BDCF9C45ADCFDE25AB
:104D6800BDCBFE25ADCB9C2981CB7C287838BA9762
:104D78006343F506DC41A5C31306400217F5FB1F84
:104D88001305054297B0FB1FE780405C97F7FB1FB0
:104D980093870741984397F6FB1F23A7E61C183C07
:104DA80019EFCA279307805737460F003305F502D6
:104DB8001306062481468145EF80F21508BC183C8D
:104DC8009D4763E4E700A1471CBC170500001305D5
:104DD80025D9313E0145F24062440561828097F74A
:104DE800FB1F23A1073697F7FB1F9387673B17C75E
:104DF800FB1F130747C098C337873200FD561307B8
:104E080027A194C7D8C797F7FB1F2383073AB7C7CB
:104E1800004023A4D7269DBF011122CC17F4FB1F05
:104E280013040433084406CE26CA4AC801E90545D6
:104E3800F2406244D2444249056182805C58E5DB15
:104E4800185C75D77000854582971844B247E3000F
:104E5800F7FE4A249305E00417F9FB1F1309C92C30
:104E680097B0FB1FE780001F2320A90269D15224B5
:104E78009305F00F814497B0FB1FE780A0537C2473
:104E88000326090263C1F402328597B0FB1FE7804D
:104E98008029014597F7FB1F23A8072A97F7FB1FCF
:104EA80023A6072A71B74E241844B387950289812F
:104EB80085043385E7001C5C08C28297C9B70111D5
:104EC80022CC17F4FB1F1304A4281C4426CA4EC680
:104ED80056C206CE4AC852C45AC0AA84AE89B28AFB
:104EE8006388071A585839CB1307F01F6366A71051
:104EF80017FAFB1F130A4A2303290A02631209043B
:104F08004A249565938515E097B0FB1FE7808014C8
:104F18002320AA022A861DC14E245C580844898190
:104F280082971C4403290A022322FA028947639EB6
:104F3800F402C1479305090C6381F9042945BDA012
:104F480003274A02E384E7FE4A249565938525E012
:104F580097B0FB1FE78000102A896DD14E242A865E
:104F68005C58084489818297D1B78D47639AF404C5
:104F7800C1479305490DE393F9FCB8219307A005B0
:104F88006312F7069E21639F97044E869105568506
:104F980097B0FB1FE780803B83270A0263872701BE
:104FA8004A8597B0FB1FE78000180145F24062442C
:104FB800D2444249B249224A924A024B0561828050
:104FC80091476397F4009305890EE39999F675B7AD
:104FD80093070010E394F4F6A147E3E137F793054C
:104FE800090F61BF83270A02E38A27F54A8597B02C
:104FF800FB1FE780401399B71D67637FE50613071A
:1050080005E099463347D702562417FBFB1F130BBD
:10501800AB113307D702330AF70083274B02639695
:10502800470103290B02631109024A249305E0048E
:1050380097B0FB1FE78000022A8909D14E245C58EB
:105048002A8689815285829791451307A00593F591
:10505800C50FB307B900B4236399E6029623639496
:10506800960291054E86CA95568597B0FB1FE78034
:10507800E02D83270B021DB7A166F916E3E0A6EC25
:105088003307E54051B7AC33D9B783270B02A9BF23
:1050980097F5FB1F83A5450BE38205EA9147930625
:1050A800A00593F7C70F3387F5003023E318D6E838
:1050B8001223631B960091074E86BE95568597B0BE
:1050C800FB1FE780A028D5B53C33E1BF97F7FB1F4E
:1050D80093870708984721C7985F31C385466310AF
:1050E800D504411122C417F4FB1F1304E403105024
:1050F80006C615C2CE27485089810297085097B036
:10510800FB1FE780400297F7FB1F23AF070297F7C3
:10511800FB1F23AD0702B2402244410182808280F6
:1051280001114AC817F9FB1F130989024EC68329C2
:10513800890022CC26CA52C406CE56C2AA842E841E
:10514800328A638D091A8327890399EB2945F2402E
:105158006244D2444249B249224A924A0561828055
:1051680083274903E5D79307F01F63E0A70C97F956
:10517800FB1F938969FB83A7090295CF0325890043
:1051880083A749026395A7048947639FF404C1472D
:10519800E31EF4FA03A509021305050C9307A005FD
:1051A8003CA106A12286D285110597B0FB1FE78096
:1051B800E019014569BF0355C9009305E00497B09C
:1051C800FB1FE78020E923A0A9024DF941B78355C9
:1051D800C9008327490303A6090289818297832787
:1051E800890023A2F9024DB78D47639AF400C1479D
:1051F800E31EF4F403A509021305450D45B79147CD
:105208006399F400E31494F403A509021305850EC9
:1052180071B793070010E39BF4F2A147E3E887F224
:1052280003A509021305050F95BF9D676373F5066E
:10523800930705E01947B3C7E7020357C90097FA70
:10524800FB1F938A6AEEB387E702BE9983A70A0217
:10525800A1CB83A74A026391370703A50A029147A6
:105268009305A0051308F00F13F7C70FB306E50061
:10527800B0226313B60683D80600B032639C980444
:10528800B307F64063C6870411072286D2853A958C
:1052980029BF21677917E36BA7EAB307F54071BF08
:1052A8000355C9009305E00497B0FB1FE78080DA37
:1052B80023A0AA0259FD59BD8355C9008327490374
:1052C80003A60A0289814E85829723A23A0371B701
:1052D80023900601B28749BF338687001106130859
:1052E800F00B6374C8002D459DB5ACA213063400BD
:1052F800719A1106B29786A2BCB279B797F9FB1FCB
:10530800938989E283A709029DCB03A509029147E6
:105318001308A0059305F00F13F7C70FB306E500B0
:10532800B0226310060583D80600B0326397980050
:10533800B307F640E3DA87F48EA2B287F1BF83475A
:10534800E9000355C9009305E0043305F502334528
:10535800050897B0FB1FE780E0CF23A0A90255F509
:10536800F5B30356C9008345E900B385C502338602
:1053780087001106E3E9C5F62381060185BF0145CB
:1053880082809C211CA1BE211CB1BE21A1833CA10D
:10539800DC213CB11145828097F7FB1F23A407BE8F
:1053A80097F7FB1F23AE07BC82800DCD411122C4A5
:1053B80026C206C6AA842E84014585C12285414697
:1053C800978502009385057297B0FB1FE78000F868
:1053D8009C2005455CA49C305CB4B24022449244B5
:1053E8004101828001458280011122CC26CA06CE65
:1053F8008947AA843284639EF5006383B6024147D5
:1054080081476395E6048A854D3741468A8522851A
:105418000DA841476392E504638FF600639EB602C8
:105428002E86A2856244F2402685D244056117B3D0
:10543800FB1F670023038A853285853F41468A859D
:10544800268597B0FB1FE780E001AA87F2406244F7
:10545800D2443E85056182808147CDBF97F7FB1F07
:1054680023A0A7B2828097F7FB1F23ADA7B0828045
:10547800011122CC622106CE26CA4AC84EC63DC8B2
:10548800832985002A88AE8403C909008147131738
:10549800496063550702B147054563F6870403551C
:1054A80028005114334404084E8633878900A286A5
:1054B8008545EFB0B003B337A00085071355694899
:1054C8007D141379F903334404089CA088B0238120
:1054D8002401C2A0014719C01387190098C40947BD
:1054E8006383E7000145F2406244D2444249B2492D
:1054F800056182800545C5BFC167F917630AF502D2
:10550800D94763F7B702011122CC2EC606CE2A84EA
:10551800EF90A007B2456368B50022856244F24067
:1055280005616FA0807CF240624405450561828078
:1055380005458280C167F9176314F5006F90E00490
:10554800411106C6EFA0006911E15D45B240410175
:1055580082809147639DF5001C211CA23C211831D3
:10556800A207D98F3EA23C3101455CA28280114539
:1055780082804111814522C426C206C6AA849D2381
:105588002A8409E997F7FB1F83A7879F81C7F945F5
:1055980026858297B2402285224492444101828026
:1055A80039714ED652D45AD05ECE06DE22DC26DAC7
:1055B8004AD856D22A8A2E8BB289B68B0DE79D3FE0
:1055C8009145EF90A00A2A844D49854A19EDF25079
:1055D8006254D254B259225A925A025BF24B4A850B
:1055E8004259216182803A84814A230034018544EA
:1055F800630A0B00DE8513051400029B9304150053
:10560800B3C404089399496063D30902C14552851C
:10561800EFA0806A654915E533069400A6852285C2
:10562800EFB0E0312A8911EDB104B3C40408914701
:105638002C0052857C8422C66485EF90B07F2A892D
:1056480059D5E3860AF8228597B0FB1FE780A0ADFD
:10565800BDBF011122CC26CA4AC84EC606CE2A8929
:105668003284B689353FAA840DE197F7FB1F83A7DB
:10567800679181CF05476317E40003C40900050457
:105688001374F40FA2854A858297F2406244424916
:10569800B2492685D24405618280AE860147054617
:1056A80097050000938525CE6DB79E211CA19E21EC
:1056B800A1831CB1094582809E211CA19E21A18342
:1056C8001CB1BE213CA1BE21A1833CB11145828001
:1056D8009E211CA19E21A1831CB1BE213CA1BE21FB
:1056E800A1833CB1DC315CA1FC215CB18A251905A0
:1056F8003345050882809E211CA19E21A1831CB1EF
:10570800094582809E211CA19E21A1831CB1BE2136
:105718003CA1BE21A1833CB111458280CA21060566
:105728003345050882809E211CA19E21A1831CB1BE
:10573800AA2109053345050882809E211CA19E21C6
:10574800A1831CB1BE213CA1BE21A1833CB1CA21C9
:1057580011053345050882809C211CA105458280DE
:105768009E21411122C406C61CA19E212E8411052A
:10577800A183A30EF5FEBE219505230FF5FE83D761
:10578800D5FFA183A30FF5FE03C6F5FF97B0FB1F56
:10579800E780C0BB4820B240224411054101828005
:1057A80089476399F5001C3118210145A207D98F53
:1057B8001EA28280114582809A21011106CE22CC38
:1057C8002EC6D94763F4E7022A84EF80105CB246FC
:1057D8009E22636DF50022856244F2400147094626
:1057E800970500009385A5EC05615DBBF240624416
:1057F800094505618280AA87A9C11421FD150547BD
:10580800B3C505086398E60013D725008D891145AF
:1058180089CD8280094711456392E602494533D70D
:10582800A502B3F5A502114591E9114501CB8507FC
:1058380034A21AA25CC20145828011458280AE86DC
:105848000147114697050000938545E791BB13F77B
:105858003500AA8701EB8981114591C50EA25CC26A
:105868000145828011458280D8218947631BF70250
:10587800011122CC2A84C84506CEAE8601C92EC69F
:105888009D4597B0FB1FE7808097B2462A872285FF
:105898006244F2401946970500009385A5E3056127
:1058A80001B30945828099E1114582801C21054791
:1058B8003EA2E37BF7FEFD1593F5F50F33D7F5020E
:1058C800B387E702E392F5FE050548C21AA201452F
:1058D8008280DC210947AE866385E70041476399EA
:1058E800E70001472146970500009385A5E74DB9D4
:1058F800094582800EA291E1014548C20145828096
:10590800AE860147294697050000938505DF49B90A
:105918000EA291E1014548C201458280AE86014749
:10592800314697050000938525DE9DB90EA291E1C9
:10593800014548C201458280DA21854763FFE702B5
:10594800011122CC2A84884106CE2EC615C1854570
:1059580097B0FB1FE780A08A2A8722856244B24657
:10596800F240394697050000938585DB05610DB93E
:10597800F240624409450561828009458280AA8710
:105988008DC518218D46114563F2E602FD15B3C594
:105998000508B3C6E5023308D702639905018507F0
:1059A80016A23AA25CC20145828011458280DC21A0
:1059B8000947AE866385E70041476399E7000147D9
:1059C8004146970500009385E5D9D9BE09458280EF
:1059D8003335B0000A058280011122CC26CA06CED2
:1059E80098258547AA842E844946631FF70099366F
:1059F8003E2049151306200963C8A700F2406244F7
:105A0800D244094505618280183485476314F7003C
:105A180013660604484001C98D4532C697A0FB1F8E
:105A2800E780E07D3246A2866244F2402A872685D6
:105A3800D24497050000938545CF056195B68D47FB
:105A480063F7B7021C311821F115A207D98F1EA2DE
:105A58003C313821B3C50508A207D98F014799C140
:105A6800130745003EA24EA218C601458280114583
:105A78008280011122CC2A84884506CEAE8601C9CF
:105A88002EC6954597A0FB1FE7806077B2462A8708
:105A980022856244F240594697050000938525CA3D
:105AA8000561FDBC3335B0000A058280AE8601472A
:105AB800614697050000938565CADDB485471145A1
:105AC80063F1D7021C320C220945A207CD8F81450C
:105AD8006384A60093052600F9161EA336A34CC3BB
:105AE80001458280014781467946814555BC9E2102
:105AF8001CA19E21A1831CB109458280BC210547B8
:105B08001CA18A216397E7000A05050533450508A6
:105B18008280C9473305F502CDBF8A210A0533457E
:105B280005088280BE211CA18A21BE213305F50209
:105B380005053345050882808A2182808A21828072
:105B48008A218280BE211CA18A21BE213305F5024B
:105B580005053345050882809E211CA19E21A1834D
:105B68001CB1BE213CA1BE21A1833CB1CA211105B3
:105B78003345050882809E211CA19E21A1831CB16A
:105B8800AA2109053345050882808947114563988C
:105B9800F6001C3214220145A207D58F1EA382806D
:105BA8009A21D947AE8663F9E70001470D46970564
:105BB8000000938505F471BC094582801145639DF9
:105BC800A6001C3214220145A207D58F1EA33C3221
:105BD8003422A207D58F3EA38280BC210547FD173A
:105BE80093F7F70F6361F7049E2195CF011122CC3B
:105BF8002A84C84106CE2EC615C1894597A0FB1F29
:105C0800E780E05F2A8722856244B246F240154663
:105C1800970500009385C5EE056125BCF2406244F6
:105C280009450561828009458280954763F0D7065A
:105C3800411122C426C24AC006C61C323A84182220
:105C4800A207B284D98F1EA03C3238229385440023
:105C5800A207D98F3EA089475CA0094613055400C6
:105C6800368997A0FB1FE780606E19478147630458
:105C7800E90093876400691923142401B2405CC4C5
:105C880022449244024901454101828011458280A3
:105C98009E2195CF011122CC2A84C84106CE2EC65A
:105CA80015C1854597A0FB1FE78060552A87228587
:105CB8006244B246F2401D4697050000938525E6EA
:105CC800056141BAF240624409450561828009458F
:105CD80082809947B2856388F600D14711454146CD
:105CE8006384F60082800946411106C650A39C31A0
:105CF800942113055700A207D58F1EA3BC31B421E8
:105D08009105A207D58F3EA397A0FB1FE7800064EB
:105D1800B2400145410182809E219DCF011122CCD4
:105D28002A84C84106CE2EC61DC1894597A0FB1FEF
:105D3800E780E04C2A8722856244B246F240254635
:105D480097050000938545DE05616FF09F90F2404E
:105D58006244094505618280094582808947114569
:105D68006398F6001C3214220145A207D58F1EA3A2
:105D78008280011122CC2A84C84106CEAE8601C990
:105D88002EC6854597A0FB1FE7806047B2462A8745
:105D980022856244F2402D4697050000938505DA76
:105DA80005616FF01F8B19BD011122CC2A84C841EF
:105DB80006CEAE8601C92EC6854597A0FB1FE78093
:105DC8000044B2462A8722856244F2403546970548
:105DD80000009385E5D605616FF0BF8793F716003D
:105DE800114581EB89476386F600858256A310C367
:105DF80001458280011122CC2A84C84106CE2EC6D4
:105E08001DC1854597A0FB1FE780603F2A87228533
:105E18006244B246F2403D4697050000938585D21C
:105E280005616FF01F83F240624409450561828075
:105E38009E219DCF011122CC2A84C84106CE2EC6B0
:105E48001DC1894597A0FB1FE780603B2A872285F3
:105E58006244B246F2404546970500009385C5CE98
:105E680005616FF00FFFF2406244094505618280C9
:105E780009458280854763F4D70208A70CB71C320E
:105E88000C220945A207CD8F81456384A60093059E
:105E98002600F9161EA336A34CC30145828011457E
:105EA8008280014781464D4681456FF08FFA8D47C4
:105EB800114563F5D7021C320C22A207CD8F1EA311
:105EC8003C322C22A207CD8F81456384A60093051E
:105ED8004600F1163EA356A30CC701458280011166
:105EE80022CC2A84884506CEAE8601C92EC69545A1
:105EF80097A0FB1FE780A030B2462A87228562441C
:105F0800F2405D4697050000938545C505616FF031
:105F18004FF4854711456395F6001C2201451CA3E3
:105F2800828001478146654681456FF08FF20111F5
:105F380022CC2A84C84106CEAE8601C92EC68D451C
:105F480097A0FB1FE780A02BB2462A8722856244D0
:105F5800F2406D4697050000938525C205616FF0F4
:105F68002FE4011122CC2A84C84106CEAE8601C98D
:105F78002EC68D4597A0FB1FE7806028B2462A876A
:105F880022856244F2407546970500009385E5BE78
:105F980005616FF0EFE0011106CE2EC6EF90B03F1D
:105FA80019C5B245F2402A2105616FE0C005F240EB
:105FB80049450561828097E7FB1FA38B07FE97E79A
:105FC800FB1F238707FE97E7FB1F23A107FE97E721
:105FD800FB1F23AB07FC97E7FB1F23A507FC97E7ED
:105FE800FB1F23AF07FA97E7FB1F23A107FA97E7E1
:105FF800FB1F23AB07F897E7FB1F9387A71C370600
:10600800840390D33707B40037C6070098C3130634
:1060180006B83747A000D8C3D0D337071000416669
:106028009306070AB70550009308060194C723A4EE
:10603800170393860501930816F8D4C723A61703F8
:10604800B706D007B7087F001308070513850601B0
:10605800410723A81703B0C39308160093860605C3
:1060680013861500D8CBF8C323A8070188CF23AE21
:10607800070023AA170323AC070223AE070223A4B1
:106088000704F0C7B4CB23AA0704ACCF23AE070597
:10609800B8D33707A000F8D71307000AB8DB1307EF
:1060A800C01CF8DB37071400B8DF0547F8DFE8D372
:1060B80023A40706930710F817E7FB1F2324F718F4
:1060C8008280011152C42A8A214522CC26CA4AC894
:1060D8004EC606CE2E84B2893689BA8497A0FB1F95
:1060E800E780001705C9930700FD1CA19947A30085
:1060F80045013CA12303250164B123123501AA857A
:1061080022856244F240D2444249B249224A05619A
:106118006FE0AF94F2406244D2444249B249224A05
:106128000561828097E7FB1F23A2A7E8828097E793
:10613800FB1F23ABA7E6828097E7FB1F23A4A7E6F4
:10614800828097E7FB1F23ADA7E48280011122CC50
:1061580026CA4AC806CE4EC62A89AE840144B30967
:10616800890063699400F2406244D2444249B249CA
:1061780005618280EFE0EF98B3470508A18323808B
:10618800F9009307140093F7F70F850963F8970050
:10619800CA97090488A31374F40FD1B73E84D1B702
:1061A800411122C417E4FB1F1304040A6A20C167C3
:1061B80006C6FD17630EF50017E6FB1F0346C62A41
:1061C80097E5FB1F9385C5DCEF90E07DFD577EA02A
:1061D800B24022444101828009C925151375F50F83
:1061E8001335850E13451500828001458280239062
:1061F8000500C9C2797122D426D252CC56CA5AC8CF
:1062080006D64AD04ECE5EC62A8B2E8AB28A3684ED
:10621800814463FF5405B307940083C907001389B9
:1062280014003349090863850904B387290163C148
:10623800FA04B307240183CB07005E85713F0DC9BB
:106248009387F9FF2310FA0063906B030509330560
:106258002401B250225492540259F249624AD24A55
:10626800424BB24B45618280CE94B3C4040855B703
:106278000145C5B701458280011122CC26CA4AC80A
:106288004EC606CE97E4FB1F938404FC2E89D0C823
:106298008CC8C8C42A8441469305F00F4A8597A044
:1062A800FB1FE78040248549631935038848C145A9
:1062B800713D41469305F00F228597A0FB1FE780AB
:1062C80080220549631525036244C844F240D2443C
:1062D8004249B249C145056195BD414681454A8556
:1062E80097A0FB1FE7802020E31535FDC1B7414685
:1062F8008145228597A0FB1FE780E01EE30625FD68
:10630800F2406244D2444249B24905618280411157
:1063180022C426C22E84AA8413060002814517E5EA
:10632800FB1F130565F206C64AC097A0FB1FE7804E
:10633800600817E9FB1F130929F197E7FB1F23875B
:106348008712A3019900EFD0504E854719C18147A4
:1063580049452300F900B2402244924402494101D0
:1063680082809DC91DC985476318F500DC3193E714
:1063780007FCDCB10545828089476316F500DC31EE
:1063880093F7F703FDB78D47E316F5FEDC3193F776
:10639800F70393E70704F1BF014582808DC10DC162
:1063A800DC311307000C054593F7070C638AE700F7
:1063B8001307000409456395E7000D4582800145F0
:1063C8008280411122C4005D06C626C21DC8AA8467
:1063D800085009C597A0FB1FE780E0D4485009C5BD
:1063E80097A0FB1FE78020D4085409C597A0FB1F7E
:1063F800E78060D3228597A0FB1FE780C0D223AC3B
:106408000402B240224492444101828019ED97E788
:10641800FB1F83C787E317E5FB1F130565E491CBD3
:1064280017E5FB1F130545B7828017E5FB1F13050A
:1064380025E3828017E5FB1F034525E1828017E5E8
:10644800FB1F032525E1828017E5FB1F0325C5E017
:10645800828097E7FB1F83A767E08843828017E75E
:10646800FB1F130767DE544B9C4285079CC22833E9
:106478009307F00F6307F500916517C3FB1F6700CB
:1064880043588280011122CC06CE2E8432C6EF906A
:1064980010019147B245631EF50097E7FB1F83A7DC
:1064A80027B099CF9C4389CF22856244F240056189
:1064B800828797E7FB1F83A727AF99C3DC43E5B71C
:1064C800F2406244054505618280797122D42A84AC
:1064D8004A214ECE06D626D24AD097C0FB1FE78067
:1064E800006997E9FB1F9389A9AC29E983C40900CE
:1064F8009307F00F639DF40097E5FB1F83C555AB29
:106508002685513C09E597E7FB1F238307AA4A2004
:10651800EF90E0789147631CF50097E7FB1F93879E
:10652800A7D25620FA236394E6007D57FAA3B25007
:10653800225492540259F249456182805825042117
:106548002A893AC6BD3D4A85EF9030344A20EF90FB
:10655800407083C70900324799C3E38F97F89307C0
:10656800F00F5220E385F4FA74202820A685913E86
:1065780079BF79715AC82A8B2E854ECE52CC56CA0D
:1065880006D622D426D24AD05EC62E8AB28AB689C8
:1065980097C0FB1FE780A05D75C5045D2A89FDC013
:1065A8009C501305400391E361459C5489C79307A8
:1065B800450133C50708638609009307C50133C53C
:1065C8000708DC5089C79307750133C5070897A0EA
:1065D800FB1FE780E0C72A8455C56146814597A01F
:1065E800FB1FE78020DD97EBFB1F83CBABC06394D9
:1065F8000B00834B0900930700FD1CA0A947A300CB
:1066080064013CA0230354018C5023124401130558
:10661800840191C908C47146130A440397A0FB1F5B
:10662800E780C0D252858C5491C948C45146130A98
:10663800450197A0FB1FE78060D15285638C090054
:1066480008C87146CE85130AC50197A0FB1FE780CD
:10665800E0CF5285CC5099C548C85D4697A0FB1F2E
:10666800E780C0CEA2855E85EFD03FBF2254B250EE
:106678009254F249624AD24A424BB24B4A85025975
:10668800456181B3B250225492540259F249624A88
:10669800D24A424BB24B4561828001114EC6AA894B
:1066A8002E8526CA06CE22CC4AC8AE8497C0FB1FC8
:1066B800E780E04B21C917E9FB1F0349A9B363141D
:1066C800090003490500194597A0FB1FE78040B85A
:1066D8002A840DC98145194697A0FB1FE78080CD04
:1066E800930700FD1CA0B947A30034013CA046A0B5
:1066F800A2856244F240D244B2494A8542490561C2
:106708006FD0BFB5F2406244D2444249B2490561F4
:106718008280797162C42A8C2E8526D24ECE52CCC4
:1067280056CA5AC85EC606D622D44AD0AE84B28BA0
:10673800368BBA8A3E8AC28997C0FB1FE7802043FE
:1067480035C52A89414597A0FB1FE78060B02A8498
:1067580031CD4146814597A0FB1FE780A0C517E5CD
:10676800FB1F034525A919E103450900930700FD0F
:106778001CA0BD47A30084013CA023047401A3040A
:10678800640123055401A305440146A023263401CE
:10679800A2852254B25092540259F249624AD24A0E
:1067A800424BB24B224C45616FD03FABB2502254A2
:1067B80092540259F249624AD24A424BB24B224C95
:1067C80045618280011126CAAA8439454AC84EC645
:1067D80052C406CE22CC2E8AB289368997A0FB1FD6
:1067E800E78000A715CD9307000D1EA1B1472A84A5
:1067F800231245013CA1CE851905194697A0FB1F18
:10680800E780C0B423062401A2856244F2404249CD
:10681800B249224A13F5F40FD24405616FD0FFA3A1
:10682800F2406244D2444249B249224A0561828018
:10683800411126C206C622C44AC097E4FB1F9384AE
:10684800A4A0B8309307F00F6308F7042A893945E4
:1068580097A0FB1FE780C09F2A841DCD930700FDEA
:106868001CA1A30025012301050097E5FB1F9385C3
:10687800259F0D05194697A0FB1FE78020AD9E2494
:10688800A285A8303EA49C305CA42244B240924425
:10689800024941016FD07F9CB24022449244024990
:1068A80041018280011156C2AA8A314526CA4AC8C6
:1068B8004EC652C406CE22CC5AC0AE84328AB6899D
:1068C8003A8997A0FB1FE780A0982DCD2A842685BA
:1068D80097C0FB1FE780A02909C55825A147631168
:1068E800F70417EBFB1F034B5B96930700FD1CA0F7
:1068F8009D47A30054013CA046A023134401231440
:10690800340123152401A2856244F240D24442494D
:10691800B249224A924A5A85024B05616FD0FF93C9
:1069280017EBFB1F034B9BB4E3910AFC97D7FB1FA4
:1069380083A7477C9C47D5DBCA864E86D2852685A9
:10694800829765B7F2406244D2444249B249224A2A
:10695800924A024B05618280411126C2AA842145D0
:1069680022C406C62E8497A0FB1FE780608E15C53B
:10697800930700FD1CA1C5473CA13C30AA853CB14A
:106988005E205EA17C207CA17C307CB12244B24098
:106998002685924441016FD05F8CB24022449244D4
:1069A8004101828041114AC02A89714526C206C622
:1069B80022C4AE8497A0FB1FE78080893DC593075A
:1069C80000FD1CA1F5473CA1BC302A849385C40076
:1069D8003CB1DE2031051946231CF5FEFE20231D9F
:1069E800F5FE9E24231EF5FEBC24230FF5FEBC34C1
:1069F800A30FF5FE97A0FB1FE7804095BC28A28552
:106A08004A853CA8DE285EA8FC287CA8FC387CB80F
:106A18009C2C1CAC9C3C1CBCBC2C3CAC2244B24006
:106A28009244024941016FD05F83B24022449244AC
:106A380002494101828001114AC82A89614526CA52
:106A48004EC606CE22CCAE89B28497A0FB1FE78043
:106A5800208025C1930700FD1CA1BC302A849385A2
:106A680084001CB195473CA1FC3011051946A30FC1
:106A7800F5FE97A0FB1FE780608DDE20230634011A
:106A8800A2853EA4BE2C4A857EA4DE2C1EA8FE2C20
:106A98003EA883C704025CA883C714025CB8BE3052
:106AA800F240D2447EA862444249B24905616FD09F
:106AB800CFFAF2406244D2444249B2490561828029
:106AC800411122C406C617D4FB1F1304E4773C20E7
:106AD8009DCBAA85194617D5FB1F1305E54B97A033
:106AE800FB1FE780A086282097D5FB1F9385C54A02
:106AF800EFF03F872244B24017D5FB1F1305C54965
:106B080041016FD04053B240224401454101828087
:106B1800411126C206C622C44AC097D4FB1F9384DB
:106B2800A472B8309307F00F6302F7042A89294545
:106B38009790FB1FE780C0712A840DC9930700FD59
:106B48001CA1A147A30025013CA1BC2097D5FB1F90
:106B5800938585441105A30FF5FE19469790FB1FF1
:106B6800E780C07EA830A285EFD02FEFB8208D47F0
:106B7800631FF70097D7FB1F83A7C74289CB9C47A2
:106B880099C72244B2409244024941018287B240E7
:106B980022449244024941018280797122D406D666
:106BA80026D24AD04ECE52CC56CA09444DCD2A8957
:106BB8000A212E8A514497C0FB1FE78040FBAA8414
:106BC8005DC197EAFB1F938A2A8A83C74A00054753
:106BD8004944FD1793F7F70F6377F7085825A1473E
:106BE8006314F70063110A089C5C4544ADEF916596
:106BF800938545711305C0029790FB1FE780804578
:106C080088DCAA894D4425C11306C00281459790A6
:106C1800FB1FE780207A8357090093864900368551
:106C28002391F90071469305490036C69790FB1FDA
:106C3800E780C07189472380F900DC24B2460356F7
:106C4800090083C50A00E11713B51700EF90907D7E
:106C58002A8463060A00D2852685EF90607201C4F3
:106C68002685EFF00FF6B25022852254925402592D
:106C7800F249624AD24A4561828097D7FB1F83C78F
:106C8800E77EFD1793F7F70F05476377F7080111BC
:106C98004AC806CE22CC26CA4EC652C43289894773
:106CA8002DC22A8AAE89368497C0FB1FE78020EC64
:106CB800AA84D14739C5485509C59790FB1FE78075
:106CC8008046F1454A859790FB1FE780C074C8D479
:106CD800AA85CD471DC5D824A147631DF70209C859
:106CE800382D1229930625015285EF90C06F2A840A
:106CF800D820936747006384090093676700DCA086
:106D0800A287F2406244D2444249B249224A3E85AF
:106D1800056182800144E9BFC9473E8582809307A7
:106D2800000463EAA70097D7FB1F9387A749332579
:106D3800F5200A21828041657D158280011122CCCF
:106D48002A842E8526CA06CEAE8497C0FB1FE7800C
:106D580000E20DCDB7470F009387F723094563E29B
:106D6800870281450A8541469790FB1FE78080642A
:106D7800A68560800A8541804081A3010100EF90CB
:106D8800304AF2406244D244056182804945D5BF09
:106D980097D7FB1F238BA76C82806F901063797144
:106DA80052CC2A8A328526D24AD04ECE56CA5AC8E2
:106DB8005EC662C406D622D42E8CB28A368BBA8BB3
:106DC8003E89C289C68497C0FB1FE78040DA05C99F
:106DD8002A84631A0A1893774B000343450085CF2A
:106DE8001363230163940B1663100914639F090846
:106DF80085E81C5C1373B3FF23026400C5EBB25033
:106E0800225492540259F249624AD24A424BB24B36
:106E1800224C456182801373D3FF13630301D9B7F2
:106E280013634300230264009C484146A6851CD492
:106E3800130584019790FB1FE780405163130C12E0
:106E4800638C0B0A485409C59790FB1FE780A02D57
:106E5800F1455E859790FB1FE780E05B48D4005CB6
:106E680059DC1C5091EB916593853571714597906C
:106E7800FB1FE780201E08D008500DC17146DE8533
:106E88009790FB1FE780804C11A8136343002302EF
:106E98006400D9F8005C630C0C0235D0639A0902CF
:106EA800A5E029A0005C21DC639409022254B250B9
:106EB8009254F249B24B224CCA865A860259424B26
:106EC800D6855285D24A624A45616FF08FEA05D865
:106ED8005C5091EB9165938525715D459790FB1FFB
:106EE800E780401748D0485045DD5D46CE859790ED
:106EF800FB1FE780A0456DB7005C11D0E39A09FC41
:106F08001C5491EB91659385157151459790FB1F22
:106F1800E780401408D4085451D95146A685979063
:106F2800FB1FE780A04259B71363430023026400A4
:106F3800E39C04EEE3080CF6485405EDF1454A8558
:106F48009790FB1FE780204D48D431A81363430076
:106F580023026400E39A04ECE3060CEEE31E09FC4A
:106F6800FDBDE31B09FC005CE30B04E8E39B0BEEAF
:106F780035B79790FB1FE780001BC9B7011126CAD8
:106F880052C406CE22CC4AC84EC62A8AAE8497C0BE
:106F9800FB1FE780C0BD35C12A8939459790FB1F83
:106FA800E780002B2A8431C997D9FB1F83C989241C
:106FB80063940900834909009307000D1EA0AD479B
:106FC8003CA0930569001305340019469790FB1FF0
:106FD800E780C03793F714005CA493D4144844B4F2
:106FE80023154401A2856244F240D2444249224A10
:106FF8004E85B24905616FD04FA6F2406244D24433
:107008004249B249224A0561828001114EC652C4E2
:1070180056C206CE22CC26CA4AC8AA8A2E8AB28965
:1070280097C0FB1FE780A0B435CDAA841305C00222
:107038009790FB1FE780C0212A842DC517D9FB1F15
:107048000349491B6314090003C904009307000D91
:107058001EA0E9473CA09385640013053400194637
:107068009790FB1FE780802ED285231554011305C6
:10707800C40041469790FB1FE780402DCE8513053D
:10708800C40141469790FB1FE780402CA2856244CB
:10709800F240D244B249224A924A4A85424905619D
:1070A8006FD0AF9BF2406244D2444249B249224A6F
:1070B800924A0561828017D5FB1F0325E5EC11CDA7
:1070C800411106C69790FB1FE780E005B24097D7AD
:1070D800FB1F23AB07EA410182808280411122C451
:1070E80006C626C24AC02E8497C0FB1FE78020A888
:1070F80029CD00D517D9FB1F0349C90FAA846314EA
:1071080009000349050041459790FB1FE78040149B
:107118002A8405CD9307000D1EA1A5473CA1DC30AC
:10712800938564001105A30FF5FE19469790FB1F80
:10713800E780C0219C54A285B2405CC4224492449A
:107148004A85024941016FD04F91B240224492448E
:107158000249410182805D71A2C4A6C286C6AA8482
:107168002E8497C0FB1FE78080A00DC954251147C6
:10717800AA874945639FE6009C5F91C3E02B97B6B9
:1071880000009386069A0A86894526854080EF90F6
:107198002016B64026449644616182805145D5BF89
:1071A80097D7FB1F83C7872CFD1793F7F70F054762
:1071B800637AF704411126C206C622C44AC0B284C3
:1071C800894715CA2E8997C0FB1FE780409A2A84F1
:1071D800D14715C1630609005C2193E727005CA12C
:1071E8004146A685130584019790FB1FE78000168A
:1071F8009C481CD48147B2402244924402493E85AF
:1072080041018280C9473E858280011122CC26CA6D
:1072180006CE2A84AE8497C0FB1FE780409519C923
:107228006C0022854486EF904012F2406244D244BA
:10723800056182805145D5BF6F80701BC167138778
:10724800E7FF6393E50297D7FB1F83A7E7D591EB89
:10725800494582804945B24022449244024941014D
:1072680082809C43F5D78287411122C426C24AC036
:1072780006C6FD172A892E84B284639AF50297D729
:10728800FB1F83A767D289C79C4399C3829711C5FF
:10729800A6854A85EFE03FD05DFD97D7FB1F238980
:1072A80027D197D7FB1FA38597D001456DB72E85AA
:1072B80097C0FB1FE780A08B51DD1C210D45E39C87
:1072C80027F922852244B2400249A6859244410109
:1072D8006FC070539307000463E1A7064111C167AB
:1072E80022C426C206C6FD172A84AE8409456380D7
:1072F800F502C5476312F4022E85EFC0705897D780
:10730800FB1F938727EC3324F420014506A0B240E5
:1073180022449244410182809307A0036316F4003B
:107328002E85EFC0104FE1BF9307B003E319F4FCBB
:1073380013F5F50FEFC0304ED9B70945828001111A
:1073480006CE2AC6EFE03FC7EF20404EEF10C07CC4
:10735800EF501236324597D7FB1F9387E7EE130796
:1073680000F0BAA3238207007D5797D7FB1F9387A6
:10737800A70FB8A388A3F240954505616F70202A2E
:10738800757126C306C722C54AC1CEDED2DCD6DA5D
:10739800DAD8DED6E2D4E6D2EAD0EECEAE8493973F
:1073A800556063D1075817DAFB1F130AEA0B034528
:1073B8000A00130B200A930BF00F9790FB1FE7802E
:1073C80020EFC167FD172A84130C1009954C394D1D
:1073D80097DDFB1F938D4DE73ECC15E01395F468C0
:1073E800BA402A449A440A49F659665AD65A465B1C
:1073F800B65B265C965C065DF64D496182801C2072
:10740800639A670103C93D00E2452A202286EFF00E
:107418006F87E1A003492A00639A87091C306390AB
:1074280097032285EFF06F8A2285EFC0FFDD0345C1
:107438000A009790FB1FE780A0E72A8479BF639B27
:10744800A7194A208567A507631AF5040C4497D93C
:10745800FB1F938969DF882115E51946850517D52E
:10746800FB1F1305E5DF9790FB1FE78020EE03C79E
:1074780009008547631CF70289472380F900EFC09C
:10748800503B5DB703C7090085476311F70297D7DB
:10749800FB1F238B07DAEFF0AFB979B709679307BA
:1074A800C70063EFA7040507636BA702E30E79F72C
:1074B800A2854A85EFC07FDA9DBF370700181307FA
:1074C800F770B357F748E5CB97D7FB1F83A787AD6E
:1074D800A1DF9C43B1DB2285829739F5C1BFF977DB
:1074E800F917AA972947B3C707086366F70C176700
:1074F800020013072760B3C7E7209C43BA97828727
:10750800F9779387A7FCAA97F146B3C70708E3F66C
:10751800F6FA3907E31CE5F897D7FB1F83A7C7A836
:10752800E38407F0DC43E38107F00965A2853905A8
:10753800A5A883298400E38B09F603C7090097D718
:10754800FB1F938767D019EB03C7290083C619006F
:107558002207558F9AA703C7390098B39423094780
:10756800E396E6F403C7090001CB97D7FB1F238DE9
:1075780007CC03C5090005B78C338A270D4798A3A4
:10758800EF70800CFDB71C448823EFF06FD869BDFD
:1075980097D7FB1F83A787A1E38807E89C43E38568
:1075A80007E80965A2852D05829705BF1C449C2321
:1075B800E39E07EE95BD896793871704E318F5EEF8
:1075C80097D7FB1F83A7879EE38007E69C43A28586
:1075D800E1FF99BD3D476394E7064A208967138711
:1075E800D7006306E50013879701631AE50097D76C
:1075F800FB1F83A7679BE38907E2DC43C9BFCD076D
:10760800E316F5EAC16717D7FB1F035747C4FD17F1
:10761800631FF70097D7FB1F83A70799E38607E047
:10762800DC43E38307E00965A2854D05B5BF97D71D
:10763800FB1F83A7E796E38907DE9C43DDB71307A3
:10764800E003E395E7E63C2005476398E7127C20D2
:1076580097DAFB1F938A4A936390071083A70A005F
:107668006387070E83C907002149683093078400A0
:10767800BE853ECEEFE09FD268B01306400281453A
:1076880068109790FB1FE780E0D23C3019469305BD
:107698008400A307F1027C304818A309F1029790EF
:1076A800FB1FE780A0CA5E207010CA852318F1026C
:1076B8007E244E852313F1041E282314F1043E284A
:1076C8002315F1045C282306F104FD57A306F104F1
:1076D8002317F104EFF02FB63C309DE3DD478358C4
:1076E80004010358E40074304E203EC23E281307BC
:1076F80084003EC0CA8705464E85EF80807128B059
:1077080083A70A0081C71145EFF0FF9A97D9FB1F9D
:107718009389098A03C50900E30805D097D5FB1F9B
:1077280083C51589EFE03F87E30005D03430930720
:1077380010036389F600522083C509004A873685FD
:10774800EFE03F9897D7FB1F23840786F1B997D9B5
:10775800FB1F83C999AF09BF97D7FB1F83A78784EE
:1077680097D9FB1F83C979AE99C3DC4399E31149C3
:10777800EDBD814501458297DDBFF91793F7F70FF6
:1077880013077002E364F7D217670200130747393B
:10779800B3C7E7209C43BA9782877C2097CAFB1F10
:1077A800938A8A7EA9EB83A70A00A9C383C9070025
:1077B8002149683093772500A5C30589130744013B
:1077C80068B02286CA854E853ACEEFF0CFA63C3007
:1077D80072479DF7DD478358C4010358A4017430EC
:1077E8004E203EC27E2C3EC0CA8731B797D9FB1FB8
:1077F80083C9B9A575BF97C7FB1F83A7A77A97D970
:10780800FB1F83C999A499C3DC4399E3114955B770
:10781800814501458297DDBF13078400BA853ACEBA
:10782800EFE0DFB7724769BF97C7FB1F83A70778E9
:10783800E38C07BEDC43E38907BE22858297EDB659
:1078480097C7FB1F83A78776E38007BE9C47E5B7EA
:1078580022868D454A2065BE9305A1021305103185
:10786800EF50E26C6C1013052031EF50426C72201F
:107878008357C1024A2063E7C70016240357A102B1
:1078880063F7E60093050002EFC0807E71BE637364
:10789800E6007AA063F3D7001EA45A2436241224E3
:1078A8006E2001488147EFC0607CBDBE2286B1458D
:1078B80055B797C7FB1F83A7676FE38707B6DC47F2
:1078C8009DBF2285EF00607B85B697C7FB1F83A706
:1078D800E76DE38B07B49C4BB9BF2285EF00F0033B
:1078E800A1B60145EF00301381B697C7FB1F83A7E8
:1078F800676BE38D07BADC43E38A07BA8145054520
:1079080082976DB697C7FB1F83A7C769E38007BA3D
:10791800DC43E38D07B8A2850945DDB722869305C8
:1079280060020DBF93F7150089CF97C7FB1F83A788
:10793800E76789C7DC4399C30145829713C51400DB
:1079480045B493F7250091CF97C7FB1F83A7876599
:1079580091C7DC4381C781450545829713C524003B
:1079680041B413F54500E30D05A697C7FB1F83A790
:10797800E76117D4FB1F1304248D89CF85475CA0CA
:1079880097C7FB1F83A7076291C7DC4381C781455F
:107998000545829748446C10EF8010756810EFF029
:1079A8002F9297D7FB1F83D7078481CF13060064D4
:1079B8003386C702914517D5FB1F0345E5AAEFC0DB
:1079C800FFAF13C5440029BC011122CC2A845545B8
:1079D80006CE26CAEFF0AFB4AA8413054002EFF032
:1079E8000FB42AC613055002EFF06FB3AA8622859A
:1079F80062443246F240B3359000D24405616FC00C
:107A0800006F397122DC06DE0D472E84631AE5000B
:107A1800BA259625F2212830CE21EFE0BFE899A8B3
:107A280009679306D700AA87631BD504BC21B9C38D
:107A380017C4FB1F130444550C408DCDDC87BC31A3
:107A4800194691054808A309F1009790FB1FE780A4
:107A5800E08F930700F03ED61C4023180100231343
:107A6800010202D4882370008145EFE0DFFC054560
:107A7800EFF06FE40545F25062542161828093066D
:107A8800E700E309D5FE930637016319D500A8215D
:107A980075D1014781460146814541B76507E30B2A
:107AA800E5FC31476319E50017C5FB1F0345F57968
:107AB800EFE09FEAC1B7130760026319E50017C535
:107AC800FB1F03459578EFE0FFED6DB741677D1724
:107AD8000145E392E7FAD831C947E31DF7F8F625DF
:107AE800D2250A24AE25EFC02068854711C55D451B
:107AF800EFF0EFA2B337A0004C202A2030007C849E
:107B0800EF70D06B3C84BDF79305A10013051031CD
:107B1800EF50E2416C0013052031EF5042413C85A3
:107B28001A246373F7001EA43C863A2463F3E70023
:107B38003EA41E243A246373F7003EA42A20EF4093
:107B4800212C7A24562432240E242A2001488147E5
:107B5800EFC0A04F05B741114AC006C622C426C2CD
:107B680017D9FB1F13094990034779009307F00FB2
:107B78006302F706AA8439CD682551059780FB1F53
:107B8800E780006D2A8439C59307000D1EA1D947E7
:107B98003CA1DE205EA1FC207CA1FC307CB19C24B1
:107BA8001CA5DC345CB5F02470A515C28C485105C1
:107BB80008C89780FB1FE7806079A28522440345A7
:107BC8007900B2409244024941016FC00FE923286D
:107BD8000500E5B7B240224492440249410182803F
:107BE800C1679386E7FF2A87639DD50097C7FB1F68
:107BF80083A787398DC39C230D45639FE7006FC01A
:107C08000044FD1749456399F50097C7FB1F83A7F3
:107C1800A737F5F7828049458280397122DC06DE74
:107C280026DA4AD84ED652D456D25AD01821854789
:107C38002A84630BF7001025930695009305E1014C
:107C48000545EFE0CFDA0DED8147014514201147D6
:107C5800638FE60217C7FB1F0327473618338D4685
:107C68006307D7028DC705C711ED0145F25062546D
:107C7800D2544259B259225A925A025B21618280E7
:107C88001C21E9B785466311D7048D8BF9DF0830CD
:107C9800930524002EC6EFE06FF008B017C9FB1F4C
:107CA8001309093283270900AA8981449DC3B24573
:107CB80017CAFB1F130A0A31130BF00F83470A0078
:107CC80063EBF400814481A08946E310D7FA858BE1
:107CD80075BF054561BF83270900939A4400D6976D
:107CE8009823630C6705983363193705194613857C
:107CF80027002EC69780FB1FE780C076B24515CDBA
:107D080083240900D69418209147C1E8E30FF7F4BB
:107D180083240900B9D883460A0081471306F00F67
:107D2800E385F6F403C8040013850401630BC80057
:107D3800850793F7F70FAA84E5B7850493F4F40F42
:107D4800B5BF98A01C301385240019469CB09780B5
:107D5800FB1FE780A05F082491659385F5710505F1
:107D68009780FB1FE780002F05C1182091476314F7
:107D7800F702C8C41024930594000505A30FC5FE97
:107D88009780FB1FE780805C1C24A1F708207D15E5
:107D980013351500E1BD88C4F1BF6311F706C84467
:107DA8001C2405C11021630DF604182091476317A0
:107DB800F706C84419C59780FB1FE780C03623A67D
:107DC8000400082491659385E57105059780FB1FDC
:107DD800E780402805C118209147631AF704C8C4F2
:107DE8001024930594000505A30FC5FE9780FB1F7B
:107DF800E780C05508243335A0008DBD88444DB7B1
:107E08009305940005059780FB1FE780A0658547CB
:107E1800E31DF5F85545EFE09FF09DBF884455D127
:107E28009780FB1FE780203023A4040059BF88C433
:107E380045BF397122DC4AD84ED652D406DE26DA3E
:107E480056D25AD05ECE2A84130925000831CA8535
:107E580017CAFB1F130A8A16EFE04FD408B083270E
:107E68000A000D47AA899C336391E70217CAFB1FD2
:107E7800130A0A1583270A00814497CAFB1F938AAD
:107E88006A146393071005452DA0EDD3144C703880
:107E98009305E1000545EFE08FB5AA841DC90327C6
:107EA8000A0085461C2118336310D7028D8BDDFF2D
:107EB8000145F2506254D2544259B259225A925A48
:107EC800025BF24B216182808946858BE310D7FAE9
:107ED800F9BF1C2011476385E7002D47E39AE7FCAB
:107EE80097CAFB1F938ACA0D83A70A00014A97CB3A
:107EF800FB1F938B2B0DCDDF03C70B00B3470A087D
:107F080063E4E700A5F46DB703A50A00131B4A0054
:107F18001C205A9518216310F7021C31639D370104
:107F28001946CA8509059780FB1FE780A05301C53C
:107F380083A40A00DA94050AC1B783A9840059A862
:107F48000C4C138519009780FB1FE780A0518547CB
:107F58006317F5085545EFE09FDC4DC191BF1C2024
:107F680011476385E7002D47639DE700C8C4703853
:107F78000505A30FC5FE0C4C9780FB1FE780003D4D
:107F8800B5A888C4EDB7850403C70A00B3C70408B9
:107F980063F8E70603250A00139B44001C205A9542
:107FA8001821E312F7FE1C31E39F37FD1946CA85F5
:107FB80009059780FB1FE780E04A71D583240A00F2
:107FC8001C201147DA946385E7002D47E397E7F60D
:107FD80083A9C4007C3803C60900E303F6F64E857E
:107FE8009780FB1FE7802014683891659385E571B9
:107FF80005059780FB1FE780E00535F1E39504E868
:1080080003C70A0083240A0081479306F00FE3FCA4
:10801800E7E68C20138604016387D5008507B284C0
:10802800B3C70708EDB7E38004E61C20CA851385AB
:1080380024009CA01C3019469CB09780FB1FE78049
:10804800E030683891659385F57105059780FB1FC9
:10805800E7804000E30905E218209147631DF70017
:10806800C8C470380505A30FC5FE0C4C9780FB1FCC
:10807800E780C02D09BD88C4EDB701114AC806CEF6
:1080880022CC26CA17C9FB1F1309093E03477900EA
:108098009307F00F630DF706AA8435C961459780E9
:1080A800FB1FE780E01A2A843DC19307000D1EA13B
:1080B800D5473CA1BC30938584002EC63CB1DE2058
:1080C8005EA1FC207CA1E830EFE04FADB24568B07E
:1080D8001946130584009780FB1FE7802027FC249E
:1080E800A285034579007CA49E281EA8BC283CA82C
:1080F800BC383CB8DC285CA8DC385CB8FC287CA818
:108108006244F240D244424905616FC00F95F24083
:108118006244D244424905618280411126C206C6A2
:1081280022C497C4FB1F93842434F8309307F00FBC
:108138006309F7022A8415C519459780FB1FE78054
:108148002011AA8519CD9307000D1EA1DD473CA17A
:108158005E202244B2405EA1E830924441016FC0E3
:10816800CF8FB2402244924441018280011126CA35
:1081780097C4FB1F9384C4E49C4006CE22CC4AC813
:108188004EC652C49DC32A89AE89131A45000144BC
:10819800884063144403638C09049780FB1FE780BD
:1081A80080F897C7FB1F23AD07E0F2406244D24432
:1081B8004249B249224A05618280B307850088474F
:1081C80009C99780FB1FE78000F69C40A29723A46B
:1081D80007009C40A297C84709C99780FB1FE78002
:1081E80080F49C40A29723A60700410455B755DDAB
:1081F800228681459780FB1FE780C01B94408147FA
:108208007D5613F7F70FE37227FB1397470036974E
:1082180010A38507FDB7797152CC17CAFB1F130A43
:10822800EAD983270A0006D622D426D24AD04ECECF
:1082380056CA5AC85EC6E9C72A8997CAFB1F938AD5
:108248006AD8814419ED97C6FB1F83A666D791CAE1
:1082580003C60A0081479305F00F13F7F70F636908
:10826800C7021395340021059780FB1FE78040FE65
:108278002A8415E921459780FB1FE78060FD2A8441
:1082880035C1C5679387073D1CC123220400A9A0F7
:1082980013974700369718236305B700850493F4AE
:1082A800F40F85075DBF930700FD1CA18547A30058
:1082B80025013CA124B1F1D8130985002322250109
:1082C800814917CBFB1F130BABCF930BF00F83C761
:1082D8000A0063F3F900A1E083270A00A285882336
:1082E800EFB0BFF703C50A008145493503250A00E9
:1082F8009780FB1FE78020E397C7FB1F23A007CCCD
:10830800B250225492540259F249624AD24A424B1C
:10831800B24B4561828083250B0093974900BE9537
:108328009C21638377032300F9009C3113052900FE
:10833800FD14A300F9001946890593F4F40F9780FA
:10834800FB1FE780A0002109850993F9F90F41B7C0
:1083580097C7FB1F83A787C6A9C7411122C406C6B2
:108368002A8415E10945EFE09F9B2A8601C98545C6
:1083780017C5FB1F0345450FEFC04F940545EFF0A8
:10838800AFE42A8411C9854517C5FB1F0345C50DF0
:10839800EFC02FBC22854135B2402244054541013A
:1083A80082800145828089679386B7006315D5006E
:1083B8009C45882371BF9386C7006317D5009C45E9
:1083C8008546882319C9FDB793861704E302D5FEAD
:1083D800938727048146E304F5FE368582800111E0
:1083E80006CE22CC26CA4AC84EC652C456C261C15D
:1083F8003C312A898DC3444199CC5945EFE03F92DD
:10840800814997CAFB1F938A6ABB131A4560834741
:10841800390063EBF900F2406244D2444249B24960
:10842800224A924A056182808387840263C847078B
:1084380083A70A00A5C72685EFF02FFE25C188244B
:1084480051059780FB1FE780A0E02A8421C9930784
:10845800000D1EA1B5473CA19C2019469385240018
:108468003CB18387840215057CA19C30A30FF5FEDF
:108478009780FB1FE78080ED902450A415C6130554
:10848800440108C8938594009780FB1FE78000EC9F
:1084980083A70A00A2858823EFB03FDC850993846F
:1084A800940293F9F90FA5B723280400D5B797C705
:1084B800FB1F83A7A7B0A5D3B93B6244F240D244BF
:1084C8004249B249224A924A014505616FF0CFCF2D
:1084D800797106D622D426D24AD04ECE52CC56CA6C
:1084E8005AC85EC655CD3C312A898DC744419DC0C6
:1084F8005945EFE0DF828904814997CAFB1F938AB7
:10850800EAAB130B00FDC14B131A456083473900D2
:1085180063EDF900B250225492540259F249624A6A
:10852800D24A424BB24B456182808387D40063C4F0
:10853800470783A70A00A5C351459780FB1FE7801B
:1085480020D12A8429C923006501A300050023013D
:10855800750183C7E4FF1946A6853CB18387D4001B
:1085680015055CB583C7F4FFA30FF5FE9780FB1FC5
:10857800E780C0DDFC20938574001305C4003CB47B
:1085880019469780FB1FE78060DC83A70A00A28555
:108598008823EFB09FCC850993F9F90FC104BDB7C3
:1085A80097C7FB1F83A787A1B5D7B5312254B2500F
:1085B80092540259F249624AD24A424BB24B01459F
:1085C80045616FF06FC0797106D622D426D24AD0A1
:1085D8004ECE52CC56CA5AC85EC662C466C2630C36
:1085E80005223C312A8985CB404115C45945EFE025
:1085F8000FF30904814917CAFB1F130A2A9C914BE0
:10860800354C175B0200130BAB5B931A456083472D
:10861800390063EFF900B250225492540259F249DA
:10862800624AD24A424BB24B224C924C45618280FC
:108638008307A40063CA571583270A0063860714B3
:10864800834CE4FF93F70C01CDC793870CFF93F796
:10865800F70F6369FC00B3C767219C43DA978287E9
:10866800230F04FE1305E4FFEFF0AFFC630E0510C3
:108678008347E4FF63EFFB1005476398E70A51451A
:108688009780FB1FE780C0BCAA84630F050E930781
:1086980000FD1CA1C147A30005003CA18347E4FFDE
:1086A8001946A2853CB18307A40015055CB583472C
:1086B800F4FFA30FF5FE9780FB1FE78020C97C24F9
:1086C80019469305F400BCB41385C4009780FB1FBA
:1086D800E780C0C765A08547230FF4FEA30A0400FE
:1086E80051B78947230FF4FEB5BF8D47E5BF9147C2
:1086F800D5BF93F78C0099C3AD47EDB713F71C00AE
:1087080093F74C0011C799C39547F9B7A147D9BF4B
:1087180013F72C0011C799C3A5477DBF9947D9B74F
:1087280099C3A947C1B79D4775BF48385105978078
:10873800FB1FE780E0B1AA8421C99307000D1EA1A1
:10874800B5473CA18347E4FF1946A2853CB183079E
:10875800A40015057CA18347F4FFA30FF5FE9780BD
:10876800FB1FE780A0BE5038D0A419C6138544016A
:1087780088C88325640199BF23A8040083270A00B9
:10878800A6858823EFB07FAD850993F9F90F7104A9
:10879800BDBD4838130505029780FB1FE78040AB35
:1087A800AA847DD19307000D1EA1C9473CA1834728
:1087B800E4FF93FC0C061946B3E797013CB18347E5
:1087C800F4FFA2851505A30FF5FE9780FB1FE78030
:1087D800E0B77C2019469305F400BCB47C301385BF
:1087E8003401DCA41C24DCB41C34FCA48307A400DE
:1087F800FCB45E249EA87C24BCA89780FB1FE7805D
:10880800E0B4503890BC09C613850402C8CC95B7AB
:1088180023AE0400A5B797B7FB1F83A7277AE38C7D
:1088280007DEEFF05F9F2254B25092540259F2498A
:10883800624AD24A424BB24B224C924C01454561A6
:108848006FF08F9817B7FB1F0327477705CB1823BF
:10885800AA870D456315F7024111854517C5FB1F0A
:10886800034585C006C6EFB0DFEE13050003EFF041
:108878009F9AB240014541016FF00F9549458280AA
:1088880079714AD017B9FB1F130949738327090067
:1088980006D622D426D2CDEB17C4FB1F1304C4BCC2
:1088A8005820C947298B51CB9165AA849385D571E6
:1088B80011459770FB1FE780E0792320A900CD4779
:1088C8002DCD78309307F00F6314F7009C207CB00F
:1088D8001146A6859780FB1FE78040A793053101C5
:1088E8001305F041EF20323097C7FB1F9387C795D8
:1088F800A023034731013334800011C30904130551
:108908001002EFE0CFC11376F50F0589E14715C5D1
:10891800154532C6EFE0AFC0BC20E8841945230AEC
:10892800F100EFE0CFBF3246AC30E8867C0838086B
:1089380054082285EFB0607BAA87B2502254925423
:1089480002593E8545618280C547C5BF1971A2DCC1
:10895800A6DA86DECAD897C4FB1F9384E4B0DC206D
:108968004944A18BB9CF97B7FB1F83A7276541441B
:10897800A9EB2A89EFE05F8C9C2455446373F504C6
:1089880097B4FB1F938444609C4045449DEB9165DC
:108998009385C57129459770FB1FE780A06B88C038
:1089A8004D4405C12946CA859780FB1FE780009A78
:1089B80013056002EFE0AFB61374F50F058909E9F6
:1089C8006144F65022856654D6544659096182801E
:1089D80013060003814588009780FB1FE780809D70
:1089E8004145EFE0CFB32316A1043D45EFE02FB397
:1089F8002319A1043545EFE08FB2231CA1043945A2
:108A0800EFE0EFB1231FA1042145EFE04FB123129E
:108A1800A1061D45EFE0AFB09C402315A1061364E5
:108A280024009C33F1C72D45EFE06FAF2310A1045C
:108A38003145EFE0CFAE2313A1041305C002EFE0E8
:108A48000FAE2317A1041305B002EFE04FAD231AB0
:108A5800A10413059002EFE08FAC231DA1041305B8
:108A6800A002EFE0CFAB2310A10613058002EFE0D0
:108A78000FAB2313A10613057002EFE04FAA9C4029
:108A88002316A106A83393854700EFD09F8D2AD6D9
:108A98009305F1031305F041EF20F21497B7FB1F7C
:108AA8009387877AAC230347F1033256B335B00076
:108AB80011C389059440FC002287A8223EC8930769
:108AC80021053EC6BC083EC49307E1053EC2DC1042
:108AD8003EC09308A106130861049C009106EFB0FC
:108AE80040612A84E30F05EC0D45EFE0CFDCD1BDF2
:108AF8002545EFE0CFA22310A10429451DBF97C744
:108B0800FB1F83C7A796A18B17B5FB1F1305854AC3
:108B180091E301456FD0AFE197B7FB1F2384074A64
:108B2800FD5717C7FB1FA304F79497B7FB1F23A98B
:108B3800074897B7FB1F23A3074897B7FB1F9387DF
:108B4800A772170700001307478698C31707000086
:108B580013072789D8C3170700001307A79798C7D3
:108B680017070000130767A6D8C717F7FFFF1307F3
:108B7800C7FE98CB97B7FB1F9387C74317F7FFFF2D
:108B88001307470698C317F7FFFF1307C7E7D8C3AC
:108B98008280411122C426C206C617B4FB1F1304E3
:108BA8006442AA8408208545EFF04FDC97C7FB1F75
:108BB80083C7C78BA98BBDC717B5FB1F1305C56A2C
:108BC80004A0EFD02FD697B4FB1F9384643F9C403A
:108BD80099C74D45B2402244924441018280082001
:108BE80019E10145C5BF91659385B5711205977067
:108BF800FB1FE780204688C069DD102081451206EA
:108C08009770FB1FE780007B142090408147FD553B
:108C180013F7F70FE377D7FC1397470032970CA3A6
:108C28008507FDB7014597B7FB1F238D0738EFD0A0
:108C38006FCF45BF17B5FB1F0325453511CD411132
:108C480006C69770FB1FE780004EB24097B7FB1F20
:108C580023AE07324101828082800111130570031F
:108C680006CEEFE0CF8B2AC613058003EFE02F8BEB
:108C78002AC413059003EFE08F8A2246B245F240DA
:108C8800AA86054505616FB080455D711305D0035F
:108C980086C6A2C4A6C2CAC0EFE06F882A8413059C
:108CA800C003EFE0CF87AA841305E003EFE02F8726
:108CB8002A891305F003EFE08F868A871377F50F6B
:108CC8009376F90F13F6F40F9375F40F0545EFB08B
:108CD8004043B640264496440649616182800111AA
:108CE80022CC06CE26CA0D472E846317E504B83178
:108CF800E947CA2197B4FB1F938404556315F7000D
:108D0800FE206387A70497A0FB1FE78040E6722038
:108D180011C172A53A2416244E202830EFD09FB8EE
:108D28005A20FE206314F700FD57FEA00545F240C7
:108D38006244D2440561828009674D07AA87631C93
:108D4800E500BC2131476385E7004547E390E7FE2E
:108D5800EFD00FC5E1BF31476319E50017B5FB1F19
:108D68000345D570EFD05FBFD1B713076002631911
:108D7800E50017B5FB1F0345756FEFD0BFC27DB780
:108D880041677D170145E394E7FAD831C947E310F5
:108D9800F7FACC212A20300023140100EF60103D9F
:108DA80071B71971A2DC17B4FB1F1304241E1C40F1
:108DB80086DEA6DACAD8CED6D2D4D6D2DAD005453F
:108DC800638A070C9305F1051305F041EF20A261B2
:108DD8009305F1051305F041EF20E26097B7FB1FFB
:108DE80093878746BC230347F105B337F00011C3C7
:108DF80089071840BEC6283393054700EFD06FD6C1
:108E08001840AAC40D452C23AEC2EFD05FF1AAC00A
:108E18001145EFD0DFF0832A04002ADE654503C739
:108E2800AA0003CBBA003ADCEFD07FEF2A84694569
:108E3800EFD0FFEEAA847145EFD07FEE2A896D4509
:108E4800EFD0FFEDAA897545EFD07FED2A8A7945E5
:108E5800EFD0FFEC2648B6476257F25606469645CD
:108E68001375F50F137AFA0F93F9F90F1379F90FB0
:108E780093F4F40F2ACC1314446002D002CE52CAE1
:108E88004EC84AC626C422C25AC093884A0005451D
:108E9800EFB0C01FF6506654D6544659B659265AF4
:108EA800965A065B09618280411122C44AC006C6EF
:108EB80026C217B9FB1F1309791283470900130744
:108EC800E00F2E846382E7041307F00F6385E7023F
:108ED80011459770FB1FE780A037AA8509CD930736
:108EE80000FD1CA189473CA1854700B13CB1034561
:108EF8000900EFB08FB6F9572300F900B2402244B9
:108F08009244024941018280AA8411459770FB1F4F
:108F1800E7800034AA857DD1930700FD1CA189470D
:108F280000B13CA124B12244B2409244024917B591
:108F3800FB1F0345A50A41016FB02FB279714AD0D2
:108F480017B9FB1F130989048327090022D406D601
:108F580026D24ECE52CC4544C5EB97B4FB1F938422
:108F6800A450DC204944958BC5C32E8A916597B7D8
:108F7800FB1F2385A706AA899385757131459770CC
:108F8800FB1FE780200D2320A9004D4435CD230089
:108F98003501A30005002946D28509059770FB1FF6
:108FA800E780C03A0327090091463C2363E7F606A9
:108FB800CD4691CF0546F546638BC7000946C9469D
:108FC8006387C7000D46C1466383C700D54634A3EF
:108FD800930571001305F041EF20E2409C83C5E33F
:108FE80017B7FB1F034767268D47631AF708EFD0AB
:108FF8000FC52C00EF70500F2800EFD07FAC45450F
:10900800EFD0FFD125E50144B25022852254925475
:109018000259F249624A45618280ED1793F7F70FCA
:1090280095460544E3E2F6FE975602009386C6BCD1
:10903800B3C7D7209C43B697828789473CA319A01A
:10904800230107006545EFD09FCD9307F007E301A3
:10905800F5F8032709003C2393E707043CA38DBFD9
:109068008547E9BF9947D9BF9147C9BF130600642F
:109078003306C50288209145EFB04FC469B7153350
:109088002A8451D1EFF01FBB41B7011126CA97B40A
:10909800FB1F9384A4EF9C4022CC06CE4AC84944C7
:1090A800A1C79C230D446391A70417B9FB1F13099B
:1090B800A93B034509008945EFB0AFE9034509001D
:1090C800914597B7FB1F239907F0EFB08FE89C40B5
:1090D8000147814680B31306F10085478545014560
:1090E800DC87EFA0907F2A84F24022856244D24434
:1090F800424905618280011106CE22CC26CA4AC89F
:109108004EC68547631EF50617B4FB1F1304C4EC4F
:109118001E20B1CB17B7FB1F0347471329E71307D7
:10912800B003636EF70297B4FB1F9384E43388207F
:109138008945EFB00FE212209307006488203306B8
:10914800F6028945EFB08FB797B7FB1F239607E85C
:10915800F2406244D2444249B24905618280938711
:1091680047FC1EA0F5B797B7FB1F83A727E2EDD3EF
:109178006244F240D2444249B2498823056131B77A
:1091880097B9FB1F938989E083A70900F1D317B921
:10919800FB1F1309692D83474900918BD5DB89474C
:1091A8006311F5062D45AE849770FB1FE780400AD2
:1091B8002A8459DD930700FD1CA1E547A30005009B
:1091C8003CA1BC3015051946230FF5FEDC2093851C
:1091D8005400A30FF5FE9770FB1FE7802017034587
:1091E80059009307F00F6315F50083A7090088233A
:1091F800A2856244F240D2444249B24905616FB047
:10920800CF85034509008945EFB0AFD46244F240E9
:10921800D2444249B24997B7FB1F239F07DA056139
:109228006FF05FA197B7FB1F83C74724958B89CF42
:1092380097B7FB1F83A787D991CB854717B7FB1F24
:10924800A30DF7D86FF07FA1494582804145828000
:1092580097B7FB1FA38307D8854501456FA0B06862
:1092680097B7FB1F83C78720958B81CB854717B797
:10927800FB1F2304F7D66FF05FA14945828097B79B
:10928800FB1F238C07D4814505456FA0D06797B78E
:10929800FB1F83C7A71D958B638B0712011122CC77
:1092A80006CE26CA4AC84EC69307C01C328463FA43
:1092B800C7000945F2406244D2444249B2490561B7
:1092C800828097B7FB1F83A767CC6384071097B783
:1092D800FB1F9387B7D0B68994231307E00F639ACF
:1092E800E60E88A31305860033450508ADC99165C8
:1092F800938565719770FB1FE780C0D5AA8455D9FF
:1093080017B9FB1F130909CD0325090009C5977073
:10931800FB1FE78040E11385840088C022868145D1
:10932800232099009770FB1FE780C0088327090056
:109338002286CE8588439770FB1FE780200183270C
:109348000900A286F240C2A36244D2444249B2490B
:10935800984305468D45054505616FA09057916571
:10936800938555719770FB1FE780C0CEAA8431D1D1
:1093780017B9FB1F1309C9C50325090009C597704B
:10938800FB1FE78040DA1385840088C02286814568
:10939800232099009770FB1FE780C00183270900ED
:1093A8002286CE8588439770FB1FE78020FA8327A3
:1093B8000900A286F240C2A36244D2444249B2499B
:1093C800984305468D45054505616FA0D050494530
:1093D80082804945C5B59307C01C63FCA7000945B1
:1093E80082800945F2406244D2444249B24905614B
:1093F8008280011122CC06CE26CA4AC84EC62A84CB
:1094080025C1AE89916521059385657133450508A8
:109418009770FB1FE78000C4AA8461D517B9FB1FAA
:10942800130949BB0325090009C59770FB1FE7808D
:1094380080CF1385840088C0228681452320990027
:109448009770FB1FE78000F7832709002286CE85E7
:1094580088439770FB1FE78060EF83270900C2A34A
:1094680097B7FB1F83A787B285CF97B7FB1F83C723
:10947800E7FF958B85CB97B7FB1F83A7A7B591CF40
:109488009843D6236244F240D2444249B249054641
:109498008D45054505616FA0D04301478146DDB77D
:1094A800014589B749453DBF9307C01C63FCA70028
:1094B800094582800945F2406244D2444249B24992
:1094C80005618280011122CC06CE26CA4AC84EC642
:1094D8002A8425C1AE899165210593855571334547
:1094E80005089770FB1FE780E0B6AA8461D517B915
:1094F800FB1F1309E9AD0325090009C59770FB1F78
:10950800E78060C21385840088C0228681452320B5
:1095180099009770FB1FE780E0E9832709002286FE
:10952800CE8588439770FB1FE78040E283270900B8
:10953800C2A397B7FB1F83A767A585CF97B7FB1F64
:1095480083C7C7F2958B85CB97B7FB1F83A747A81F
:1095580091CF9843D6236244F240D2444249B2495B
:1095680005468D45054505616FA0F03601478146E2
:10957800DDB7014589B749453DBF9307C01C63F472
:10958800A70009458280797122D406D626D24AD00E
:109598004ECE2A842DC1AE899165210593857571BA
:1095A800334505089770FB1FE780C0AAAA840945C0
:1095B800A9C817B9FB1F130969A10325090009C523
:1095C8009770FB1FE78020B61385840088C0228629
:1095D8008145232099009770FB1FE780A0DD832732
:1095E80009002286CE8588439770FB1FE78000D646
:1095F80083270900C2A397B7FB1F83A7279989EB85
:109608000145B250225492540259F2494561828070
:1096180097B7FB1F83C787E5958B4945FDD36C003A
:109628001305D030EF30B210B24793F7070FE9DBDC
:1096380097B7FB1F83A787999443D2238D45054588
:10964800EFA0302A7DBF97B7FB1F83A7A79889CFC4
:10965800D2238C43411106C69770FB1FE78000CFC9
:10966800B2400145410182800945828097B7FB1FBE
:1096780083A7479685C717B7FB1F032767958947B1
:1096880019CF52230C43411106C69770FB1FE78080
:10969800E0CBB24081473E854101828089473E85C3
:1096A800828097B7FB1F83A7E79285C717B7FB1F71
:1096B8000327C791894719CF52230C43411106C686
:1096C8009770FB1FE78080C8B24081473E85410103
:1096D800828089473E858280797126D206D622D437
:1096E8004AD04ECE97B4FB1F938404B68D4783C9E6
:1096F800240063FAA7000945B25022549254025933
:10970800F2494561828098202A844145E316F7FE94
:109718009307F4FF93F7F70F854663E8F60A2E8957
:10972800B1ED99452800EFC07FA2A0A0914517B5DB
:10973800FB1F034565D3EFB0CF812800EFD04FB8AA
:1097480055E9930571001305F041EF10D2499C8348
:10975800D1EB8D476318F4084545EFD04FDC59C16C
:1097680037761800130606A03306C502914517B5CB
:10977800FB1F034565CFEFA0DFF5ADA01946814576
:1097880028009770FB1FE780E0C219462C004A8525
:109798009770FB1FE78000CD39FD19469305F00F40
:1097A80028009770FB1FE780E0C019462C004A8507
:1097B8009770FB1FE78000CB1DFD1946CA8528005E
:1097C8009770FB1FE78080B88DB7630FE400914561
:1097D80017B5FB1F034545C997B7FB1F238707A686
:1097E800EFA03FF7014509BFC8442C00EF70C00F38
:1097F800A0A00DDD2381340101B797B7FB1F83C7F4
:10980800E7C6918B8DC3411117A5FB1F1305C57BB7
:1098180006C6EFC01F93B240FD5717B7FB1F2318AA
:10982800F7A24101828001456FC0BF91FD5717A77C
:10983800FB1F2305F77AF95717A7FB1FA300F77A31
:1098480097A7FB1FA38B077897A7FB1F238707788A
:1098580097A7FB1F2392077897A7FB1F23AC0776D0
:1098680097A7FB1F23A6077697A7FB1F23A00776BA
:1098780097B7FB1F938787A0170700001307E720F8
:1098880098C31707000013074787D8C317F7FFFFC8
:109898001307675198C717F7FFFF1307473CD8C747
:1098A80017F7FFFF1307A73E98CB97F7FFFF93879C
:1098B800474317A7FB1F2329F7708280411126C24F
:1098C80097A4FB1F9384846C9C4006C622C495CB46
:1098D8002A840D459770FB1FE7808097AA8519C9D0
:1098E800930700FD1CA18D4700B13CA19C40882333
:1098F800EFA0BF9619C42244B240924441016FF0D0
:109908006FB3B240224492444101828079714AD0B7
:1099180017A9FB1F130989678327090006D622D4D4
:1099280026D24ECE6383070E98338547AA8497B90B
:10993800FB1F938969916301F70483C749008DE789
:109948000D459770FB1FE780A090AA8501CD93076E
:1099580000FD1CA1914704B13CA18327090088237D
:10996800EFA0BF8FEFF00FAD0545B25022549254CF
:109978000259F2494561828097A7FB1F83A7876533
:1099880089CB9443D2239305E1000545EFC03F8678
:1099980011ED0145EFD0AFB82A8621C6894517B524
:1099A800FB1F034565ACEFA07FB125A81C21858B63
:1099B800EDD30545EFD0AFB69307B0032A8463F122
:1099C800A7045D6613060670894517B5FB1F034596
:1099D800A5A9130444FCEFA0DFCF97A7FB1F239D85
:1099E800875E83270900094798B383C7490091C751
:1099F80097B7FB1F238C078485BF2685C135ADB774
:109A0800930700643306F50249BF0145B9BF411108
:109A180022C42A840D4506C69770FB1FE780408341
:109A28000DC1930700FD1CA1CD4700B13CA1224404
:109A3800B240AA8517A5FB1F0345455A41016FA0EF
:109A4800DF81B240224441018280411122C42A842C
:109A58000D4506C69760FB1FE780807F0DC1930701
:109A680000FD1CA1ED4700B13CA12244B240AA85EB
:109A780017A5FB1F0345855641016FA00FFEB24095
:109A88002244410182805A210111896606CE22CCE6
:109A980026CA13866600AA876316C7009C47014535
:109AA8008C2371A8138606046365E604138656039F
:109AB800636FE60013869600630BC7081386A6003B
:109AC800630DC712A1066309D7060145A5A8F97653
:109AD8009386A6FC3697A94633470708E3E7E6FED0
:109AE800974602009386C6123347D7201843369705
:109AF8000287138616056307C71893862605E3169B
:109B0800D7FC1C45802397A7FB1F83C7074D2285D9
:109B1800639D07160D459760FB1FE7806073AA8554
:109B28000DC1930700FD1CA1F14700B13CA117A589
:109B3800FB1F0345A54A91A29C4705458C23EFF0DE
:109B4800AFB60545F2406244D2440561828017A74A
:109B5800FB1F0327A743014575D79C47882359E96D
:109B680085471CB30545EFA0404DE1BF1C4597A4B0
:109B7800FB1F9384B4461307E00F80239C20638B5C
:109B8800E7021307F00F6384E70211459760FB1F94
:109B9800E780006CAA8501CD930700FD1CA18947C9
:109BA80000B13CA1A30105008820EFA00FEBF957F5
:109BB8009CA041BF97A4FB1F9384443D9C40014552
:109BC800D1D305E805447D454085EFD04F9568869B
:109BD80013050002EFD0AF949C40C8851307B1006D
:109BE80080B374001306A10085450545EFA0E04E3B
:109BF80089BF2285EFF09FCCA9B79C476244F24009
:109C0800D244882305616FF07FD01C4509458C2319
:109C18003DB71C4588232DE56C001305D030EF3087
:109C28000231B247414793F7070FE38CE7F09305FA
:109C3800B10013056031EF30822F88858545EFA08C
:109C4800804A01B71C45802397A7FB1F83C7F738B5
:109C580022859DE70D459760FB1FE780605FAA8519
:109C6800E30105EE930700FD1CA1D14700B13CA11B
:109C780097A7FB1F83A787318823EFA00FDED1B5F5
:109C88007933C1B51C45882319C1C1335DBD8545EC
:109C98000545EFA0404775B5411122C417A4FB1F25
:109CA8000344C47C06C6158809CC17A5FB1F1305F9
:109CB800E55CEFC06FC84D44B240228522444101A3
:109CC80082800145EFC04FC7C5BF98219376250014
:109CD8009377D70F99C29367270093F6F70713175F
:109CE80045606354070093E607081378850093F7E7
:109CF800760F6304080093E786009376050299CEF1
:109D080093E707029CA1635707001C2293E7C7004B
:109D18001CA282801375A5026DF9828093F7F7FD66
:109D28009CA1E34407FE9377A502E5F37DF11C228D
:109D3800CD9BF9BF2D45631C0710011126CA4AC8DF
:109D48004EC606CE22CC9821BE8989472E89B68474
:109D5800631EF704DC413284983394232207558F1D
:109D68008D66938746A01316576063C9C70293860A
:109D7800F69F63DDC602F5779387F75F3E978D47B9
:109D8800C8453347070863E7E7029746020093860A
:109D9800E6EA3347D7201C43B6978287938766AA9B
:109DA800630EF608938686B8630FD60823900400DE
:109DB800054525A09760FB1FE780E062334605084C
:109DC8003356360B92A08325C9001DA01E210947D2
:109DD8009AA01CA0A1831CB00145F2406244D24461
:109DE8004249B2490561828099479EA01946AA85D1
:109DF80022859760FB1FE7806055F9BF85479EA0C5
:109E08001C211CA0D1BF05C9A1479EA01E211CA0D2
:109E18001E21A1831CB03E213CA03E21A1833CB061
:109E28005E215CA05E21A1835CB07E217CA07E21A6
:109E3800A1837CB055B72390040079BF85479EA0C5
:109E4800DC459C237DBFE1479EA06146ADBF828073
:109E5800797122D44AD006D626D24ECE52CC56CAD2
:109E68003A89982189472E84631DF7025C40B6849D
:109E7800B28503C8170094238D6722083368D80079
:109E8800938627A013185860630BD8102A8A63CCCE
:109E98000601938607A0630BD802938717A0630077
:109EA800F80A854711A8138737A0630FE80A1387B4
:109EB80067AA8D47E317E8FEB2502254925402591C
:109EC800F249624AD24A3E8545618280484432C698
:109ED8009760FB1FE78020519D4733450508E36DD8
:109EE80025FD97AAFB1F938AAA1083C70A00B30906
:109EF8009900B24563D43701B5477DBF48442686EB
:109F0800B3C909084A959760FB1FE780204403C638
:109F18000A00484481450506330636414E95976048
:109F2800FB1FE780204997A7FB1F83A7A70C99E38E
:109F3800814759B79C438145E5DF528525A0AD4748
:109F4800E31C09F6E39AE4FA1C321822A207D98F17
:109F580058441EA397A7FB1F83A7C709F1DB9C439F
:109F68008545F9D78297E9B717A7FB1F0347F70776
:109F78008D4739D3AD47E31109F49947E39EF4F6C9
:109F8800484419469760FB1FE780403C97A7FB1F92
:109F980083A74706D1DF9C43C1DF8D4579BF17A74B
:109FA800FB1F034707F4218B8D4719D7AD47E315EE
:109FB80009F08547E392F4F4182293070008E3EDCB
:109FC800E4EE5C4498A3ADB7411122C4094497A7B5
:109FD800FB1FA38987F097A7FB1FA38487F097A788
:109FE800FB1F238087F097A7FB1F23A5070097A7D0
:109FF800FB1F238607FE97A7FB1F238B07FE97A748
:10A00800FB1F239607FE97A7FB1FA38007FEA14708
:10A018001946814517A5FB1F1305C5FC06C617A7DA
:10A02800FB1FA30FF7EA9760FB1FE780A03897A7ED
:10A03800FB1F238787EAB707A00017A7FB1F130793
:10A04800A7E9938707051CC3B707E8035CC397A76D
:10A05800FB1F238187E885476146814517A5FB1FBC
:10A068001305053617A7FB1FA305F7E697A7FB1FE0
:10A07800238187E697A7FB1FA38C87E497A7FB1F7D
:10A08800238007F69760FB1FE780C0321306001392
:10A09800814517A5FB1F1305A51F97A7FB1F23893C
:10A0A80087E297A7FB1FA38C07F29760FB1FE78047
:10A0B800603097A7FB1F9387E7DBB240224417075E
:10A0C8000000130767C798C317070000130787D84E
:10A0D800D8C323A4070041018280797122D426D2F3
:10A0E80006D64AD04ECE52CCA1472E84B28463EB1A
:10A0F800A70017470200130767B53345E5201C4141
:10A10800BA978287930710086304F51C63ECA700CD
:10A1180093072004630EF516930700086303F518E8
:10A12800094591A093072008E31CF5FE8547639B2A
:10A13800F50208229377250095E797A7FB1F83C7A9
:10A14800C7EA1387F7FF97A5FB1F938565141207C6
:10A1580092072E97A1075047BE9585AA9307800FAF
:10A1680063FBB7006145B250225492540259F24938
:10A17800624A4561828017AAFB1F130AAAD6834741
:10A188000A0017A9FB1F1309A9109207CA97C84705
:10A1980009C99760FB1FE78000F997A7FB1F238970
:10A1A80007E4130614001376F60F9165938505717D
:10A1B800328583490A0032C69760FB1FE78080E931
:10A1C80083470A009209CA99920723A6A900CA9749
:10A1D800C84749D9324681459760FB1FE780801DF3
:10A1E80083470A002286A68592073E990325C9005F
:10A1F8009760FB1FE780801597A7FB1F238A87DEE0
:10A20800014595B78947E39FF5F41E2217A7FB1F61
:10A21800231FF7DCF5B78547E396F5F41C2217A74B
:10A22800FB1FA304F7DCE9BF9947E39DF5F2194644
:10A23800A68517A5FB1F1305E5DA9760FB1FE780C6
:10A24800E0107DBFA147E39FF5F02146A68517A53D
:10A25800FB1F130565C8D5B78547E395F5F01C22A4
:10A2680017A7FB1FA307F7C661BFE147E39CF5EEFD
:10A278006146A68517A5FB1F130585147DBF854775
:10A28800E392F5EE1C2217A7FB1FA30AF7D48DBF94
:10A298008547E399F5EC1C2217A7FB1F2303F7C496
:10A2A80085B78547E390F5EC97A7FB1F83C787C35E
:10A2B8001387F7FF97A5FB1F938585FD12072E9738
:10A2C800920750478820A107BE95EFF01FA00DBF49
:10A2D8008547E399F5E897A7FB1F83C727D1C9BF2F
:10A2E800AA8721472E85636DF700174702001307D9
:10A2F8002798B3C7E7209C43411106C6BA978287BF
:10A3080013072004638BE70889473E85828017A7D7
:10A31800FB1F034727BD120797A7FB1F938747F724
:10A32800BA97CC47894785C117A6FB1F034646CC79
:10A338009760FB1FE780800131A097A7FB1F83D799
:10A3480007CB9EA18147B2403E854101828097A7F5
:10A35800FB1F83C797C91CA1F5B7194697A5FB1F13
:10A36800938545C8F1B7214697A5FB1F9385C5B6C8
:10A37800EF901FDBC1BF97A7FB1F83C797B5E1BF4E
:10A38800614697A5FB1F9385A5035DB797A7FB1F9C
:10A3980083C7F7C4C9B789477DB797A7FB1F83C78A
:10A3A80047B49CA1814795B7630F053897A7FB1F52
:10A3B8009387E7C2982363180738054798A397A798
:10A3C800FB1F9387E7EC894698A717A7FB1F23165F
:10A3D80007EC17A7FB1F1307E7B294A397A6FB1F69
:10A3E800938606B6D8C7D4C37D57630CE534137774
:10A3F8001500854529C717A6FB1F231806EA094734
:10A4080097A6FB1F938606B317A6FB1F130696ADE8
:10A4180098ABD4CBD0CF854617A6FB1F2304E6AC58
:10A428002380E70217A7FB1F130747B0D8D394AFC1
:10A438002384D70217A7FB1F231107E88D4513773D
:10A44800250025C3139745003E9797A6FB1F9386C3
:10A4580066AE094654C317A8FB1F130898A885467B
:10A4680010A314A723260701231507001387150037
:10A478003347070817A8FB1F230AE8B612073E97B9
:10A4880010A314A717A6FB1F130606AA97A6FB1F5F
:10A498009386E6B5890550C32315070054C7B3C58D
:10A4A80005081377450025C3139745003E9797A6DF
:10A4B800FB1F938626A8094654C317A8FB1F130839
:10A4C80048A2854610A314A72326070123150700D1
:10A4D800138715003347070817A8FB1F2307E8B0A1
:10A4E80012073E9710A314A717A6FB1F130686A3EF
:10A4F80097A6FB1F938676AF890550C323150700DF
:10A5080054C7B3C505081377850021CF13974500B5
:10A518003E9717A6FB1F1306E6A150C305468946BA
:10A5280010A717A6FB1F1306B69B14A32315070035
:10A5380050C7138715003347070812073E9714A31F
:10A5480097A6FB1F9386C69D54C3A14614A797A63A
:10A55800FB1F938626A989052315070054C7B3C591
:10A5680005081377050121CF139745003E9797A655
:10A57800FB1F9386269C094654C317A8FB1F130884
:10A588002896854610A314A723150700232607013C
:10A59800138715003347070812073E9710A314A71F
:10A5A80017A6FB1F1306869797A6FB1F9386C692CE
:10A5B800890550C32315070054C7B3C50508137789
:10A5C800050221CF139745003E9797A6FB1F938658
:10A5D8006696094654C317A8FB1F1308A88F85461B
:10A5E80010A314A7231507002326070113871500B6
:10A5F8003347070812073E9710A314A717A6FB1F97
:10A608001306469197A6FB1F9386B68C890550C3FF
:10A618002315070054C7B3C505081377050421CFD0
:10A62800139745003E9797A6FB1F9386A690094669
:10A6380054C317A8FB1F1308C889854610A314A77D
:10A64800231507002326070113871500334707083A
:10A6580012073E9710A314A717A6FB1F1306C68B55
:10A6680097A6FB1F9386C697890550C32315070035
:10A6780054C7B3C505081377050821CF13974500BC
:10A688003E9717A6FB1F1306E68A50C35146894614
:10A6980010A717A6FB1F1306B68314A323150700DC
:10A6A80050C7138715003347070812073E9714A3AE
:10A6B80097A6FB1F9386C68554C3854614A797A6FD
:10A6C800FB1F9386E6CF89052315070054C7B3C53A
:10A6D80005081375051039C9139745003E9797A6C5
:10A6E800FB1F9386268554C3094685461795FB1F8D
:10A6F8001305057E10A314A72315070048C7138761
:10A708001500334707081207BA9717A7FB1F130747
:10A718002780D8C317A7FB1F1307778C890590A339
:10A7280094A723950700D8C7B3C505089796FB1FBC
:10A7380093864674414617A5FB1F130565B56F3010
:10A74800E0414D454DB9014582800111FD1522CCEE
:10A7580006CE328426CA3E864AC813F8F50FAD479E
:10A7680063E8070B3A89173702001307A7523348E3
:10A77800E82083270800B684BA9782878545EFB01A
:10A788001FB901E5EFF04FD10145F2406244D244D0
:10A798004249056182808945EFB07FB77DF5228502
:10A7A800EFE02FBFD5B7914532C6EFB05FB632465E
:10A7B80069FDCA852685EFB03FACEFF0EFCDEFF02D
:10A7C800CF83EF60A07AC9B7A14532C6EFB03FB4D6
:10A7D800324645FDCA852685EFB01FAA2285EFE0DF
:10A7E8004FBBEFE0CFB1EF60407679BFB14532C6DD
:10A7F800EFB0FFB1324651F9CA852685EFB0DFA721
:10A808002285EFE00FB9EFE08FAFEF60007475B706
:10A818000945A5BF79714ECEAE896C0022D426D2E7
:10A828004AD006D62A89B284EF00306E2A840DE118
:10A83800CE854A85EFB0CF8C2A8419E93245268720
:10A8480097B6FFFF9386460B2D468145EF1000060D
:10A85800B2502285225492540259F24945618280AD
:10A86800397126DAAE844C0022DC4AD84ED652D44E
:10A8780006DEAA893289368AEF0030692A8421E9FE
:10A88800A685630D09009E202C007C84BE207C8553
:10A89800930720307C86930780025C874E85EFB053
:10A8A8004F832A840DE55946A6851305A100230484
:10A8B80021019760FB1FE78060A91245528797B670
:10A8C800FFFF938686FE25462C00EF00307EF2506F
:10A8D80022856254D2544259B259225A2161828047
:10A8E800797126D2AE846C0022D44AD04ECE06D6D8
:10A8F800AA893289EF0070612A840DE1A6854E8508
:10A90800EFB0CF812A8419E932454A8797B6FFFF0D
:10A91800938646003546A685EF005079B2502285C9
:10A92800225492540259F249456182807547AA8798
:10A938006365B702114701456378B702ED1593F5D2
:10A94800F50F61476361B702973602009386863731
:10A95800B3C5D52098413697028793F5F5071307B5
:10A968002005638AE50001458280C84782808843C4
:10A97800828088478280C84382809307F00F630FE4
:10A98800F506011126CAAA841305000222CC4AC87A
:10A998004EC652C456C206CE2E8AB28AB6893A89A3
:10A9A8009760FB1FE780C08A2A844D450DC893072E
:10A9B80000FB1CA0A300540123114401230234010D
:10A9C80013058400614663050902CA859760FB1F69
:10A9D800E780C097A2852685EF903F880145F24021
:10A9E8006244D2444249B249224A924A056182806D
:10A9F80081459760FB1FE780E09BE9BF094582809E
:10AA0800011122CC06CE2A844C86D0869780FB1F63
:10AA1800E780E01505C15425214797A7FB1F9387B9
:10AA2800A7A4639DE600E82378009306E0070146A3
:10AA3800A285A137F240624405618280C83378005C
:10AA48009306E0070146A285EDB793070064330635
:10AA5800F6026F90FFBB15C1411122C406C62A84B5
:10AA680008219307D00F63E6A700EF903FD8FD5762
:10AA78001CA0B2402244410182808280797122D494
:10AA880006D626D24AD04ECE9E2509448DEBAE84FA
:10AA98006C00AA893289EF0050472A840DE1A68507
:10AAA8004E85EFA07FF32A8419E932454A8797B685
:10AAB800FFFF938626F24D468145EF00305FB25086
:10AAC8002285225492540259F249456182801A2102
:10AAD8009307000B6310F7025C214947639AE7006C
:10AAE800183985476398E7002A2185456F30902AF1
:10AAF8006D47CDBF828001116C846C0022CC26CAC0
:10AB08004AC806CE2A89B6847085EF0010402A8488
:10AB18000DE12C004A85EFA09FD22A8419E932451D
:10AB2800268797B6FFFF938646CD15462C00EF0083
:10AB3800F057F24022856244D2444249056182803E
:10AB48007971930720306C8470857C862C0093077C
:10AB58008002014606D65C87EFF09FD0B25045616F
:10AB68008280C177797185073EC4894726D27C8661
:10AB7800AE84930780024C0022D44AD006D62A8994
:10AB88005C87EF0090382A840DE12C004A85EFA0FD
:10AB98001FE22A8419E91245268797B6FFFF938694
:10ABA80046DE45462C00EF007050B25022852254F4
:10ABB8009254025945618280B28605466FF05FCA99
:10ABC800797126D2AE846C0022D44AD04ECE06D6F5
:10ABD800AA893289EF0070332A840DE1A6854E8553
:10ABE800EFA09FBD2A8419E932454A8797B6FFFF2F
:10ABF800938646BB0D46A685EF00504BB250228582
:10AC0800225492540259F24945618280797193071E
:10AC180020206C8470857C862C0093078002014676
:10AC280006D65C87EFF0DFC3B25045618280011120
:10AC380022CC26CA4AC806CE2A84AE84328936C6B1
:10AC48009780FB1FE780A0F215C95025A14632471F
:10AC580097A7FB1F93874781631DD600E823CA8601
:10AC68002686A2856244F240D244424905616FF0CB
:10AC7800DFD0C833CA862686A285EDB7F240624483
:10AC8800D24442490545056182806FF0BFB86FF034
:10AC98007FB86FF0FFC46FF0BFC479714ECEAE8934
:10ACA8006C0022D426D24AD006D62A89B284EF0074
:10ACB800D0252A840DE1CE854A85EFA0FFC72A84D6
:10ACC80019E93245268797B6FFFF938666C63D4643
:10ACD8008145EF00B03DB25022852254925402596A
:10ACE800F24945618280B28601466FF07FB7011153
:10ACF80022CC2E846C0026CA06CEAA84EF00F0204F
:10AD0800DD476309F500930710101EA4A285268568
:10AD1800EFA09FCCF2406244D24405618280239424
:10AD280005006FF0BFD5E5BF1797FB1F0347073135
:10AD3800854763F8E702011122CC2E846C0026CAED
:10AD480006CEAA84EF00701C01E9930700101EA428
:10AD5800A2852685EFA05FC8F2406244D24405610F
:10AD68008280594582809797FB1F23A9A728828054
:10AD78009797FB1F23A2A7288280011122CC26CAFD
:10AD880006CE2A84AE849780FB1FE78040DEA68526
:10AD98002285EFA06FF605E9228564869780FB1F60
:10ADA800E780E0DC0DC1542521479797FB1F938767
:10ADB800A76B639FE600E82378009306F007014637
:10ADC800A285EFF09FBBF2406244D24405618280C5
:10ADD800C833DDB7797122D44AD0AE8706D6BA8592
:10ADE80026D24ECE7547328436896364F7042147EC
:10ADF800636CF70015476388E7021947638DE70816
:10AE0800C167FD1785441DA037061400DD1713061A
:10AE18000620B317F0287D8E49EE19677D8F25EB44
:10AE280093F71710F1DFC167FD1789446316F40221
:10AE380021A813F7F70793062005E313D7FC41670A
:10AE48007D17631EE6048D442EC6EFA0AFEEB24513
:10AE5800330495403344040833858400334505089A
:10AE6800EF30D000AA87B3C9040821C963040900D8
:10AE7800231089002254B25092540259B30530412C
:10AE8800F2493E8545611753FB1F67004337C16789
:10AE9800FD17954461BFC167FD179D4441BF130766
:10AEA800200D8D44E39AE7FA1304C60033440408DE
:10AEB80065B7C167FD178D4495BFB25022549254AF
:10AEC8000259F24945618280011122CC26CA06CE78
:10AED800D0212E841307000281469945AA84DD3DBE
:10AEE8002AC621C51E205020930554007C803E2090
:10AEF8007C8189477C82930780025C839750FB1F83
:10AF0800E780C0445C208A8526857C84EFA0DF9595
:10AF18002A8411C532459750FB1FE780C020F240B4
:10AF280022856244D244056182804D44CDBF397187
:10AF380022DC26DA4AD806DE89472A84AE84368996
:10AF48006306F600C14709456315F60432C6A9C071
:10AF58004C082285EF00607B324605EDC1778507F6
:10AF6800A6851305D1013ECC230EC1009750FB1FC7
:10AF7800E780C03D2C082285813F01ED52454A8774
:10AF880097B6FFFF9386E68C1D462C08EF0010123B
:10AF98000145F2506254D25442592161828039717C
:10AFA80026DA4AD84ED63289AE893686BA848146A0
:10AFB80013071002D94522DC06DE2A8432C6EFF0D8
:10AFC8007FE12ACE1DCD3246A685231A3101F084B1
:10AFD800231B21019750FB1FE780403722854C082F
:10AFE800EFA03FA92A8411C572459750FB1FE7803F
:10AFF8008013F25022856254D2544259B2592161C9
:10B0080082804D44FDB7011122CC06CE26CADD4709
:10B018002A84639FF5085439B1441C49B3869602C3
:10B028003287B697904314436306D6020A20230654
:10B0380001006C00EFA09FA70824B165938505B8AF
:10B04800EF90EFB9E5473CA097B7FFFF9387C7A5F7
:10B058005CC091A85623D223E31AD6FC88470C4734
:10B068009750FB1FE7800040AA870A2089E723063C
:10B0780001006C00C1B75C385828850793F7F70FB3
:10B088005CB863F4E702B38797021848BA97984701
:10B09800D623B2238E23213751F90824B16593852D
:10B0A80005B8EF90CFB3D94431A87C285C86D1B7D6
:10B0B8000A21AE846C0023060100EFA03F9F85475C
:10B0C800E39CF4F6F24062442685D244056182800E
:10B0D800011122CC06CE26CADD472A840A216398AC
:10B0E800F508EFA02FC5522C3E284E286D162A963B
:10B0F800334606083307F64052ACAA86334707089A
:10B108000A206372B7061388C6FFB388E54063D484
:10B118000803AE97918FB3C607081C4C0E283E97BC
:10B12800EFF0FFE709ED0824B165938505B8EF90C6
:10B138000FABD944B1A0ED16B3C60608F9BF0A2073
:10B14800230601006C00EFA07F960824B165938563
:10B1580005B8EF90CFA8E5473CA097B7FFFF9387C6
:10B16800A7945CC0F9B785475C866C00E9BFAE84DC
:10B178006C0023060100EFA07F938547E397F4FC5A
:10B18800F24062442685D24405618280397126DA0C
:10B19800AE842C0022DC4AD84ED606DE2A89B28933
:10B1A800AD232A8431E54A85EFA0CFB8D6206D15A6
:10B1B80063C4A600B34605089844B2208E204A8589
:10B1C800EFF0FFDD2A840DE53146A6850808230641
:10B1D80001009750FB1FE7806017BE2022454E876D
:10B1E80097B6FFFF9386E6855D466C00FC867D2D4D
:10B1F800F25022856254D2544259B2592161828058
:10B2080071B769B7797122D406D626D24AD04ECE04
:10B2180052CC56CA5AC80944C1CD3289094449CAD0
:10B22800AE84BA8A2A8A368BEFA0CFB0138744003F
:10B2380081477115162363DEA608850793F7F70F74
:10B248003107E319F9FE8A855285C1212A842DE147
:10B2580031453305A9029165938515704D44975082
:10B26800FB1FE78020DFAA8921C531463306C902C2
:10B27800A6859750FB1FE780600D9844D620B22022
:10B288008E205285EFF0BFD12A8415ED02458547FF
:10B29800568797A6FFFF9386C67A5D464C005C8268
:10B2A8004EC423062101A306010023076101FD2BDB
:10B2B800B2502285225492540259F249624AD24A23
:10B2C800424B456182804E859750FB1FE780A0E581
:10B2D800C5B76D44F1BF79714ECEAE89C16526D22E
:10B2E8000147AA8489461796FB1F130626C2FD1537
:10B2F800054522D406D64AD0EF101001054429C9C5
:10B308002A891307300281461146F5452685EFF054
:10B318007FAC2AC655440DCD0357A900CE860146F9
:10B32800788411477885054718A1B2472C002685EF
:10B33800A38007003247FD573CA332473CB3EF10C8
:10B34800E0712A8411C532459750FB1FE780A0DDC4
:10B35800B2502285225492540259F24945618280A2
:10B36800411106C6EFF08FDC19C5B24041011753F1
:10B37800FB1F670043DBB24041018280011106CE0A
:10B388002AC6EFA06F81324591459797FB1F23A7E7
:10B3980007C69797FB1F23A107C69797FB1FA3858F
:10B3A800A70CEF30C027F24005616F20700F79714C
:10B3B8004AD006D622D426D201499397556063D83D
:10B3C80007041795FB1F0345350A2E899750FB1F65
:10B3D800E78000EE2A845DC518219307000A6310F0
:10B3E800F70A85474C08DC85EFA08F88AA841DC51D
:10B3F8009C8599C7084409C59750FB1FE780A0D2D0
:10B408002A208545EF300019CD47639AF406B250DB
:10B41800225492544A8502594561828083476101CA
:10B4280091CF71476363F7064D476378F7069386B4
:10B43800C7FE130730143357D74825C31797FB1F88
:10B44800032787BB01C7034751012DCB9C8599C7AB
:10B45800084409C59750FB1FE780E0CC5247B7075F
:10B468000001938707F07D8FB707120093870710B5
:10B478006307F70003476101ED476302F70A228576
:10B48800EF809FD81319F96859B7138717FE1377F8
:10B49800F70F93060002E3F3E6FA858B9DCB9797A7
:10B4A800FB1F83A7A7B5A5C72A201306B1004C0820
:10B4B80082979C85AA84ADEBD5D099B75C869947CD
:10B4C8002308F1002A206C0023170100EFA0EF9C4D
:10B4D800B5BF9797FB1F83A727B285CB2A201306F2
:10B4E800B1004C088297AA8435D183475101E39172
:10B4F80007F023089100834761012A206C005C86CD
:10B5080023170100EFA06F99E5B59944F9BF9C8511
:10B5180099C7084409C59750FB1FE780C0C02A2077
:10B528008545EF302007A1BF084459D59750FB1F28
:10B53800E78060BF51B75D71A2C4A6C286C6CAC003
:10B548004EDE52DC56DA5AD85ED6A5472A84B28433
:10B558006392F50E834745021A2232228507230299
:10B56800F5029307F7FFB307F602D440B3C70708FD
:10B57800B697542503CB070003C917008547638B8B
:10B58800F60493178900B3E7670141677D17638A5B
:10B59800E70A1A2863F7E70A50248507B3C707089C
:10B5A80085467EA40A209305E400631BD6007C84AC
:10B5B800930720307C869307800278855C872C006F
:10B5C800EFA02FB10824B165938505B8EF803FE15E
:10B5D80059458DA83307C702239004008149014AC1
:10B5E800930B3501B34A0708E3FD59F9B620DC404F
:10B5F8002C2813865900ED163E965E85B3C60608BC
:10B60800EF909FDE1DC1630B3A01C840B220B3051D
:10B61800350152959750FB1FE78040D3BE203E9AD4
:10B628009E20334A0A0885079EA0BE20BE99B3C94A
:10B6380009085DBF5822A9476311F70283474502ED
:10B6480089CF0145B640264496440649F259625AC4
:10B65800D25A425BB25B616182803428130934019B
:10B668004A8689451795FB1F1305858DEF90DFD70F
:10B6780039ED34284A8689451795FB1F1305058C33
:10B68800EF909FD629E534284A8689451795FB1FF0
:10B698001305858AEF905FD51DE934284A868945C8
:10B6A8001795FB1F13050589EF901FD40DE1DC20CA
:10B6B80009476380E702ED1793F7F70F2947636897
:10B6C800F70013079048B357F700858B99E30545B2
:10B6D80095BF8347440285072302F402BE2075B54F
:10B6E800411122C406C62E849770FB1FE780E03DF7
:10B6F80009C93C25138717006315E40093F707F879
:10B708003CA5B240224441018280411122C406C6B0
:10B718002E849770FB1FE780403B1DC111C008C0F5
:10B728001C251307E00F5D456388E7001307F00F3A
:10B7380059456393E7000145B240224441018280A4
:10B748000945DDBF411122C42A84210526C206C647
:10B758004AC0EFF04FB02420A51493F4D40F81E829
:10B7680058248547631DF7041C483149A1E3FD5758
:10B77800230104001CB4230204021305C40022445C
:10B78800B240924402496146814541011753FB1F6B
:10B79800670043C2B38724033E95084509C59750FF
:10B7A800FB1FE7804098850493F4F40F5C28084851
:10B7B800E3E2F4FE9750FB1FE780E0964DBF084C8C
:10B7C80075F975B7411122C4416406C626C29307AC
:10B7D800E4FF6301F502AA849DE19770FB1FE780EF
:10B7E800C02E09E91305F4FF9770FB1FE780E02DD1
:10B7F80011C106A1B240224492444101828085478A
:10B808006392F5049770FB1FE780202C2A847DD172
:10B81800FD571EA11C241307F00F6382E7021307CC
:10B82800E00F6389E7003420083401475146A685B4
:10B83800EFF0AF942285EFF0FFF0FD571CA423052D
:10B8480004004DBF8947E397F5FA8545EF40C046A8
:10B8580055F126859770FB1FE78020272A845DF91C
:10B8680051BF21C5011122CC06CE18259307F00F30
:10B878002A846308F70234210E21083501475D4602
:10B88800EFF0AF8F3820E1476318F7000A206C000B
:10B8980023060100EFA08FA1F9571CA42285EFF021
:10B8A8007FEAF24062440561828082809307F00F4C
:10B8B8006306F706011122CC26CA2A844AC84EC656
:10B8C80052C4B689328A3A8993068500AE8479468D
:10B8D800AA8517050000130505F906CEEFF0EF96C7
:10B8E800A3042401230144012322340185C0130544
:10B8F800C4006244F2404249B249224AA685D24471
:10B90800614605611753FB1F670043A4F240624478
:10B91800D2444249B249224A05618280828097878F
:10B92800FB1F2381A76E8280411122C406C695475A
:10B938002A846391F50683474502854685072302D5
:10B94800F5021E2258423022FD17B3C70708631EAE
:10B95800D602B3C7E72098239C330145A207D98FA5
:10B968007A2463F0E7020A2085075EA49305C400E1
:10B97800EF90FFEC0824B165938505B8EF803FA6EA
:10B988005945B240224441018280C946B387D70253
:10B99800BA97D1B75822A9470545E314F7FE0345DE
:10B9A800440213351500F1BF411122C406C69D4754
:10B9B8002A846396F5048347450285072302F50226
:10B9C8001E225842FD17B3C7E72098239C33A207CD
:10B9D800D98F7A25014563F0E7020A2085075EA41E
:10B9E8009305C400EFF04FCE0824B165938505B8E0
:10B9F800EF80FF9E5945B24022444101828058227F
:10BA0800A9470545E319F7FE034544021335150018
:10BA1800DDB7411122C426C206C6B5472A84B284BE
:10BA28006394F5048347450285072302F5020A213A
:10BA3800EF905FB09E201307F5FF014563C1E70251
:10BA48007A240A209305C400BA977EA4EF901FEDCC
:10BA58000824B165938505B8EF807F985945B240B1
:10BA6800224492444101828058229D470545E318AB
:10BA7800F7FE0345440213351500D5B7411122C41A
:10BA880006C6C5472A846390F5061E223A22FD178A
:10BA9800B387E7020347450205072302E502584238
:10BAA800B3C707083E973C333823A207D98F4167AD
:10BAB8007D176397E7000145B24022444101828027
:10BAC800138717005AA57A25E3F7E7FE9305C50003
:10BAD8000A21EF90DFED0824B165938505B8EF8062
:10BAE8001F905945D1BF5822A9470545E316F7FCD1
:10BAF8000345440213351500C1B7011126CA4AC8C7
:10BB08004EC656C206CE22CC52C4BC211547AA8ABC
:10BB18002E89B289B684639EE7023686CE854A8529
:10BB2800EFF09FE02A84631E0510854703459900BE
:10BB38006393F910D820A9476319F70C054A83467F
:10BB480029000345990001476946D685EFE0FFE2E1
:10BB5800F9A83547638CE7086361F7041D47638BD1
:10BB6800E7062547638EE706A547638FF90A05446C
:10BB7800034599002687CE860146D685EFE0FFDF8C
:10BB8800054A19E5CE852685EFE05FDA133A1500F8
:10BB98005DD4D9476306F40259A84547638EE70484
:10BBA8005D47E393E7FCD82585473686CE854A85E9
:10BBB800631AF704EFF02FC58547054AE306F5FA3F
:10BBC800F2406244D2444249B249924A5285224ADA
:10BBD800056182803686CE854A85EFF0FFDC99B70D
:10BBE8003686CE854A85EFF01F952DBF3686CE85E1
:10BBF8004A85EFF01FE23DB73686CE854A85EFF0DD
:10BC0800FFE70DB7EFF0CFCC45BF26878546014645
:10BC1800D685EFE09FD6E31305F285452685EFE04C
:10BC2800FFD0133A150021BF9E20B1F3054A4A857B
:10BC3800EFF05FB171B7A547E39CF9F29E208DFB49
:10BC4800F5BDA547E396F9F29E20E39307F2054A6E
:10BC580089B79E21639F071C397126DA4ED652D4C4
:10BC680006DE22DC4AD8A021ED47AA89AE84328AB2
:10BC78006315F4021787FB1F0347C7389307F00FB4
:10BC88000144631FF7049947F2506254D254425951
:10BC9800B259225A3E8521618280F5476311F40822
:10BCA8009786FB1F83C606361307F00F9947E38D67
:10BCB800E6FC9770FB1FE78040E12A8415C1302518
:10BCC80005C29317466063D40700814775BFF545E1
:10BCD8004E85EFE0FFD23C2493E707F83CA4F5B784
:10BCE800D62090448C3088203800EF903FDDAA871A
:10BCF80041FDB42038000146CE851785FB1F03455A
:10BD08006530EFE09FC7AA8741F1B24799C3230086
:10BD18000A00BC207547E39AE7FA69F07DB7977087
:10BD2800FB1FE78080DA2A894DD185476317F40421
:10BD3800CE2088443000EF90DF81AA8731F5834711
:10BD4800290015476382E702E51793F7F70FC14605
:10BD580063E1F6043317F0281377574411E7639A21
:10BD6800D7028327090195C7B0203400CA854E85BC
:10BD7800EFF0BFD82300AA0089BF38219147E31507
:10BD880087F05841E30207F0CE208844300002973C
:10BD98006DB7034599009787FB1F83C7F76C6381CD
:10BDA800A702B42038000146CE85EFE01FBD2A84E3
:10BDB80009E9AC202800EFE07FB719C123000A0089
:10BDC8000144034729008D476318F7043C8403574F
:10BDD800C90063F4E7002316F9008355C9004E85AE
:10BDE800EFE0BFF91787FB1F03578737ED4763F568
:10BDF800E7028357C900DD4663F0F60293863700F1
:10BE080063D1E60211669385470013060629B3C578
:10BE180005084E85EF80A01F4A85EFF0BF92A287E4
:10BE2800A5B511669305B00F13060629B355B70AD1
:10BE3800CDB799473E858280011106CE26CA4AC8E9
:10BE480022CC4EC652C49784FB1F9384E461882495
:10BE58009307800291653305F5029385657017890C
:10BE6800FB1F1309E919334505089740FB1FE780B5
:10BE7800601E90249307800281453306F602232032
:10BE8800A9009740FB1FE780E052832709004D4532
:10BE98009DCB0144130A8002FD599C24636DF40272
:10BEA80017050000130525DBEFE0FFEB1705000081
:10BEB80013054583EF908FDA170500001305C59029
:10BEC800EF30B0560145F2406244D2444249B2498B
:10BED800224A05618280B3074403032509006146AD
:10BEE800814505041374F40F3E9523103501230191
:10BEF8000500231435012305050023020502310539
:10BF08009740FB1FE780004B49BF01458280178798
:10BF1800FB1F0347F755814763E4E700014582802B
:10BF28009221938645006314A6002E85828085079A
:10BF3800B685DDB71DC5411122C406C63821930751
:10BF4800D00F2A8463EBE7000E2128310147F94618
:10BF58005D46EFE09FA2F9573EA0B240224441015E
:10BF6800828082801787FB1F034797508147FD56C1
:10BF780063E3E700828016A1230105008507110508
:10BF8800C5BF014582809785FB1F9385B5F693074A
:10BF9800000285469CA1FD571787FB1F230CF7F469
:10BFA8001787FB1FA307F7F41787FB1F2303F7F473
:10BFB8009787FB1F239ED7F29787FB1F23920706BD
:10BFC8009787FB1F23AC07049787FB1F23A607044B
:10BFD8009787FB1F23A007041786FB1F1306C6F0CD
:10BFE8009787FB1F938707F65CC29787FB1FA38B76
:10BFF80007009787FB1F938767E9094718A298A34B
:10C0080098AB2380E7022388E7021787FB1F1307F3
:10C0180027F294A7D0C794AFD8DB1785FB1F130569
:10C0280025F20D471786FB1F1306C6F09786FB1FE0
:10C038009386C6ED238CE702C8C323950700D0CBAF
:10C04800239D0700CCCFD4D323840702239507026E
:10C0580023A60702239D07021787FB1F0327C7FA9A
:10C06800D8DF9787FB1F9387A7E1170700001307FF
:10C07800870B23A00700D8C323A40700828041119F
:10C0880006C6EFF0DFE809C52821B24041018280E9
:10C098000145E5BF411122C426C24AC006C6AA848A
:10C0A8002E893284EFF0BFE6AA8711E94165CA8577
:10C0B8007D15EFF0DFE5AA87454581C786A3A0A3D4
:10C0C8000145B2402244924402494101828021E361
:10C0D80009483547639E0603011106CE22CC182273
:10C0E80010322206598E32C6B377F64085E7CC4522
:10C0F8002A842EC4EFF0BFF832460147630EC5000C
:10C1080022856244A245F24005616FF0BFF82D47D1
:10C118003A85828013070008F24062443A85056137
:10C12800828083C80500094863910803DC4103C87D
:10C1380007009C33A207B3E707010D68130828908E
:10C148006395070189476FF09FF8054582800111C3
:10C158004EC606CE22CC26CA4AC89789FB1F9389A9
:10C1680059D903C709009307F00F630FF7022A890B
:10C178002945AE8432849740FB1FE780600DAA856D
:10C1880005C59307100B1EA12302050002A56244F2
:10C198002311250166A1F24003C50900D244424992
:10C1A800B24905616F806F8BF2406244D2444249C4
:10C1B800B24905618280411126C2AE849785FB1F72
:10C1C80083A585E422C406C62A84EFF05FEB0989BB
:10C1D80009C922852244B240A685924441016FF0E4
:10C1E8008F8FB2402244924405454101828041111B
:10C1F80022C426C24AC006C6AA84130445001309ED
:10C20800850B1E209DC3084409C59740FB1FE78086
:10C2180080F12285314681459740FB1FE7808019D0
:10C228003104231A04FEE31E24FDB2402244FD57C4
:10C238009EA002499244410182809786FB1F83C6D3
:10C2480036239787FB1F83A7A7DC01476394E60083
:10C25800014582808E231386870B6394A5003E8553
:10C26800828005071377F70FB287CDB7AA8717859E
:10C27800FB1F032565DA01C95A216314F700084535
:10C2880082800841CDBF8280411106C6EFF01FFEB3
:10C2980009C50845B240410182800145E5BF797171
:10C2A80022D41384450026D24AD052CC5AC82E8AAA
:10C2B80006D64ECE56CA5EC622892287014B8144D5
:10C2C80081468147BD45122345CAB5EE46233E2324
:10C2D800B286A697B3C70708050B3107E315BBFE5F
:10C2E800ADC491659385457026859740FB1FE7800F
:10C2F80060D6AA8B39C90C44D1C9814A81495220D8
:10C3080033853B019740FB1FE78040045E200844CB
:10C31800BE99B3C909089740FB1FE780C0E063983E
:10C328000A003109854A832589004A84E9F931469A
:10C3380081452285850A9740FB1FE780A007638215
:10C348006A053109CDB7630ED6000145B2502254B3
:10C3580092540259F249624AD24A424BB24B456161
:10C3680082803223E313F6FE5223B294B297B3C409
:10C378000408B3C707088DB78547E3E367F70545A2
:10C38800F1B723267A0123149A00D5BF1309C400F4
:10C39800854A814949BFAA871785FB1F032585C799
:10C3A80011E1828018453A276314F700110582804D
:10C3B8000841FDB7411106C6EFF0FFFD09C50A2186
:10C3C800B240410182800145E5BF411106C6EFF048
:10C3D8009FFC09C52821B240410182804145E5BF43
:10C3E80041111786FB1F1306E6C222C40042AA8623
:10C3F80006C62E8501471DCC1C44AE271C406396FB
:10C40800D5021DC71CC301C92146930544009740A6
:10C41800FB1FE780A0F322859740FB1FE780A0D091
:10C428000145B24022444101828022873E84E1B71F
:10C438001CC2D1BF0545F5B701119786FB1F93862E
:10C44800A6BD26CAAA84884222CC06CE2E840147DD
:10C458000DCD52211C416315960215C71CC3974088
:10C46800FB1FE78040CC2C002685EFF07FF701E525
:10C4780019C0B2471CC0F2406244D24405618280B0
:10C488002A873E85F1B79CC2D9BF0545EDB7411152
:10C4980022C42A84090506C6EFE0EFDBFD573CB04D
:10C4A800B240224441018280411122C4416406C63F
:10C4B80026C29307E4FF6301F502AA849DE1976011
:10C4C800FB1FE780A06309E91305F4FF9760FB1FD2
:10C4D800E780C06211C106A1B240224492444101E2
:10C4E800828085476392F5049760FB1FE7800061AF
:10C4F8002A847DD1FD571EA13C201307F00F6382CB
:10C50800E7021307E00F6389E70028300147F9467F
:10C518005146A685EFE06FC62285EFF05FF7FD571D
:10C528003CA0230204004DBF8947E397F5FA8545EF
:10C53800EF30807855F126859760FB1FE780005C17
:10C548002A845DF951BF5D71A2C4CAC086C6A6C25D
:10C558004EDE52DC56DA5AD82E84AC21F9472A89A5
:10C568006392F5049760FB1FE78040592A8405C150
:10C5780038219307D00F63ECE70028310147F946CB
:10C588000146CA85EFE06FBF2285EFF05FF00145F5
:10C59800B640264496440649F259625AD25A425B3A
:10C5A80061618280832A0400B7070001938707F03E
:10C5B80037071200B3F7FA0013070710B28981444E
:10C5C8006388E7022EC69760FB1FE7802053B245B9
:10C5D800AA8419CD502109CE93174660E3C907FAFA
:10C5E8004A85EFE0EFC1DC2093E707F8DCA045B708
:10C5F800178AFB1F130A0A9003470A009307F00FD4
:10C608001945E307F7F8E147E3E4B7F893D71500CE
:10C61800FD17171702001307E776B3E7E72003A80B
:10C628000700E30708F603AB4700E3030BF6B3CABA
:10C638000A0863850A00C947E39CF5F456201044AC
:10C648000C3008203808029821F52C084A85029BEE
:10C658001DCD183015FF3820230AA100B94723083B
:10C66800E1006314F702E24798239C33A207D98FAD
:10C678000C084A85FC81EF904F8211D914080546B1
:10C68800D9454A85EFE0AFDA21B7BC84D5B7342065
:10C698009147E38EF6EE03450A0038080146CA853D
:10C6A800EFE0AFADE31605EE2C202808EFE00FA869
:10C6B80019C1238009001840B7070001938707F0C4
:10C6C8007D8FB707120093870710E302F7ECE3802A
:10C6D80004EC3C2021BF411122C406C62E84976079
:10C6E800FB1FE780A04109C95C2113871700631568
:10C6F800E40093F707F85CA1B2402244410182802C
:10C70800397152D42E8A4ED69305E100AA895285F2
:10C7180022DC4AD856D25AD05ECE06DE26DA3289D4
:10C72800368BBA8BBE8A9760FB1FE780A03F054413
:10C7380025C1AA8428873944EFF05FB331C903289B
:10C74800450063070804D6875E87DA864A86A68589
:10C758004E8502982A840DED9307E00F638AFA024A
:10C76800982089476316F702DC4098239C33A20778
:10C77800D98F0D6713072790639CE700834719003B
:10C7880003460900D285A2075D8E4E85EFF03F9CD7
:10C79800F25022856254D2544259B259225A925ABE
:10C7A800025BF24B21618280797122D422214ECE24
:10C7B800AA89228556CA06D626D24AD052CC5AC849
:10C7C8005EC662C4AE8AEFF05FA705E52285EF90EA
:10C7D8004FF5594411E10144B25022852254925434
:10C7E8000259F249624AD24A424BB24B224C456145
:10C7F800828003C7890085476307F700EFF03F9FF2
:10C8080003D52900E9B7AA85AA8413858900EFF022
:10C818001FA92A8415CDFA209624D044CE2003D50A
:10C828002900E147EFF0DFEDD9472A846318F500C6
:10C8380023A604002685EFF09F9B71BF19E126858A
:10C8480075BFDE2026852390FA00EFF05F9A69B75E
:10C8580013894400014AB94B594C3D4B8355090093
:10C8680085CDE14763077A010357C900D94711E32A
:10C87800E14703572900835649000326890003D559
:10C888002900EFF0FFE72A846310850323240900B9
:10C89800050A3109E3146AFD2685EFF05F952DD06E
:10C8A800D947E31BF4F205BF65D5835709002390E8
:10C8B800FA00F9BF011170879307E00F1306E10032
:10C8C8000147894606CEEFF0BFE3F240056182805A
:10C8D80079714AD00359850022D426D22A84AE849D
:10C8E8004A859305210106D69760FB1FE7808023C0
:10C8F80079C51C252AC693F707029DC7A881EFF0C2
:10C90800BF98B245AA8711E9239024013945B2504E
:10C91800225492540259456182802A2049468297BE
:10C9280001C51E249EA0E5B7035924004A85EFF0EF
:10C93800DF9001ED41657D15EFF03F9009E51E247C
:10C9480025459EA0E9B72310250113074500814717
:10C95800BD46122339EE3147B387E70293058400B9
:10C9680031462EC691073E959740FB1FE780009EF3
:10C97800B245314648089740FB1FE780209D522466
:10C988002A2041478146DD45EFE0CFC42ACE09E59C
:10C998001E2445459EA0A5BF0C4852249740FB1F66
:10C9A800E780C09A2A204C08EF906FD32DD15945C3
:10C9B800B9BF85073107E39ED7F825459DB70545DB
:10C9C8008DB7797122D42A840A254AD02E899305F5
:10C9D800E1004ECE06D626D2B2899760FB1FE780CB
:10C9E80060142DC91C25AA8493F707028DEF183807
:10C9F8009307200511E35C20362450440E242A2096
:10CA08000147EFF0FFCF21E11C38B9E32A20EF906E
:10CA18004FC9AA8759458DCFB25022549254025912
:10CA2800F249456182802887EFF01F86AA870DC5E5
:10CA38002A204946A68582975DD91E242310F9002D
:10CA48001C3899E7D1BFD947E319F5FE23800900BF
:10CA58000145D9B70545D5B73945C5B7797122D448
:10CA68004AD04ECE52CC56CA06D626D2AA892E8A8B
:10CA7800B28A36899760FB1FE780400809440DC5D4
:10CA88003C211307E00FAA845D44638FE700130776
:10CA9800F00F5944639AE70063920A02D2854E85E3
:10CAA800EF902FCC2A8421C1B2502285225492546F
:10CAB8000259F249624AD24A4561828003550A0006
:10CAC8009305E100231701009760FB1FE7808005AD
:10CAD8002887EFF09F8FAA8505464E85EF20107DA9
:10CAE8002A844DDDD1B79307F00FE30FF9FA938647
:10CAF80024007946A68517F5FFFF1305E543EFD017
:10CB0800DFF4A38124014DB7797126D24ECE52CCE1
:10CB180056CA5AC85EC606D622D44AD062C466C26D
:10CB2800AA8A2E8BB28B368ABA899774FB1F83A484
:10CB3800644EB9C0804483DC44000149035CA4000E
:10CB4800631499018440F5B73E2463F7570105093A
:10CB5800410433490908EDB7E36BFBFE63090A009A
:10CB68000C204840D2865E86EF801F886DD1638492
:10CB7800090023908901A284B25022540259F24933
:10CB8800624AD24A424BB24B224C924C268592546E
:10CB9800456182809A21B621854763E3E60429C36B
:10CBA800D42101111386550022CC1775FB1F1305DC
:10CBB80025392E84894506CE32C6EF80FF82C147CB
:10CBC80019C9542032462E200A200147EFF0DFF31E
:10CBD800A94711C18147F24062443E8505618280C0
:10CBE8003E8582802E860A22AE21854763E1A50212
:10CBF80019CD542241110147150606C6EFF0DFF0A2
:10CC0800A94711C18147B2403E85410182803E85D6
:10CC180082802E860A22AE21854763E1A50219CDBE
:10CC2800542241110147150606C6EFF0FFEDA9474A
:10CC380011C18147B2403E85410182803E85828094
:10CC480039714ED6BE2183D9050006DE22DC26DAEC
:10CC58004AD852D456D25AD05ECE62CC66CA63E461
:10CC680037152A8A054563830912416BAE8A231456
:10CC7800010002C6014401497D1B894B054CC94C82
:10CC880083D52A000147814601464E8523130100BA
:10CC9800EFF09FE7AA8471C509EC130720029306F9
:10CCA80061005A8695455285EFE0CF922A84630E3B
:10CCB800050E38849C2025C71885630187054147E0
:10CCC8006394E70ABE244146130524001CA0BE2431
:10CCD800A1831CB0CC409730FB1FE7802067490434
:10CCE8003C848507B3C707087C8463FC2707BE24F8
:10CCF800638967078509B3C9090859B76396770730
:10CD0800BE240946130524001CA0BE24A1831CB020
:10CD1800CC409730FB1FE78060631104D1B722C66F
:10CD280003596100B82413052400638F7701335930
:10CD380099032305710118A0BE244146A1831CB0A4
:10CD4800CC401379F90F41BF2305810118A0BE24F7
:10CD5800135929001379F90FA1831CB0CC40094657
:10CD68004DBF3C8429459DC32C005285EF80FFE6CA
:10CD780009CD34001546D9455285EFD05FEB11C572
:10CD880032459730FB1FE780003A0145F250625464
:10CD9800D2544259B259225A925A025BF24B624C0F
:10CDA800D24C216182800545D5B74545C5B717776F
:10CDB800FB1F0347A728854763F7E706011122CC25
:10CDC80026CA4AC806CE2A84AE8432899760FB1FD9
:10CDD800E780C0D211C538219307E00F6307F70435
:10CDE800631B090022856244F2404249A685D24469
:10CDF80005616F90CF938A209305E1002317010006
:10CE08009760FB1FE78000D22887EFF00FDCAA8528
:10CE180005462285EF20904971D5F2406244D244FC
:10CE2800424905618280594582805D45FDB74111BF
:10CE380022C406C626C293F705022A84328585C312
:10CE4800EFF0AFD8AA8505462285EF2030469547F2
:10CE58006305F500BD476315F502214515A093F755
:10CE68008500B6849DC3EFF04FD6AA850546228576
:10CE7800EF20D04309C59C3481C79C2491C3014548
:10CE8800B24022449244410182809397456063D71F
:10CE98000700EFF08FD3AA850146D1BF89890D45D8
:10CEA800F9FDF9BF7971AE8622D42A848A229305C6
:10CEB800E10106D636C69760FB1FE780A0C611C9F8
:10CEC8000C2522852254B246B087B25045616FF0D6
:10CED8001FF6B2502254054545618280411122C493
:10CEE80006C693F705022A8432858DC3EFF0EFCD8D
:10CEF800AA8505462285EF20703B1547AA8763055A
:10CF0800E5003D47631DE502A14715A893F7850095
:10CF180099CBEFF08FCBAA85054622852244B240F3
:10CF280041016F20B0381397456063570700EFF051
:10CF3800CFC9AA850146D5B7898991E18D47B24005
:10CF480022443E85410182807971AE8622D42A84AA
:10CF58008A229305E10136C606D69760FB1FE78053
:10CF680060BCB24609C90C2522852254B087B2504C
:10CF780045616FF0BFF6B250225405454561828085
:10CF88003E257971416722D426D24AD04ECE06D6A4
:10CF9800231701007D17AA84328436898149638D5D
:10CFA800E7009420D040138517001307E1003345AC
:10CFB8000508EFF07FB5AA899420D04089451775F8
:10CFC800FB1F1305E5F7EF802FC215C5A2242285A4
:10CFD800EFF04FBE09C57D142A9433440408630456
:10CFE800090023108900B2502254925402594E85E8
:10CFF800F249456182809420D04089451775FB1F0E
:10D008001305C5F3EF804FBE71F19420D0408945D8
:10D018001775FB1F130505F2EF800FBD11C9E388D3
:10D0280009FA3C87E39587FA03D4A9007D1475B7FC
:10D03800A22475B7397122DC26DA4AD84ED652D4E2
:10D0480056D25AD05ECE06DEBE8B9C252A8AAE8486
:10D05800C18BB28A36843A89C289468B9DEF942067
:10D0680089476383F6065685EFF04FA005CD8328E0
:10D0780005006389080222866254F250925A5A883F
:10D08800CE87025BB2595E87CA86F24B4259A685A3
:10D098005285D254225A216182883285EFF0CF9E80
:10D0A800AA8709ED3945F2506254D2544259B2590F
:10D0B800225A925A025BF24B216182802946A68548
:10D0C8005285829749DDC5B7DC4003C31700982312
:10D0D8008D6722033363E300138647901317536069
:10D0E800E343E6F81386F78F634BE60293862780BF
:10D0F800630FD70863C8E604F977938707803E93E0
:10D10800854733430308E3E067F62D45E39D0BF8B5
:10D11800DC449023CC432310C90022851DA2F57757
:10D128009387F76F3E938D473343030863E0671295
:10D1380017170200130747BF3343E3208327030071
:10D14800BA97828793873780E31FF7F02D45E39CD2
:10D158000BF485472310F900DC4481459C231CA06F
:10D16800AA240505334505089760FB1FE780809BC7
:10D17800835709004DE991072310F90011468145AD
:10D18800130514009730FB1FE780C02241A82D45E6
:10D19800E39B0BF0DC446C0083C917009823A209B9
:10D1A800B3E9E90011472310E9009C234E851CA030
:10D1B800DC449C331CB09760FB1FE780A096AA84D0
:10D1C80025C13086C1659306E100FD158329C50098
:10D1D800EFF01FDB09ED9420D04089451775FB1F40
:10D1E8001305C5D5EF804FA019E1FD577C8703C70C
:10D1F800090089476310F70283A54900094613050A
:10D2080044009730FB1FE7806014835709008907A3
:10D218002310F9003C873CA0A1833CB0014561B5CF
:10D2280023173101C5BF18218907BA972310F900C0
:10D238003E251CB03E25A1833CA010214C4113057E
:10D2480034009730FB1FE7806010C9BF2D45E39C71
:10D258000BE42310D900DC449C231CA0DC449C3341
:10D268001CB06DBFC8449730FB1FE780C017334719
:10D2780005081D45E36977E36380EB02B38679010E
:10D2880063C6E60033077741B3490708CC44231047
:10D2980039014E86DE9551B58149CDBF2D45E394C0
:10D2A8000BE0CC445285EFE09FDD89472310F9005D
:10D2B80008A0218108B09DB72D45E3960BDE89476C
:10D2C8002310F90049BF2D45E39F0BDCDC441D47C3
:10D2D8002310E900982318A0983318B0BA2338A06F
:10D2E800BA23218338B0D82358A0FA2358B0FE2394
:10D2F800A1837CA025B75D71A6C2AA842A214EDE2F
:10D3080052DC56DA5AD85ED662D466D26AD06ECE6D
:10D3180086C6A2C4CAC0AE8AC16BEF80AFA1130C87
:10D32800F5FF2A8A8149977DFB1F938DED0A977C2B
:10D33800FB1F938CACCE177BFB1F130B6BCEFD1B17
:10D34800334D0C08DE2463F6F90083D70D0063CD56
:10D358008701AA209775FB1F93850508EF809FA971
:10D368002A841DCD59442DA89C449305E100B3A7F8
:10D37800F92003C917009C2322093369F9004A855B
:10D388009750FB1FE780007AAA851DE923902A01A0
:10D3980003A54D0009C59730FB1FE780C0D8054499
:10D3A800B6402285264496440649F259625AD25A12
:10D3B800425BB25B225C925C025DF24D61618280ED
:10D3C80083C8440083A60C003087AA206A88814756
:10D3D8005A87EFF03FC62A8419C923902A0103A56A
:10D3E8004D005DDD9730FB1FE780E0D355BF83A775
:10D3F8004D0099EFAA20514781465E86BD45EFD082
:10D408007F9D23A2AD0009E523902A01454449BF29
:10D4180083D70D0003570B003E9763474701330737
:10D42800FA407D172310EB0003A54D0003560B00AF
:10D4380083A50C003E9585099730FB1FE78000F116
:10D4480083D70D0003570B00B3C90908BA97239077
:10D45800FD00CDBD397126DAAA842A214ED65AD0CC
:10D4680006DE22DC4AD852D456D25ECE62CC66CAD8
:10D478006AC82E8BEF800F8CAA89D424AE248A2404
:10D4880078001386D400EFF02FE805C5938BB9FF19
:10D498002A84E5190149177CFB1F130C2CB8977CCB
:10D4A800FB1F938CECB733CA090863497901631BE6
:10D4B80009109E2429452310FB009DA8035DC10087
:10D4C80083C8440083260C00AA20528881476687B7
:10D4D8006A86A285EFF01FB619C9AE242285930685
:10D4E800E1006A86EFF0DFA92A8461F0C9B783D723
:10D4F8000C009228E313F6FE83250C00C8489730E9
:10D50800FB1FE78020F671D99779FB1F9389C9EC37
:10D5180083A7490095EFAA204166454781467D16B5
:10D528009D45EFD03F8B1DE19E2445452310FB0010
:10D53800F2506254D2544259B259225A925A025B5A
:10D54800F24B624CD24C424D2161828023A2A90049
:10D55800AE24835AA40022859306E1006A86EFF080
:10D568003FA22A84E3830AF883A749001307190016
:10D5780033470708CA972380570183A7490093DADE
:10D588008A0093062900BA972380570113073900A8
:10D59800110983A74900B3C606083347070833496A
:10D5A800090811C93087B69790A383A7490021823B
:10D5B800BA9790A3DDBDB697FD5694A383A74900FB
:10D5C800BA9794A3AA209775FB1F9385E5E0135992
:10D5D800290023902501EF80AFEB39D9594589BF40
:10D5E800411122C406C693F705012A84328585C3F2
:10D5F800EFE0BFDDAA8505462285EF20204B954741
:10D608006305F500BD47631DF502214515A893F78D
:10D61800450099CBEFE07FDBAA85054622852244A9
:10D62800B24041016F20804893F7050491C7EFE0AD
:10D63800DFD9AA850146DDB713C5F5FF05890605BB
:10D64800B240224441018280797122D426D252CC40
:10D6580006D64AD04ECE56CA5AC82A8AAE84014443
:10D66800DE206364F400014581A083AA04009319B5
:10D67800140013891900B327542103CB0700B3877B
:10D688002A0188239305E100220533656501975037
:10D69800FB1FE78020491DE123806A019C40054566
:10D6A8003E990347090098B3B25022549254025944
:10D6B800F249624AD24A424B456182800C25308742
:10D6C8005285EFF0FFF101CD9C40BE9903C70900D8
:10D6D80098A39C403E990347090098B3F1B7050405
:10D6E80033440408B5BF0111AE8722CC2A848A23AB
:10D6F8009305E10006CE9750FB1FE780A04209C9B9
:10D708000C25228562443087F24005616FF05FED99
:10D71800F240624405450561828039715AD02A8BEE
:10D728002A2126DA4AD806DE22DC4ED652D456D230
:10D738005ECE62CC66CAAE84EF70DFDF2A8983468C
:10D74800CB008355AB0003558B0078001306DB0034
:10D75800EFF08FBB63050516C16A130AA9FFAA8BF0
:10D7680001449779FB1F9389698B977CFB1F938CE6
:10D77800ACC6FD1A6D19334A0A08035CC10083C59B
:10D788008B0003552B006286EFF09FE563180514A4
:10D7980083484B0083A6090003552B005288814714
:10D7A8001777FB1F1307C7876286DE85EFF09F8810
:10D7B8006316051205CC83D72C001777FB1F035778
:10D7C800278611076395E700A29763C42707977513
:10D7D800FB1F938565C0BE2103552B003354F4020B
:10D7E80082A1EF80EFE415C1594505A003552B0030
:10D7F800494781465686C545EFD0CFDD23A2AC0008
:10D8080015E183D7AB0045459EA0F2506254D2542F
:10D818004259B259225A925A025BF24B624CD24C8C
:10D82800216182809767FB1F83D7877F91072391A8
:10D83800FC0083A74C0003D7AB006286A29798A38D
:10D8480083A74C001307140033470708BA9703D778
:10D85800AB009306E1005E85218398A38355AB0056
:10D86800176CFB1F130CCC7BEFF08FF103A74C0058
:10D878003C87130624003346060832971CA303A7E7
:10D888004C0093063400A183B3C6060836971CA340
:10D89800AA8B03A54C0011043344040803560C005A
:10D8A80083A50900229563910B029730FB1FE7803F
:10D8B800E0A983570C00A29733C4070809F88357D7
:10D8C8008B0029459EA091B79730FB1FE78000A8E1
:10D8D80083570C003E943344040845B583D7AB0006
:10D8E8009EA0E31604EE83578B009EA039BF1D71DE
:10D8F800A6CACAC8AA84035985002A21A2CCCEC6C2
:10D90800D2C4D6C2DAC05EDE62DC6AD886CE66DAF7
:10D918006ED6AE8AEF701FC2130BD5FF0144711586
:10D92800138CD400976BFB1F938B4B6F176AFB1FED
:10D93800130A0A6F177DFB1F130D0DAAB3490508BB
:10D94800635D6411D424AE241307E10162864A851D
:10D95800EFF08F9BAA8C630205100359A500B087CE
:10D968000C25AA2032C6EFF0BFC7631D050E83C879
:10D97800440083A60B003246AA204E88814752876E
:10D98800E685EFF02FEB79ED15C483570A000357AE
:10D998002D0089076302F7069775FB1F9385C5A3BA
:10D9A800BE21AA20B357F4029EA1EF80EFB60DC1A5
:10D9B800594539A8AA2041664D4781467D16A54597
:10D9C800EFD04FC12322AD001DE123902A01454528
:10D9D800F6406644D6444649B649264A964A064B16
:10D9E800F25B625CD25C425DB25D256182808357E6
:10D9F8000A0089072311FD0083570A00A29763DEF6
:10DA0800670583274D0003D7AC00930D2400A29728
:10DA180098A383274D0003D7AC00050433440408BA
:10DA28002183A29798A303254D0003560A0083A5D6
:10DA38000B00B3CD0D086E959730FB1FE780009162
:10DA480083570A00BE9DC167FD1733C40D08E3095B
:10DA5800F9EE050933490908E5B5294515FC239070
:10DA68002A01BDB76DDC0DBF1E21411126C206C6B5
:10DA780022C44AC0444189EB8947B24022449244B7
:10DA880002493E85410182809420D0402A848945FC
:10DA98001765FB1F1305C54AEF701F9511C93C2078
:10DAA8002547E51793F7F70F637FF700E147F1B7CD
:10DAB8009420D04089451765FB1F13052548EF7052
:10DAC800BF9271FD55BF1769FB1F13096942835641
:10DAD80009008547DDD21A203697C166E3CFE6F8FC
:10DAE80091659385257031459720FB1FE780805607
:10DAF800AA84CD4759D1314681459730FB1FE7802D
:10DB0800608B1A208355090001468147B386F500CA
:10DB1800B3C6060863E9E70201C62E972310E90099
:10DB280023A004002146A285138544009730FB1FDB
:10DB3800E780C0811767FB1F1307C74D1C4381CFC0
:10DB48003E879C43EDBF50401395470085072A96B2
:10DB580036A6054665BF04C3814705B7011106CE41
:10DB680022CC26CA4AC809E90944F24022856244FF
:10DB7800D2444249056182802AC6AA84280036898F
:10DB88006C845085EFF05FEE2A8465F1E30F09FCA1
:10DB9800BE24F9DB91659385557031459720FB1FAD
:10DBA800E780404BAA8715C1BA249766FB1F938666
:10DBB800A646232005005AA198422324250101C71F
:10DBC800BA861843EDBF9CC24DB74D4479BF9767DD
:10DBD800FB1F9387374398230DE3054798A30589CF
:10DBE80009CD9766FB1F9386A6294146914517657F
:10DBF800FB1F1305A5296FF07FF601458280976703
:10DC0800FB1FA388A72E828041677D176315E50057
:10DC18002E856FE02FB5411106C6EFE04FAF09C55D
:10DC2800FD571EA123010500B24041018280011168
:10DC380026CA06CE22CC4AC88547AA846392F50430
:10DC48002685EFE08FDF31E941699305F9FF130776
:10DC5800E10089461766FB1F1306862D0545EFE090
:10DC6800BFEA2A847D1905C44C442685EFF0DFF904
:10DC7800308722858146CA85EFF08FB02A84E5B7C0
:10DC880089476396F5008545EF20000355D9F24092
:10DC98006244D244424905618280EFE04FD56DB7B6
:10DCA800411122C406C626C21764FB1F1304C47B95
:10DCB80008349767FB1F23AD07349767FB1F23A71B
:10DCC80007349767FB1F23A1073459C59307200C16
:10DCD8003305F5029165938515709764FB1F93844E
:10DCE80024331905334505089720FB1FE780803644
:10DCF80010349307200C81453306F60288C01906B4
:10DD08009720FB1FE780006B9C4018348145938661
:10DD180047007D5563EAE5069306800BB306D702F4
:10DD280001460507FD55B6979766FB1F23A0F62EFB
:10DD3800BE868EA2ACB2ACA2238206000506990666
:10DD4800E369E6FEF95696A399463307D702BA97D0
:10DD58001767FB1F232AF72A17E5FFFF1305E57E40
:10DD6800EFD00F8117F5FFFF13052597EF70AFEF81
:10DD780017E5FFFF13058573EF10306BB24022449F
:10DD88009244014541018280239EA6FE368613886F
:10DD9800460B23100600232406003106E31B06FF6A
:10DDA80085059386860BBDB7411106C622C42A8411
:10DDB800EFC08FA1EFE02F9D1765FB1F0325C5243A
:10DDC8009767FB1F23878712EFE0CF999767FB1FA1
:10DDD800238287122244B24017050000130565E527
:10DDE80041016F1090649397556063DB072E79713A
:10DDF8001765FB1F0345E50F22D44AD006D626D265
:10DE08004ECE2E899720FB1FE780804A2A8441CD79
:10DE180018219307000B6315F70885479764FB1FC4
:10DE28009384C41FDC849C402315010081EFEF001C
:10DE3800C0759165938535709720FB1FE780802119
:10DE480088C031C9614681451765FB1F1305C55850
:10DE58009720FB1FE7800056834944008947639356
:10DE6800F90825279764FB1F938404578AA02A2062
:10DE7800A685EF70FFD2AA869E202A201A248DEE4E
:10DE88006363F7001EA40E24EFC03FEF2285EFC0A6
:10DE98001FC49C8491C74C2013058400EFD04FCC3D
:10DEA8002285EF606FB6B25022549254F24913158E
:10DEB800F9680259456182806363F7001EA41E2435
:10DEC800D9459766FB1F938626510D469EA0EFC045
:10DED8001FD68D4545DD1765FB1F1305E54FEFD0B0
:10DEE8002FC86DB79387A9FF93F7F70F4947E36FDB
:10DEF800F7F817070200130727E4B3C7E7209C4386
:10DF0800BA9782879305A1002285EFF0AFD4AA843F
:10DF180035DDD9476394F40A85092A2093F9F90F66
:10DF28009766FB1F9386464B4E86D945EFC03FD078
:10DF380031DDCE854DB79305A1002285EFF03F9BDB
:10DF4800F9B7835984006C004E859750FB1FE78012
:10DF580060BDAA842DC12A2041669306E100554779
:10DF68007D16AD45EFC01FE79769FB1F9389C9462A
:10DF780023A2A900AA8655CD834844000358E1008E
:10DF880030862A20A68581474E87EFF0AF8AAA847B
:10DF98006312050E2A20CE85EF70BFDDE30805EE7B
:10DFA8002A20D945CE862D46EFC07FC8AD45E30F60
:10DFB80005EC4E852DB72315310185441830D1471E
:10DFC800E306F7EC5C209769FB1F9389E9402A2058
:10DFD8002380F9003C85CE85238299002391F9009E
:10DFE800EF70AFEBE30405EA2A20CE860546D94553
:10DFF800EFC0FFC3E30C05E8854565BF835984007E
:10E008006C004E859750FB1FE780C0B1AA8445D5A8
:10E018002A2041669306E10059477D16B545EFC0B1
:10E028007FDB9769FB1F9389293B23A2A900AA8656
:10E0380009E51E24C5447C8551B78348440003582C
:10E04800E1003E2430862A20A6854E87EFE09FFE19
:10E05800AA840DE12A20CE85EF701FD5E30805E2DA
:10E068002A20D945CE863546EFC07FBCB545E30F9B
:10E0780005E081B7D94703A549006397F4009720C5
:10E08800FB1FE780400A19B59720FB1FE780A0090E
:10E098001E247C8525B79305A1002285EFF0AFA546
:10E0A800BDB59305A1002285EFF02FE78DB51306C6
:10E0B80091009305A1002285EFE0BF9089BD9305EB
:10E0C800A1002285EFE0DF80AA84E31405E4A3041D
:10E0D80001006DBB9305A1002285EFE0EFEC05BDC3
:10E0E80001458280F1CE011156C2AE8A854526CA05
:10E0F8004EC652C406CE22CC4AC82A8AB284B689F1
:10E10800EF10903BD1471DC51767FB1F034717F357
:10E118009767FB1F83C757F2014999E03E89BA8781
:10E12800131749001764FB1F032444F03A94636DE6
:10E13800F900D547F2406244D2444249B249224AE2
:10E14800924A3E850561828036201307040191C6F4
:10E1580005091379F90F3A84D9BFB1C89565938534
:10E1680025C0130500029720FB1FE780A0EE48C4D6
:10E1780069D1130600028145130909049720FB1F82
:10E18800E7804023230004002311240123134401C2
:10E198009C341767FB1F0327A7E9998C1CA45C44D0
:10E1A80091849180C4AF23A08900814761B7232659
:10E1B8000400230004002313440123045401E5B799
:10E1C80085473E858280AA869765FB1F83C515E72C
:10E1D8001767FB1F032787E581476394F50001450F
:10E1E800828032233A8519C2E30CD6FE850793F75D
:10E1F800F70F4107DDB7AA861766FB1F034616E42B
:10E208001767FB1F032787E281476314F600014560
:10E2180082802E233A8581C54C23E38BD5FE850762
:10E2280093F7F70F4107D5B7AA869765FB1F83C5F4
:10E23800C5E01767FB1F0327A7DF81476394F50035
:10E248000145828012233A8519C2E30CD6FE850760
:10E2580093F7F70F4107DDB7AA861768FB1F034836
:10E26800B8DD9767FB1F83A767DC01476314E800E5
:10E2780001458280B2233E8509CAF2236317D6007E
:10E28800D04701C63222E306B6FE05071377F70F1B
:10E29800C107E9BF411126C2444522C406C62A84E3
:10E2A80095C0C84409C59720FB1FE780C0E7C84848
:10E2B80009C59720FB1FE78000E726859720FB1FED
:10E2C800E78060E62285414681459720FB1FE7806D
:10E2D800600EFD571CB4B240224492444101828032
:10E2E800011122CC2A842A2106CE2EC6EF102069DD
:10E2F800324622858145EF00505822856244F2401B
:10E3080005616FF03FF905C53E21411122C406C6DB
:10E318002A8491CBDD45EF00505922852244B24032
:10E3280041016FF03FF7B240224441018280828070
:10E33800411122C4B1471304C5FFB307F40226C232
:10E348009764FB1F9384C40A06C6A697BA27631569
:10E35800B702C84315C19307F00F6305F6001C21E7
:10E36800639CC7009720FB1FE780E0DBB1473304BD
:10E37800F402A29423A20400B24022449244410130
:10E388008280411122C42E8426C24946AA8481452E
:10E39800228506C69720FB1FE780C0018DCCD82CAC
:10E3A8009767FB1F83A7C7C81207BA979A231AA0B3
:10E3B800BA23FE233AA01767FB1F0357A7C75AA023
:10E3C8009A207AA0BA201AA4DA203AA4FA205AA4E9
:10E3D8009A241EA87AA4B240224492444101828021
:10E3E8002A869765FB1F83C575C51768FB1F032819
:10E3F80028C49766FB1F83A666C30147014563933C
:10E40800E50082809C2281CFDC4691CBDC2F9207ED
:10E41800C2976316F6009307150013F5F70F050763
:10E428001377F70FC106E1BF130600643386C502F0
:10E4380093069500AA8517050000130505ED6F6082
:10E448002F9D411122C406C62A840835EF600FBAF1
:10E45800FD571CB4B240224441018280011122CCF4
:10E468004AC84EC652C456C25AC006CE26CA2A89BF
:10E47800AE890144176AFB1F130A1ABC976AFB1F6F
:10E48800938ACABA1D4B83470A006369F404639DE3
:10E4980009029769FB1F938979BA176AFB1F130A48
:10E4A800EAB8930AF00F83C709006364F4061144BD
:10E4B800A14422851306F00FCA850504EFF05FE733
:10E4C80033440408E31794FEF2406244D2444249BC
:10E4D800B249224A924A024B0561828083A40A000B
:10E4E80093174400BE949C208DC3FE20639F270190
:10E4F80063956901AA20EF10804826854E868145DC
:10E50800EF00B0372685EFF0FFD805041374F40F39
:10E518009DBF83240A0093174400BE949C208DC39A
:10E528009C34638F5701FE20639C27012685EFF0FA
:10E538005FF12685D145EF0050372685EFF09FD54E
:10E5480005041374F40F85B7C167F917630BF50257
:10E55800411122C406C685472A846399F50022859D
:10E568002244B240814541016FF05FEF89476396CD
:10E57800F5008545EF1040747DD1B2402244410139
:10E58800828082809D456FF07FED1765FB1F0355E4
:10E5980065AA8280011106CE68876C861767FB1F03
:10E5A800034787A985476318F70070009305E100C2
:10E5B8000545EF509026F24005618280A947631D0A
:10E5C800F6029C319821A207D98F1EA1BC31B8212F
:10E5D800A207D98F3EA1DC31D821A207D98F5EA12D
:10E5E800FC31F821A207D98F7EA19C359825A20776
:10E5F800D98F1EA501458280054582809147631EFB
:10E60800F6009C319821A207D98F1EA1BC31B821F0
:10E61800A207D98F3EA10145828005458280938754
:10E62800C5FF0D47B3C60708636ED7003147338768
:10E63800E7029767FB1F9387A7DBBA97A8A38EA368
:10E648000145828009458280930740203355F50AA9
:10E6580071159767FB1F239FA79C9767FB1F238F45
:10E66800B79C9767FB1FA38AB79C82809565411169
:10E678001905938535C006C6334505089720FB1F45
:10E68800E780409D01C9B240E95541011723FB1FAE
:10E698006700E3B6B240410182809767FB1FA38FF2
:10E6A80007989767FB1F238B07989767FB1F23869D
:10E6B80007989767FB1FA38107989767FB1F238D10
:10E6C8000796854741111767FB1FA306F79606C6ED
:10E6D80022C426C22A849767FB1F238E0794976754
:10E6E800FB1F239907949767FB1F23A10794EF103B
:10E6F800E0311765FB1F1305A5CF130600038145FD
:10E708009767FB1F238D87929720FB1FE78080CA9E
:10E718001764FB1F1304049108209764FB1F93845C
:10E72800B4911DC99565938545C012059720FB1FB7
:10E73800E78040921767FB1F232CA78E11CD1C3052
:10E74800102081459CA09767FB1F2388C78E12065F
:10E758009720FB1FE78000C69C201765FB1F034519
:10E7680025D11764FB1F1304748D3E951375F50F9F
:10E77800956508A0938555C012059720FB1FE78073
:10E78800608D9764FB1F9384648A88C035CD102000
:10E79800814512069720FB1FE780C0C198401420CE
:10E7A800814725077D56639BF604EF106047B14704
:10E7B8003305F5029565938565C0334505089720AF
:10E7C800FB1FE78020899767FB1F23AFA7842A8454
:10E7D80001CDEF10E04431463306C502814522855C
:10E7E8009720FB1FE78000BD2244B24092441705E2
:10E7F80000001305A5D541016F102043850710A31C
:10E8080093F7F70F410745B79767FB1FA388078260
:10E818009767FB1FA382078249BF411126C206C61C
:10E8280022C44AC0AE849397556063DB0708176912
:10E83800FB1F1309C980034509009720FB1FE780C8
:10E8480020A72A8421C91821930700096311F70416
:10E858001831CD476314F7069756FB1F9386067E3B
:10E8680028219C221768FB1F0348788F1306640031
:10E87800814501476318E50291C19CA29C2281CB86
:10E888000345090085459740FB1FE78080172285CF
:10E89800EF509F971395F468B2402244924402497E
:10E8A800410182800E2205071377F70FAE9793F781
:10E8B800F70F09068545B3D7070B6DBF0123C1BF05
:10E8C80013F5150071D9EF00105319CD9757FB1F99
:10E8D80083C7C77691CB85451755FB1F034525761A
:10E8E8009740FB1FE780E01113C5140075B7054773
:10E8F800637EC7029C319421A207D58F1EA163991C
:10E90800E700BC31B821A207D98F3EA1014582801A
:10E918000947E39DE7FEBC31B821A207D98F3EA184
:10E92800DC31D821A207D98F5EA1CDB705458280F9
:10E938009147631EF6009C319821A207D98F1EA12A
:10E94800BC31B821A207D98F3EA101458280054577
:10E9580082809147631EF6009C319821A207D98FC7
:10E968001EA1BC31B821A207D98F3EA101458280E2
:10E9780005458280A1476318F6029C319821A207B9
:10E98800D98F1EA1BC31B821A207D98F3EA1DC3195
:10E99800D821A207D98F5EA1FC31F821A207D98F0F
:10E9A8007EA1014582800545828089476319F6006A
:10E9B8009C319821A207D98F1EA101458280054567
:10E9C80082803E2279714ECE06D622D426D24AD0F3
:10E9D8001307F007AE896371F70209473AC47C86CA
:10E9E800300093F5F50FEF007078B250225492542E
:10E9F8000259F249456182805A22D9462A893284CD
:10EA080063F7E6007E2263F4F6006379F7002314C7
:10EA18000100300093F5F90F4A85F1B70A2202C4C4
:10EA2800EFF09F80AA8435C5EFF09F9B9C24636913
:10EA3800F5001146A246CE854A85EF00F06975B704
:10EA4800340026869305F00F4A85EFF0AFE975F19B
:10EA5800A2471A24DC479AA33A20BAA35A20DAA379
:10EA68007A20FAA3DA209AA7DC4495C793F4F90F21
:10EA78002286A6854A858297C167FD172A86E31BE9
:10EA8800F5FA22459947F9451CA144A1EFF0DF9911
:10EA9800A9BF094645B7014671BFA947631DF602DC
:10EAA8009C319821A207D98F1EA1BC31B821A20799
:10EAB800D98F3EA1DC31D821A207D98F5EA1FC31C4
:10EAC800F821A207D98F7EA19C359825A207D98F56
:10EAD8001EA501458280054582809C211CA19C3190
:10EAE8001CB1BC31B821A207D98F3EA18280232254
:10EAF8000500D82189476304F70005458280F6217F
:10EB080001114EC606CE22CC26CA4AC80D47AE8988
:10EB18006379D7049C4584339023A033A204D18C15
:10EB2800B023220493874400518C639CD702930737
:10EB3800C4FF2A89B3C707086361F70203A58900E0
:10EB48002311990023108900F1559710FB1FE780C6
:10EB5800006B2322A900014531A02285EFF0AFE622
:10EB680071FD0545F2406244D2444249B24905610B
:10EB78008280797122D426D22E8406D64AD01C20CF
:10EB88001947AA84B2856390E70630202800EFF081
:10EB98003FDA0DE92884EFF00FE30C302A890DC91C
:10EBA8002E86171700001307E7D134009D452685E8
:10EBB800EF00D0304A8509468145C1214A85EFF0EA
:10EBC8006FED0145B250225492540259456182803A
:10EBD80089477C803C840A867C813C857C822685AA
:10EBE800EF00D058F9BF49476395E7023220280063
:10EBF800EFF05FD861F91755FB1F1305657F5E2598
:10EC0800E9D3183068253C00C9460146A685DD2CA5
:10EC18004DBF5147639DE70032202800EFF01F9A4F
:10EC280055F10C3030002685EFF0BFD959BF594750
:10EC3800639CE70432202800EFF05F9C41F52C84A8
:10EC48002685EFF06FE115C9584534851E23B69720
:10EC5800B3C707081EA3B5D75C47A5D79757FB1FAF
:10EC680083C7C73DB9DF85451755FB1F0345253DBC
:10EC78009740FB1FE780E0D8A9B789473EC03C848E
:10EC88000C300A867C82A1BF0C30231001000A8652
:10EC980081BF5D71A2C456DA86C6A6C2CAC04EDE5E
:10ECA80052DCAA8A88312E8432C6EFF0CFD4B2451E
:10ECB80001ED0144B6402285264496440649F2599E
:10ECC800625AD25A6161828023020500231105002D
:10ECD800834904008547AA846399F90030202808ED
:10ECE800EFF0FFC02A8405491DA09D476391F904F0
:10ECF80018218D47E31FF7FA302028080549EFF05F
:10ED08005FC52A8409E5054681452685BD262685F1
:10ED1800EFF02FF388243C080147CE862286D6855B
:10ED2800D522E30909F82685EFF0CFD661B7CD479C
:10ED3800639BF90018219147E31DF7F63020280856
:10ED4800EFF0BFC645B7D547E395F9F6034A050086
:10ED58008947E310FAF6302028080549EFF0FFD379
:10ED68002A8455F583570102A1EBB8841306F003F2
:10ED7800DC44930607FCB3C60608636AD600B08570
:10ED8800D94663F6C600B486D94563EDD500BAA363
:10ED98000145EF00D03E054903560102D28526857C
:10EDA800AD2CB5B7AC87BAA3D2A38EA3F6A385477B
:10EDB8009CA0014A0149CDB7014AF9BF7971AA85DA
:10EDC80022D426D22221AA84280806D64AD0EFF0D7
:10EDD8001FD2F24599E53DE185452285EFF08FFB8D
:10EDE80075A0BC8415476395E706B8858D4763F71A
:10EDF800E7046800EFF07FCE0359E100DD4763FBCD
:10EE080027018C86B70717008507100822853EC89A
:10EE1800EF00D035BC851109638527012285EFF005
:10EE28006FF61C8672466C00858B1106228591CF81
:10EE3800EFF03FE601C52285EFF0CFF4884449DDC5
:10EE48009710FB1FE780202E41BFEFF09FD2DDB760
:10EE580011476389E7001387A7FF854633470708EB
:10EE680063ECE6023147F117B387E7021757FB1F38
:10EE780013070758BA979A2371D3A8233008A28595
:10EE88000D204DFDB8849147E318F7F4B250225491
:10EE980092540259456182802C082285212E59FD01
:10EEA800F5B701114AC82A89314526CA4EC606CE89
:10EEB80022CCAE89B2849710FB1FE780603929C144
:10EEC8009307000A231135011EA12A842146110542
:10EED80095C0A6859710FB1FE7804047A2854A8505
:10EEE800EF50AFB70145F2406244D2444249B249BB
:10EEF8000561828081459710FB1FE780A04BF9BF11
:10EF08000545D5B701114AC82A891305000226CA42
:10EF18004EC652C456C25AC006CE22CCAE8A328BD6
:10EF2800B6893A8ABE849710FB1FE780603221C9F0
:10EF3800930720FA1CA1A3006501231155012302A0
:10EF48004501A30235012A84614621059DC0A68595
:10EF58009710FB1FE780803FA2856244F240D244AD
:10EF6800B249224A924A024B4A85424905616F508A
:10EF7800CFAE81459710FB1FE780C043F1BFF24039
:10EF88006244D2444249B249224A924A024B05613C
:10EF980082805C45797122D406D62A84AE86A5C7BC
:10EFA800BA23F885130720066396E504FA23175653
:10EFB800FB1F035626083357C70AB22B9E2B13771D
:10EFC800F70F918F93F7F70F01E6890793F7F70F7C
:10EFD800BA97FD17B3C7E702FC863E206E200824C7
:10EFE800FC8401473C080146EFF0DFF1B25022549F
:10EFF80045618280D82F9757FB1F83A767031207A5
:10F00800BA97FE23D1BF2EC6194681452808971006
:10F01800FB1FE780203AB246C9B7797122D406D6D9
:10F0280026D22A8491CD08242E866E202254B250EE
:10F038009254814701479306000645616FF09FECA3
:10F04800B284280059469710FB1FE780A0366484D5
:10F0580099E43E2048446C007C85EFF08FB26E2026
:10F0680008243C000147930600060146EFF09FE99B
:10F07800B2502254925445618280797106D68147F4
:10F0880099E53E2170867C845C4589EF3C002E869C
:10F098006E210825014793060006EFF0BFE6B2503F
:10F0A80045618280BE237C85D5B7411122C406C63E
:10F0B8001C2111472A846392E7022E866E210825B7
:10F0C80081470147CD46EFF0FFE349466E202244D1
:10F0D800B240154541016FF0AFA513F7B70F894648
:10F0E8006317D7000146EFF05FF35146C5B70D47E8
:10F0F8006398E7002244B240014641016FF0FFF7F0
:10F10800B2402244410182809A21B14771173307E6
:10F11800F7029757FB1F9387A72DBA97D84301EBA0
:10F12800D841AAA70145D8C3BA219AA782805945D0
:10F138008280797126D2444522D44AD006D62A84C0
:10F148002E89B1C4C84419C59710FB1FE780A0FDDC
:10F1580023A604009E206E2008247C85BE2001473B
:10F16800930640067C869E244A867C879C483EC837
:10F178003E207C843C00EFF0FFD8A38E240123A816
:10F188000400B250225492540259456182802800EA
:10F19800314681459710FB1FE780C0213E206E2035
:10F1A80008247C8401473C00930640064A86EFF019
:10F1B8007FD5C1BF797152CC2A8A8A2126D206D638
:10F1C80022D44AD04ECE56CAAE84EFE0DFFF6302A7
:10F1D800051240452A89630E04107E21639B47115E
:10F1E8001E24638A0710542C975AFB1F938A4AE4FB
:10F1F80003A70A009206FD1736977A23B3C70708B4
:10F208001EA46316F70093053006EFF09FD85C48FC
:10F21800B5EBC840834915001C21A209B3E9F900E0
:10F22800BE2013872900631AF702F9559710FB1FB0
:10F23800E780E0FCC8C02391340103458900268695
:10F24800D285EFF01FC61DEDB250225492540259D8
:10F25800F249624AD24A456182809565938515C014
:10F268004E859710FB1FE780E0DE48C8C840231C86
:10F278003401F9559710FB1FE78060F8BE20C8C01D
:10F28800F917BEA048482DCDB220362C1E2C3308C5
:10F29800D60063C90707582C83A70A0095451207AB
:10F2A800BA97BE2363CA0705CC4036959710FB1F53
:10F2B800E780C0093A2CBE20BA971A2CB3C70708B2
:10F2C8003EAC6398E70203572900034589003000E4
:10F2D80078845848D2857C853AC6EFF09FBC11C522
:10F2E80048489710FB1FE78000E4232A0400232CDA
:10F2F8000400054591BF99454A85EFE07FFED5BFDB
:10F30800A545DDBF9145CDBFBE21F9C3011126CA70
:10F3180006CE22CC1757FB1F0357C7D1AA846D45C9
:10F328006363F70A2E84484091459710FB1FE780D6
:10F3380000ED3E20AA861CA13E20A1831CB11E2000
:10F348003CA11E20A1833CB13220C167F9171106E8
:10F3580033460608639FF4022AC4314532C6971023
:10F36800FB1FE780E0EEAA854D45B1CD930700F974
:10F378003246A2469CA1F957BEA18947DCA1F2A159
:10F3880094C51755FB1F034585CBEF401FED01457D
:10F398001DA881452685EF40F05C11E91757FB1F32
:10F3A8001307C7C91C23E5D7FD171CA3CDB7894789
:10F3B8006302F5029D476301F502C9476300F50240
:10F3C800FD47E30DF5FCF2406244D24405618280BA
:10F3D8006D4582805145C5BF1145F5B70945E5B76B
:10F3E800011122CC4AC831441309C5FF33048902EC
:10F3F80026CA9754FB1F9384A4FF06CE26945C402C
:10F40800A9C31757FB1F034767C30DC768843EC6C8
:10F418002A241E242C007C85EFF01FEF11C54840DC
:10F428009710FB1FE78020D0B1473309F902CA942F
:10F4380023A204000545F2406244D24442490561D2
:10F4480082800145CDBF797126D244454ECE52CC3B
:10F45800FE20BA289759FB1F83D9C9BD06D622D4E6
:10F468004AD056CAB3D9F90A2A8A9E282DCF998F2D
:10F478004E8463D4370133C4070889452285EFF0E9
:10F48800EF9E2A89CD4A31C5BE202AC660857C8474
:10F49800BE2899EB9E28130925001CA19E28A1834C
:10F4A8001CB1637434058228BE28CC4422864A8560
:10F4B800BE959710FB1FE78060E903556A002C0092
:10F4C800EFF09FE4AA8A15C54A859710FB1FE780CD
:10F4D80080C5B250225492540259F249624A568564
:10F4E800D24A45618280890761B779143344040898
:10F4F80065BFBA289E203A949A28FD17B3C7070813
:10F50800334404089EA0A2A86376E400F9F3FD57EB
:10F51800DCBCC1B781455285EFF0BFC15DBF7971D1
:10F5280022D44ECE56CA5AC85EC662C406D626D261
:10F538004AD052CC9759FB1F9389E9AF03CA0900F7
:10F54800975AFB1F938A8AAE054B5284930BF00F90
:10F55800175CFB1F130C5CAE83A40A0093174400CE
:10F56800BE9403C90400631D6907DC44B5CBD847C2
:10F5780025CB9A2339CB9757FB1F83C727AC99CF45
:10F588002685EFF05FECAA8505ED05049757FB1F6C
:10F5980083C797AA6351F40223808900B25022548A
:10F5A8009254F249624AD24A424BB24B224C4A85A3
:10F5B8000259456182809757FB1F238E07A6F9BF22
:10F5C8002685EFF01FB70149D1BFDC3F639A770169
:10F5D800930520062685EFF0DF9BDC44A38E070009
:10F5E80083470C0005041374F40F6363F4000144AB
:10F5F800E31444F7C9BF4111154506C6EFF05FDEB5
:10F6080009C50545B240410182801945EFF05FDD2B
:10F618006DF91145EFF0DFDC6DF51D45EFF05FDCAE
:10F628006DF11755FB1F034535A169DDB240410156
:10F638006FF0FFEE9E210D47F117B3C7070863630C
:10F64800F706DC41411122C406C626C22E84A9CF82
:10F658008545AA84952539CD2685AD2BC167F9172F
:10F66800638FF40009ED3E2099CB16201947639566
:10F67800E6041757FB1F0357E79B63FFE7029757FB
:10F68800FB1F83C7A79BA285268599C72244B24042
:10F69800924441016FF05FC72244B2409244410155
:10F6A8006FF09FA6094582800945B24022449244E2
:10F6B800410182805145D5BF6D45C5BF797126D2BC
:10F6C80052CCAA842E8A5D4589454AD04ECE56CA68
:10F6D80006D622D4B289B68A3A89EFE03FF925C521
:10F6E8002A84014563060900D6851305440002995A
:10F6F800935785003CB093074500230044017C855F
:10F70800954728A07C84A300340122C69757FB1F85
:10F7180083C7C7922C00268585C7EFF0FFBEAA8451
:10F7280011C522859710FB1FE780E09FB250225435
:10F738000259F249624AD24A26859254456182802A
:10F74800EFF09F9CE9BFCD44D5B7797126D24AD056
:10F7580052CC56CA2E8906D6BE8522D44ECE99479B
:10F76800B284368ABA8A6314F9062A220944EFE079
:10F778009FA52AC625C55C4583596500BE239EA062
:10F78800B247154723805701BAA31757FB1F130722
:10F79800978A10239305160093F5F50F0CA3D0A3B1
:10F7A80099E1854614A351476317E9001547BAA0A4
:10F7B800DC479A249AA75287A686CA854E85EFF019
:10F7C800FFEF2A8432450DC4EFE0DFAC01A8428682
:10F7D8007400AA89EFE01F912A845DD1B250228576
:10F7E800225492540259F249624AD24A45618280AF
:10F7F800F945EFE07FC3DDB79E211CA19E21A183BF
:10F808001CB1BE213CA1BE21A1833CB1114582801F
:10F818009E211CA19E21A1831CB1BE213CA1BE2119
:10F82800A1833CB1DE215CA1DE21A1835CB1FE2174
:10F838007CA1FE21A1837CB1214582809E211CA14F
:10F848009E21A1831CB1094582809E211CA19E2175
:10F85800A1831CB1BE213CA1BE21A1833CB1DE2104
:10F868005CA1DE21A1835CB1FE217CA1FE21A183E4
:10F878007CB19E251CA59E25A1831CB529458280A7
:10F888009A218546AA8718A19A21218318B19A211D
:10F898006319D700BA2138A1BA21218338B111459B
:10F8A80082800945631DA700BA211945B8A3BA216A
:10F8B8002183B8B3DA21D8A3DA212183D8B382808F
:10F8C8009E211CA19E21A1831CB1BE213CA1BE2169
:10F8D800A1833CB111458280797126D24AD04ECE9F
:10F8E800B2842A89AE8929468145480022D406D6A1
:10F8F80036849710FB1FE780E0AB64868DE43E20DA
:10F908007C829747FB1F83D7E7727C845C4481CF56
:10F91800D42F1747FB1F0327A7719E2792063697F8
:10F928003A237C8578834A8517070000130727F256
:10F93800540013F6F90FD545EFF05FD82A8911C1A5
:10F9480095E085471CA023020400014681452285D5
:10F95800EFF0AFECB25022549254F2494A85025962
:10F96800456182802285EFE0FF92EDB7B2861707E6
:10F978000000130727F12E8685456FF03FD401114B
:10F9880068874165700001489307F00F0D47970697
:10F9980000009386A6E699457D1506CEEFF0FFDABE
:10F9A800F24005618280B28701482E86114797068A
:10F9B8000000938626E6C9456FF03FD9B28617073F
:10F9C80000001307E7E72E86CD456FF03FCF011102
:10F9D80022CC26CA4AC84EC606CEAA842E891754F7
:10F9E800FB1F1304E4A39759FB1F938969A61C40C6
:10F9F80081C7CA85268582971104E31A34FFF2402D
:10FA08006244D2444249B24905618280411122C40C
:10FA180006C626C21747FB1F130787737C2B783B44
:10FA28001754FB1F130444A41CB4BA9793F7F70F99
:10FA38001CA4A5CB1305C0033385A702A5658505BE
:10FA48009744FB1F9384C45F9700FB1FE780806087
:10FA580010249307C00381453306F60288C0971027
:10FA6800FB1FE780209514249C4001477D56634185
:10FA7800D7022244B2409244130600038145175529
:10FA8800FB1F1305E59941011713FB1F67008392BC
:10FA9800B2A32382070023A6070205079387C7039B
:10FAA800F9B7B2402244924441018280411122C4F4
:10FAB80026C24AC006C62A892E84B2849730FB1F04
:10FAC800E780E00A09EDC167F91751456313F900AA
:10FAD8000145B24022449244024941018280545572
:10FAE8005C2195C213F727014146630BC700C18B00
:10FAF8003D45E5D3BC2E0145E3FD87FC3145D1BF2B
:10FB08001545F5D4F9B7C18B0145E1F71545D1B7CE
:10FB180079714AD0416922D426D24ECE52CC56CAE7
:10FB28005AC806D6AA8401449759FB1F9389C993DA
:10FB3800174AFB1F130ACA50930AC0037D19054BC5
:10FB480083C789006364F400014525A8330754037B
:10FB580083270A00BA97BA2363162701050413748A
:10FB6800F40FF9BFC833300093856700EFB09128D0
:10FB78001946A68528009710FB1FE780A08EE31F73
:10FB880065FDB250225492540259F249624AD24A4F
:10FB9800424B456182804166AA869755FB1F83C503
:10FBA800258D1747FB1F0327A74981477D166394B7
:10FBB800F50001458280035827003A856306C8008E
:10FBC80003480700E308D8FE850793F7F70F1307E4
:10FBD800C703F1BF411106C69730FB1FE78020F924
:10FBE80009C54A29B240410182800145E5BF17474E
:10FBF800FB1F0327E7449756FB1F83C66687110739
:10FC0800814701456393F6008280102301C60505EC
:10FC18001375F50F850793F7F70F1307C703DDB7BC
:10FC28001755FB1F0345C58482801747FB1F130721
:10FC3800277F81473A86B1460C4391E5B3C7C72071
:10FC480088C30145828085071107E397D7FE4D4594
:10FC58008280411106C622C49730FB1FE78020F13D
:10FC68000DCD2A842A218545EFF07FD6485409C551
:10FC78009700FB1FE780204B22851306C0038145B0
:10FC88009700FB1FE7800073FD573EA02302040086
:10FC98000145B2402244410182800945DDBF41113E
:10FCA80006C69730FB1FE78080EC09C54825B2409F
:10FCB800410182800145E5BFC167F9176305F50277
:10FCC800411122C406C62E849730FB1FE78020EA24
:10FCD800AA87014589C7DC237D8C33358000B24073
:10FCE80022444101828005458280411122C406C612
:10FCF8002E849730FB1FE78080E701CD5A29AA8719
:10FD0800054563048700C2AB0145B2402244410166
:10FD180082800545DDBF39CD01114AC8416922CC31
:10FD280026CA4EC652C456C206CEAA840144974972
:10FD3800FB1F93896973174AFB1F130A6A30930ADA
:10FD4800C0037D1983C78900634BF400F240624405
:10FD5800D2444249B249224A924A05618280B30795
:10FD6800540303250A003E953E21638327018294AC
:10FD78000504C9BF82809747FB1F83A7672CC1660C
:10FD88001746FB1F0346C66E890701450147FD1646
:10FD980091456313E600828003D807006309D80001
:10FDA80003C8A7006315B80005051375F50F050707
:10FDB8001377F70F9387C703E9BF9746FB1F83A6FF
:10FDC80026281746FB1F0346A66A91060147814766
:10FDD800631FE600858393C7F7FF0545B3C7070888
:10FDE8006361E5023315A0283345050882808C221B
:10FDF80099C1CE36CD8F05071377F70F9386C603C3
:10FE0800C1BF93F61700F9FE050585831375F50F35
:10FE1800C1BF797156CAAA8A2E8526D24AD04ECE3B
:10FE280052CC5AC85EC662C406D622D4AE84328B7F
:10FE3800368CBA8B3E8AC28946899730FB1FE78089
:10FE480000D33DED41657D159730FB1FE78020D23B
:10FE58002A84554531C81946DE8513056400A30276
:10FE680084019700FB1FE780604E8357010326A09B
:10FE7800230264013EA8835741032300540123262B
:10FE880004025EA823064401231734012318240121
:10FE9800EFF0BFF20AB8232A04022685232C0402B5
:10FEA8008145EFF0DFB20145B25022549254025915
:10FEB800F249624AD24A424BB24B224C4561828097
:10FEC8004545DDB79746FB1F83C6865A1747FB1F74
:10FED8000327071781476395F60041657D158280E2
:10FEE8000E3B1306C7036394A5002A238280850767
:10FEF80093F7F70F3287C5B741661748FB1F0348CA
:10FF080028579746FB1F83A6A61301477D169548D9
:10FF180011436314E80001458280BE223685638E52
:10FF2800C702CC5A9DC9BC31AC2189CD938597FDB8
:10FF380093F5F50FE372B3FE9387D7FA93F7D70FCC
:10FF480089EF82809385F7FD93F5F50FE3F6B8FC0A
:10FF58009387D7FA93F7D70FE1D305071377F70FEE
:10FF68009386C6037DB741669745FB1F83C54550F9
:10FF78001747FB1F0327C70C81477D162548639445
:10FF8800F5000145828036233A85638BC600545BB1
:10FF980081CAB4329386E6FD93F6F60FE374D8FE71
:10FFA800850793F7F70F1307C703D1BF011122CCB9
:10FFB8002A84494506CEEF609FD61DC12AC62285F0
:10FFC8009730FB1FE780A0BA01CD624432460E3954
:10FFD800F2401745FB1F0345554905616F400FCE99
:10FFE800F24062440561828079714ECE52CCAE896E
:08FFF8002A8A930530054145FA
:020000025000AC
:1000000026D24AD056CA5AC806D622D4328B36894E
:10001000BA8A9700FB1FE7806004CD4429C92A846F
:100020008944638109044146814523126101970097
:10003000FB1FE780A0385686CE8522859700FB1FE0
:10004000E78040312146630F0902CA8528009700E6
:10005000FB1FE7802030A28650002C005285EF4025
:100060000000AA8422859700FB1FE780400CB25055
:1000700022540259F249624AD24A424B268592548E
:1000800045618280814528009700FB1FE78000338F
:10009000D9B7411122C4405926C206C6AA8429CC28
:1000A000085409C59700FB1FE7806008285809C558
:1000B0009700FB1FE780A007685809C59700FB1F42
:1000C000E780E006285C09C59700FB1FE780200653
:1000D000685C09C59700FB1FE780600503250408DD
:1000E00009C59700FB1FE780800422859700FB1F4E
:1000F000E780E00323AA040222448E38B2409244EF
:100100001745FB1F0345F53641016F400FE54111CF
:1001100026C206C622C4AE849730FB1FE780A0A586
:1001200031C9032345032A84630603048328C307D4
:1001300003288307832743070327030783466300B6
:1001400003560300834523002685EF60DFC5228523
:10015000EFF03FF4EFF0BFE111CD2244B240924402
:100160001745FB1F0345F530854541011733FB1F3C
:100170006700A389B2402244924441018280411128
:1001800022C426C206C6AA842E849730FB1FE780AD
:10019000809E5C5989CF9E23639B97008547631897
:1001A000F4002244B240924441016FF09FEEB2400D
:1001B0002244924441018280411106C622C426C2D3
:1001C000EFF01FD429C144592A8495CCBC209DC787
:1001D0009747FB1F83A7C7E789C7DC4399C32685D9
:1001E0008297B8309307F002631FF7002A20224459
:1001F000B2409244814541016FF07FF19747FB1F68
:1002000083A7C7E4D1BFB240224492444101828017
:10021000411126C24AC006C622C4AA842E8997303C
:10022000FB1FE780409505CD405955C41E206394BF
:10023000970A3C30130710026395E7083C20ADCFC6
:100240007C5403270408DE2B15E313F7170019CF9E
:1002500018545A23058B19CB930720023CB0B240A7
:1002600022449244024905454101828013F7270048
:1002700001CB18545A23098B01C793074002F9BFD9
:10028000918B81CB1C54DE23918B81C79307600235
:10029000F1B79747FB1F83A7A7DBF1D3DC43E1D37B
:1002A0002285829738309307F0028145E319F7FAE7
:1002B0002685EFF0DFE565B79747FB1F83A707D9D2
:1002C000E9BF1307A0026398E7006304090013095C
:1002D0002003CA85F1BF631C090026859730FB1FE8
:1002E000E780608909C55C2193E707015CA1A685C9
:1002F0004A85EF600FBBA5B7011126CA99476C85E7
:10030000AA842E858D4522CC4AC806CE32893684F1
:100310007C84EFE02FB62AC61DC9AA854A850294BF
:100320002A8419E52C002685EFF04FB12A8411C5E7
:1003300032459700FB1FE78080DF2685EFF09FC7DF
:10034000F24022856244D2444249056182804D4494
:10035000EDB7411122C42E862E8497160000938695
:10036000667B894506C626C24AC02A89EFF0DFF8B7
:100370000C20AA844A85EFF09FD9B240224402495A
:1003800026859244410182809747FB1F83A707CCB3
:1003900085CB9C4395C71D71A2CC86CE9841100891
:1003A0002A843AC8D84185453ACA829711C54886F9
:1003B0002A206C00EFF0FFF9F64066442561828048
:1003C0008280AA872E8591CFFC5781CF982398A150
:1003D000983398B1B82BB8A1982FDC4BB8B1DCC1D9
:1003E0008280414681451703FB1F670023FD974725
:1003F000FB1F83A7E7C581C79C4791C38287094537
:1004000082801747FB1F032727CB1DC75843AA87A6
:1004100005450DC703A50708411106C69306050249
:100420001306050C93050506130505040297B24053
:100430001375F50F410182800545828082804DC988
:10044000357122CD2A840A2126CB52C556C35AC102
:1004500006CF4AC94EC7DEDE2E8AB28A368B972077
:10046000FB1FE7804071AA8431C50C182285EFF08C
:100470005FF53C20938B6400A9CBEF503FFC2A89A9
:10048000014583C95400EF50FFF8AA840C100818E6
:10049000EF10804A08542C10EF10A04ADE88A68B7B
:1004A0005AC04E88DE874A8714103010D685528590
:1004B000EF200076FA406A44DA444A49BA492A4AA7
:1004C0009A4A0A4BF65B0D618280EF503FF7AA898A
:1004D000014503C95400EF50FFF32ACE08540C1015
:1004E000EF1080452C100818EF10A045F2484DBFC2
:1004F0008280AA8701CD1855414511CBFC5781CB8D
:1005000028333D476375A700882F8280414582804C
:100510006DC5411122C406C626C2AA872E8409458C
:10052000E1C998337D761306F67F98A1B8234D452F
:1005300098B1B833B8A1D823B8B1D433DA21858AB9
:10054000A2061377F7EF558FDAA1D43333470708A4
:100550001377F7DF93D61648A606558FDAA1D43362
:10056000334707081377F7BF93D62648AA06558F57
:10057000DAA1D43333470708718F93D63648AE06D5
:10058000558FDAA1F42333470708799B858A558F65
:10059000DAA1F42333470708759B898A558FDAA1BE
:1005A000F423334707086D9B918A558FDAA1F8230E
:1005B000DE21218BDD9BD98FDEA1EF60CFF6AA84EF
:1005C0005145EF604FF6383093F4F40FAA87494550
:1005D0006360970293F7F70F63ECE70018209147E9
:1005E000614563E7E7001830854763E3E7000145AD
:1005F000B24022449244410182800945828015C55F
:100600002A87AE87094585C5411106C6143313856F
:100610001700194694A1930527009700FB1FE78058
:1006200060D3B240014541018280094582808280C9
:100630000DC9AA872E8709459DC5411106C6B42359
:10064000903313052700A206D18E96A121469385EB
:1006500037009700FB1FE780E0CFB2400145410122
:1006600082800945828082801DC12A87AE87094524
:100670008DC141113E8541469305170006C697007E
:10068000FB1FE78020CDB240014541018280094532
:1006900082808280AA87094591CB89C99C333D47D6
:1006A00061456365F7009CA101458280828005C594
:1006B0002A87AE87094595C141113E85130600047E
:1006C0009305170006C69700FB1FE780A0C8B2403D
:1006D0000145410182800945828082801D71A2CC42
:1006E0002A84084586CEA6CA230601000421354780
:1006F0009387F4FF93F7F70F6362F70A17D70100A8
:100700001307C76EB3C7E7209C43BA9782870C08CC
:10071000EFF01FE0C947631CF50499475C862A2067
:100720006C00EFF01FC3F6406644D644256182801A
:100730000C08EFF03FF61DED2A209720FB1FE78005
:100740008043A14705C15825631CF7041747FB1FC9
:10075000032707909D4719C7184309C71008A685A6
:100760000297AA875C8629A00C08EFF07FEC69D578
:100770001C86D5F72A20EFF0FF8375B70C08EFF041
:100780001FE8F5B71C312308F1007DB70C08EFF026
:100790001FF2F1BF0C08EFF03FEDD1BF9D47BDBF89
:1007A0001747FB1F0327878A75B7411122C406C666
:1007B00026C24AC01821930720092A84631AF71019
:1007C0001C3139476395E70A56210967610781475C
:1007D0006398E6089744FB1F9384C487884049C107
:1007E0000C4403C90500631D09001C218505214631
:1007F000B9CB29059700FB1FE780C0B59C40A5C376
:1008000049459700FB1FE78020A52A841DC1930757
:1008100010FC1CA1A30025018C4009054146890557
:100820009700FB1FE78000B39C40A2858833EF3020
:100830005FA388409700FB1FE780608F9747FB1FEF
:1008400023AA078029A809059700FB1FE78080B02D
:10085000EF30B00005495DF19C40238027018547BA
:10086000B2402244924402493E85410182801307EE
:10087000E003639DE706382195476319F7024A2193
:10088000EFF06FC29147E31CF5FC9737FB1F83A77E
:10089000E77BF1D79C47E1D772244A209305640097
:1008A0002244B2409244024941018287A147631B1E
:1008B000F7006C204A202244B24092440249410190
:1008C0006FF01F95930600038147E31BD7F8D5B758
:1008D0009306000A8147E315D7F8EFF03FE008449C
:1008E0003DDD9700FB1FE780808495BF81478DBF6A
:1008F000011122CC06CE26CA4AC8094415CDAE84C1
:1009000009449DC92A898D456800EF50BF841C8722
:1009100026866C0093F7F70393E707044A855C8704
:10092000EF2000262A8409E90D466C001385340067
:100930009700FB1FE78000A2F24022856244D24468
:100940004249056182805D714EDE86C6A2C4A6C2A0
:10095000CAC052DC56DA5AD85ED6894955C932899E
:1009600089495DC6138B45002A8AAE8A334B0B0832
:10097000930530055A8597F0FA1FE780206E2A8488
:10098000CD4959C5EF507FADAA845686D28593DAFA
:10099000840013DA040193FBF40F1305440093FA67
:1009A000FA0F137AFA0FE1809700FB1FE780C0B0BF
:1009B000A301740123015401A300440104A0EF50DA
:1009C0003FA9AA85414608089700FB1FE780C0AEF3
:1009D000214734005A86A2850808EF20E040AA8902
:1009E0001DE121462C0023007901A30059012301B8
:1009F0004901A3019900130549009700FB1FE780F7
:100A0000A0ABEF505FA6228597F0FA1FE780207217
:100A1000B640264496440649625AD25A425BB25BBB
:100A20004E85F25961618280411126C2AA842E85C9
:100A30004AC006C622C42E899720FB1FE780A01358
:100A400069C5405969C45C30094793F6B70F63879D
:100A5000E60011471305E00F6395E7081E200945DE
:100A600063912709130984004146A6854A859700AA
:100A7000FB1FE780208E4146A68513058401970061
:100A8000FB1FE780208D383085469307F7FE93F7EC
:100A9000F70F63EEF6049304C4039737FB1F83A795
:100AA000A761C14526858DC79C4F9DC3829793063C
:100AB000C4022686CA852285EFF07F983C2081CF2C
:100AC00022852244B2409244024941016F10C00C79
:100AD000EF504FE8E9BF3830C947E303F7FE3CB0B9
:100AE0000145B24022449244024941018280930769
:100AF0001005E317F7FE3C20E5D722852244B240DB
:100B00009244024941016F10600F0945D9BF494520
:100B1000C9BF797152CC2A8A328522D44AD04ECEAE
:100B200006D626D2AE8932899720FB1FE780A00423
:100B3000494405C9445949448DC49E206393270301
:100B4000DC30A18B85EB0944B8309307B005631AFC
:100B5000F7002685EF106007BC20ADCB9307C005DA
:100B6000BCB0B2502285225492540259F249624AD2
:100B7000456182801739FB1F130909548327090037
:100B80001304E00FF9DF9C47E9DF13848401228519
:100B90004146D28597F0FA1FE780C07B8327090082
:100BA00083A5040822869C47938505042E850A8721
:100BB000814682972A844146CE850A859700FB1F8D
:100BC000E780C08A49D11374F40FBDBF9307E005D5
:100BD00041BF39C9011122CC26CA06CEAA842E846F
:100BE000094595CD0D468D05280097F0FA1FE78041
:100BF00060761C8570002C0093F7F70393E70704D9
:100C000026855C85EF10D07719E90D46A28568002E
:100C10009700FB1FE78080857D153335A000F240EB
:100C20006244D2440561828009458280011152C428
:100C30002A8A32854EC656C25AC006CE22CC26CA51
:100C40004AC82E8BB28AB6899720FB1FE780A0F294
:100C500009ED8944F24062444249B249224A924A2B
:100C6000024B2685D244056182805C592A89C5449D
:100C7000F5F34D45EF602F8B1374F50F5145EF6081
:100C80008F8AE38809FC03C78901E36487FC9377B3
:100C9000F50FE3E0E7FC930530051305400897F0F6
:100CA000FA1FE780A03B232AA9022A84CD445DD104
:100CB00013064008814597F0FA1FE7802070A301D2
:100CC000040023014401230264012310540123265C
:100CD000340723240402A302040063070A002285C8
:100CE000EF00D065AA8419E18144ADB74A85EFF0E1
:100CF0004FBA8DB7397122DC06DE26DA4AD84ED6D5
:100D000052D456D25AD05ECE62CC66CA0944630A27
:100D10000610BA84094463060710AA8B2E89328B09
:100D2000368C9720FB1FE78000E5AA8A514475C9DD
:100D300093053005414597F0FA1FE7802032AA89D4
:100D40004D4465C198309C2003CA340022075D8F52
:100D5000BC20620AC207D98F336AFA0083A78A02CD
:100D600063E647017D5709446398E70A6307090072
:100D700083C74A000544898BC5C3214681450A853E
:100D800097F0FA1FE7808063930C4C0093053005C1
:100D9000B3CC0C08668597F0FA1FE780202C2A89CF
:100DA0004D443DC96286DA85110597F0FA1FE78048
:100DB000A0701146A6854A8597F0FA1FE780C06F9C
:100DC000414693858A014E8597F0FA1FE780C06EF1
:100DD00021478A866686CA854E85EF20E0002A84F0
:100DE0001DE521468A85280097F0FA1FE780C06C30
:100DF000214693854400280097F0FA1FE78000679A
:100E00008547631EF502D2855E85EF60AFAD4A85EA
:100E100097F0FA1FE780A0314E8597F0FA1FE78020
:100E20000031F25022856254D2544259B259225AAA
:100E3000925A025BF24B624CD24C21618280054493
:100E4000F9B7797122D406D626D24AD04ECE2E8456
:100E50009397556063D607049734FB1F93844461CE
:100E6000A83097F0FA1FE78020452AC609CDEFF099
:100E7000DF93B24511E5A8209307F00F631FF5003B
:100E80002E85EF30EFB81319F468B2502254925403
:100E9000F2494A85025945618280EF308FBCE5B73F
:100EA00013F9150063070900EFF00FB1134914009F
:100EB000E9BFE1DD854421A0850493F4F40FEFE060
:100EC000BFD6E3F4A4FCB3179028B3C90708E18F99
:100ED000E5D74E85EFE09FFFC167FD176305F5007D
:100EE000DD45EFF0CFA23349340145B79737FB1FFB
:100EF00023A207169737FB1F23AC07149737FB1F56
:100F000023A607149737FB1F9387C75517070000C1
:100F10001307475E98C3170700001307472FD8C36E
:100F200017F7FFFF1307070D98C79737FB1F938726
:100F3000A752171700001307C74698C317170000DA
:100F4000130747FFD8C3171700001307872A98C74E
:100F500082809737FB1F83C7E751A18B014789C761
:100F60001737FB1F130707509737FB1F23A2E70E06
:100F7000014582809737FB1F83C7C74F918B01477D
:100F800089C71737FB1F1307274D9737FB1F23AF61
:100F9000E70A01458280011106CE2AC6EFF01FF54F
:100FA000324599459737FB1FA385A74CEFD0AFE794
:100FB000F24017F5FFFF1305C51C05616FE07FC701
:100FC0001C5599C321458280411122C426C22A841E
:100FD000AE84130500049305300506C64AC097F099
:100FE000FA1FE780A00708D469C913060004A68584
:100FF00097F0FA1FE78000367454B82A9377870079
:10100000FDCB1C54BC23A18BFDC783270408D5E767
:10101000930530051305001097F0FA1FE7800004D0
:10102000AA872320A4080D45D1CB74549C30983254
:10103000C1CF3337E0000E07936707016C545CB0F3
:10104000B829058B19CB1854854638230D8B6316A8
:10105000D70078201367170078A00327040809C772
:1010600078201367870078A00547639FE70C130972
:101070008400414681454A8597F0FA1FE780003495
:10108000814513058401414697F0FA1FE78000333C
:101090009304C4039737FB1F83A70702C145268526
:1010A000B5CF9C4FA5CF829783270408BDCB22855F
:1010B000EF00D0349307000549C12145B2402244D6
:1010C0009244024941018280A1472DFBBC20918BB3
:1010D00091E7BC2A918B99E385478DB7982094229C
:1010E00095473307F70297D701009387A7D3BA979D
:1010F000B6979C23A1B79C3081C79032E1471DFE73
:10110000BC205D8F118B69DB9820954794223307B3
:10111000F70297D701009387A7D2D1BFEF508F83F3
:1011200061B722859306C4022686CA85EFF02FB1E7
:101130002285EF00702651F1C1470A203CB081455D
:10114000EF505FE401459DBF13F7870151C7C18B85
:10115000930484004146B1CB8905268597F0FA1F98
:10116000E780401F814513058401414697F0FA1F2F
:10117000E780C0247C201309C403C14593E74700DE
:101180007CA09737FB1F83A727F34A8595C79C4F01
:1011900085C78297832704089DC32285EF00102608
:1011A00009FD930720053CB071BF8145268597F066
:1011B000FA1FE780A0207DB7EF40DFF9E1BF93067B
:1011C000C4024A86A6852285EFF06FA72285EF002C
:1011D000B01CCD4769D9D5B5094785456388E70077
:1011E00093F7D70F11476396E70089450A20EF5020
:1011F0007FD97C2093E747007CA08327040881C720
:10120000930710054DB7C54779BF3C216385072675
:10121000397122DC06DE26DA4AD84ED652D43C3169
:10122000130750052A846397E70803497500173AA6
:10123000FB1F130A6AE89309C50393573900AA975D
:10124000842783270A00C1454E85B5C39C4FA5C39B
:10125000829783270A00A1C79C47B1C303250408CE
:1012600013797900B3D62441858A930505041808BB
:1012700093E606084E861305050882971375F50F49
:1012800019ED41460C081305C40297F0FA1FE780D8
:10129000600C2285EF005010930760053CB0F250BF
:1012A0006254D2544259B259225A21618280EF408D
:1012B0007FEA45B7130710026392E7021C55032724
:1012C0000508DE2361EB13F7071069C778555A2B21
:1012D0001377071061C3930770023CB03C301307CB
:1012E0007002639FE70C3C5885E393053005714518
:1012F00097F0FA1FE78080D628D819C57146814536
:1013000097F0FA1FE780800B2458A1C8BC2C89E70E
:101310002285EFF00F9EA8AC28588145414697F0F2
:10132000FA1FE780A00928583D472C2D9387F5FF29
:1013300093F7F70F6364F700EF40DFE1EF20FFFC66
:101340003C58A1458AAB13852701EF40BFE02C58DC
:101350000A20EF003034631A0510930780023CB076
:101360000A209720FB1FE7800081414609C57E25A2
:1013700013D617003E966254F250D2544259B259D5
:10138000225A1735FB1F0345D50E060685452161F8
:101390006F304F9313F7072009CB78545A2B1377EC
:1013A000072001C7930790020DBF93F707409DD711
:1013B0007C54DE2B93F7074095D39307B00231BFDF
:1013C000130780026397E7023C5899C78E2B0A20C7
:1013D00013862701EF0070311C54DE2313F707201A
:1013E00029CF78545A2B1377072021CB93079002EB
:1013F000BDB713079002639BE700EF50CF84AA8527
:101400000A20EF00902D9307A00291BF1307A002BE
:101410006390E704EF508F82AA8585470145638476
:10142000F500814505452EC6EF40DFFE2A86B24510
:101430000A20EF0030271C54DE2393F707409DC39A
:101440007C54DE2B93F7074091CF9307B00201BF86
:101450001307B0026398E700EF409FFFAA850A20B8
:10146000EF00102C9307F00215BD38309307F002FF
:10147000E318F7EE2DB58280411122C4405926C2EF
:1014800006C67C54AA84DE2B13F7071011C7185424
:101490005A23137707100DE313F7072011C71854C9
:1014A0005A231377072009EB93F707408DCB1C5481
:1014B000DE2393F7074085C7930710023CB02285CF
:1014C000EFF0BFD438309307F002631EF7002244D8
:1014D000AA20B2409244814541016FE05FC3930767
:1014E000F0023CB0EDB7B240224492444101828008
:1014F000397122DC405926DA4AD84ED606DE2A89CE
:10150000AE84B289630604382A211E206391A71293
:101510003C20638A07389387E5FF93F7F70F2D4741
:101520006363F73817D7010013074793B3C7E72062
:101530009C43BA97828722856254F250D254425912
:10154000B259B28521616FF0BFA74146CE85130520
:10155000C40497F0FA1FE780E0DF2285BD2538300C
:1015600093074005631AF700930790053335A000F1
:10157000931435003CB06DA893066005D147E3177E
:10158000D7FE9307A005DDB71309C4054A85414678
:10159000CE8597F0FA1FE780E0DB032504085DC5E0
:1015A0003C30130790056397E7002285452D93078C
:1015B000E005A5A81307A0056394E7087C3013D7BE
:1015C0003700229714279D8BB3D6F640858A97372C
:1015D000FB1F83A767AE93E60608B1CB9C47A1CB60
:1015E0009305050818084A861305050482971375A4
:1015F000F50F15ED41460C081305C40497F0FA1FCA
:10160000E780C0E67C304D47850793F7F70F7CB045
:10161000E36DF7F885451735FB1F034595E59710F2
:10162000FB1FE780803E930750053CB031A8A144E2
:10163000F25062544259B2592685D25421618280B7
:101640001307C005E383E7F68144DDB793098400FF
:101650004A86CE8522851408EFE07FDE4146930559
:10166000C404080897F0FA1FE78040E071D18A8629
:101670001306C403CA854E85EF10A06DA1440DE189
:101680002285EFE01FE72A870A209737FB1F83A7F1
:10169000E7DD814601468A858297B334A0008E0437
:1016A00093072002C1BD0C22EFE07FA671BF383046
:1016B000930720026319F71E7C5889EB93053005C8
:1016C000714597F0FA1FE780609968D86858630CF5
:1016D000051C4146CE8597F0FA1FE780A0C76458E5
:1016E0002285EFE01FE1A8AC930730023DBF383000
:1016F000930730026319F71A1E2268582146938512
:1017000029001EA9490597F0FA1FE780A0C47C5460
:10171000DE2B13F727002DC718545A23098B2DC32E
:101720009307400219B7383093074002631DF7163C
:101730003C5C81EB85455D4597F0FA1FE7800092A0
:1017400028DC285CE30205F083C709004146CE850A
:101750007CA997F0FA1FE780E0BF93075002F1B52C
:101760003830930750026310F714285C19469385AC
:101770001900410597F0FA1FE780C0BD7C54DE2BAD
:10178000918B95CF1C54DE23918B95CB93076002F0
:1017900069BD7C5C89EB93053005514597F0FA1FD4
:1017A000E780C08B68DC685CE30305E84146CE85D2
:1017B00097F0FA1FE78000BA7C5C7D5798CB4A858A
:1017C000EFF09FCB51B50325040813060004CE8526
:1017D0001305050497F0FA1FE780C0B72285EFE0F4
:1017E0005FC23C30130700056395E700930740058F
:1017F0002DBD13071005E38FE7E013072005E395E0
:10180000E7E49737FB1F83A7278BE38207E29C4718
:10181000E38F07E083250408930484001808938568
:101820000508814626862E8582970A201008A685FF
:10183000EF502FFE9307B005CDBB38309307E0057E
:101840006313F7068325040841464E8597F0FA1F77
:10185000E780C0C1AD44E30D05DC03250408414623
:10186000CE8597F0FA1FE780E0AE2285EFE07FC8D3
:101870002A872C580A209737FB1F83A727BF81464A
:1018800001468297B334A0008E0493071002DDB1A5
:10189000AD47E39BF5DA14222E21130665000821DB
:1018A000EF40DFF255B39D4461B3AA87094541C6B5
:1018B000D9C11CA29C211CB29C313CA2BC213CB2CF
:1018C000BC31A30206005CA2DE2193D787485CB23C
:1018D000DA211377072001C793E727005CB2DE21E6
:1018E00093F7074089C75C3293E747005CB2DE217B
:1018F0001317B028F98F89C75C3293E787005CB271
:1019000023030600DE21858B7CA2DA21098B01C727
:1019100093E727007CA2DE21918B89C77C2293E785
:1019200047007CA2DE21A18B89C77C2293E7870038
:101930007CA20145828082802E86AA8505456FF0B3
:10194000DFF62E86AA8509456FF03FF68DC52A87FA
:10195000094505C7411106C6AE878D4694A113857A
:1019600017004146BA8597F0FA1FE780A09EB24063
:101970000145410182800945828082808DC52A8788
:10198000094505C7411106C6AE87914694A1138546
:1019900017004146BA8597F0FA1FE780A09BB24036
:1019A0000145410182800945828082808DC52A8758
:1019B000094505C7411106C6AE87994694A113850E
:1019C00017004146BA8597F0FA1FE780A098B24009
:1019D0000145410182800945828082809DC92A8714
:1019E000094515CB411106C69D4694A11623AE8725
:1019F0001385370094B116232146A182B4A1930523
:101A0000270097F0FA1FE780E094B24001454101BA
:101A100082800945828082808DC52A87094505C755
:101A2000411106C6AE87A14694A113851700414611
:101A3000BA8597F0FA1FE780E091B2400145410175
:101A4000828009458280828085C92A8709451DC711
:101A5000411106C6A54694A11423AE87138527001D
:101A600094B119469305170097F0FA1FE780808E0E
:101A7000B2400145410182800945828082808DC546
:101A80002A87094505C7411106C6AE87A94694A114
:101A9000138517004146BA8597F0FA1FE780808BBF
:101AA000B24001454101828009458280828095C50E
:101AB0002A8709450DC7411106C6AE87B14694A1D4
:101AC0001385170013060004BA8597F0FA1FE78004
:101AD0006088B24001454101828009458280828050
:101AE0008DC52A87094505C7411106C6AE87B5468B
:101AF00094A1138517004146BA8597F0FA1FE78035
:101B00006085B24001454101828009458280828022
:101B1000AA87094581C999C7154798A19C23014502
:101B20009CB182808280AA87094581C999C72D47C7
:101B300098A19C2301459CB1828082800DC55D7176
:101B40008A8586C6A2C42A84EFE0BF870A200A8657
:101B500097060000938686DE9D45EFE0EFF9B640DC
:101B6000264461618280054582800DC55D718A854C
:101B700086C6A2C42A84EFE0DF840A200A8697067C
:101B80000000938646DC9D45EFE00FF7B640264403
:101B900061618280054582805D71A2C49305C502A2
:101BA0002A8441460A8586C697E0FA1FE780807A34
:101BB0000A200A8697060000938686D9C545EFE07D
:101BC000AFF3B6402644616182805D71A2C4930583
:101BD000C5032A8441460A8586C697E0FA1FE78036
:101BE00060770A200A8697060000938666D9C54565
:101BF000EFE08FF0B6402644616182809727FB1F9B
